 java

 Timestamp is ffffffff (Sun Feb  7 06:28:15 2106)

 Preferred load address is 10000000

 Start         Length     Name                   Class
 0001:00000000 0001138fH .text$mn                CODE
 0002:00000000 00000520H .idata$5                DATA
 0002:00000520 00000004H .00cfg                  DATA
 0002:00000524 00000004H .CRT$XCA                DATA
 0002:00000528 00000004H .CRT$XCZ                DATA
 0002:0000052c 00000004H .CRT$XIA                DATA
 0002:00000530 00000004H .CRT$XIZ                DATA
 0002:00000534 00000004H .CRT$XPA                DATA
 0002:00000538 00000004H .CRT$XPZ                DATA
 0002:0000053c 00000004H .CRT$XTA                DATA
 0002:00000540 00000010H .CRT$XTZ                DATA
 0002:00000544 00000000H .gfids$y                DATA
 0002:00000550 00001888H .rdata                  DATA
 0002:00001dd8 00000004H .rdata$sxdata           DATA
 0002:00001ddc 000002fcH .rdata$zzzdbg           DATA
 0002:000020d8 00000004H .rtc$IAA                DATA
 0002:000020dc 00000004H .rtc$IZZ                DATA
 0002:000020e0 00000004H .rtc$TAA                DATA
 0002:000020e4 00000004H .rtc$TZZ                DATA
 0002:000020e8 000000a4H .xdata$x                DATA
 0002:0000218c 00000020H .didat$2                DATA
 0002:000021ac 00000020H .didat$3                DATA
 0002:000021cc 0000000cH .didat$4                DATA
 0002:000021d8 0000002cH .didat$6                DATA
 0002:00002204 0000000cH .didat$7                DATA
 0002:00002210 00004168H .edata                  DATA
 0002:00006378 000000f0H .idata$2                DATA
 0002:00006468 00000014H .idata$3                DATA
 0002:0000647c 00000520H .idata$4                DATA
 0002:0000699c 00001d84H .idata$6                DATA
 0003:00000000 00000dbcH .data                   DATA
 0003:00000dbc 0000000cH .didat$5                DATA
 0003:00000dc8 000004bcH .bss                    DATA
 0004:00000000 00000060H .rsrc$01                DATA
 0004:00000060 00000318H .rsrc$02                DATA

  Address         Publics by Value              Rva+Base       Lib:Object

 0000:00000000       ___arm64x_native_entrypoint 00000000     <absolute>
 0000:00000000       ___hybrid_code_map_count   00000000     <absolute>
 0000:00000000       ___guard_longjmp_table     00000000     <absolute>
 0000:00000000       ___guard_fids_count        00000000     <absolute>
 0000:00000000       ___x64_code_ranges_to_entry_points 00000000     <absolute>
 0000:00000000       ___guard_iat_table         00000000     <absolute>
 0000:00000000       ___guard_eh_cont_count     00000000     <absolute>
 0000:00000000       ___arm64x_redirection_metadata 00000000     <absolute>
 0000:00000000       ___arm64x_extra_rfe_table_size 00000000     <absolute>
 0000:00000000       ___arm64x_extra_rfe_table  00000000     <absolute>
 0000:00000000       ___guard_iat_count         00000000     <absolute>
 0000:00000000       ___dynamic_value_reloc_table 00000000     <absolute>
 0000:00000000       ___hybrid_code_map         00000000     <absolute>
 0000:00000000       ___guard_longjmp_count     00000000     <absolute>
 0000:00000000       ___guard_fids_table        00000000     <absolute>
 0000:00000000       ___enclave_config          00000000     <absolute>
 0000:00000000       ___hybrid_auxiliary_iat    00000000     <absolute>
 0000:00000000       ___guard_eh_cont_table     00000000     <absolute>
 0000:00000000       ___arm64x_redirection_metadata_count 00000000     <absolute>
 0000:00000000       ___volatile_metadata       00000000     <absolute>
 0000:00000000       ___AbsoluteZero            00000000     <absolute>
 0000:00000000       ___x64_code_ranges_to_entry_points_count 00000000     <absolute>
 0000:00000001       ___safe_se_handler_count   00000001     <absolute>
 0000:00000100       ___guard_flags             00000100     <absolute>
 0000:00000000       ___ImageBase               10000000     <linker-defined>
 0001:00000000       _Java_java_security_AccessController_ensureMaterializedForStackWalk@12 10001000 f   AccessController.obj
 0001:00000003       _Java_java_security_AccessController_getInheritedAccessControlContext@8 10001003 f   AccessController.obj
 0001:00000008       _Java_java_security_AccessController_getProtectionDomain@12 10001008 f   AccessController.obj
 0001:00000018       _Java_java_security_AccessController_getStackAccessControlContext@8 10001018 f   AccessController.obj
 0001:0000001d       _Java_java_lang_reflect_Array_get@16 1000101d f   Array.obj
 0001:00000031       _Java_java_lang_reflect_Array_getBoolean@16 10001031 f   Array.obj
 0001:00000047       _Java_java_lang_reflect_Array_getByte@16 10001047 f   Array.obj
 0001:0000005d       _Java_java_lang_reflect_Array_getChar@16 1000105d f   Array.obj
 0001:00000073       _Java_java_lang_reflect_Array_getDouble@16 10001073 f   Array.obj
 0001:00000095       _Java_java_lang_reflect_Array_getFloat@16 10001095 f   Array.obj
 0001:000000b4       _Java_java_lang_reflect_Array_getInt@16 100010b4 f   Array.obj
 0001:000000ca       _Java_java_lang_reflect_Array_getLength@12 100010ca f   Array.obj
 0001:000000da       _Java_java_lang_reflect_Array_getLong@16 100010da f   Array.obj
 0001:000000f0       _Java_java_lang_reflect_Array_getShort@16 100010f0 f   Array.obj
 0001:00000106       _Java_java_lang_reflect_Array_multiNewArray@16 10001106 f   Array.obj
 0001:0000011a       _Java_java_lang_reflect_Array_newArray@16 1000111a f   Array.obj
 0001:0000012e       _Java_java_lang_reflect_Array_set@20 1000112e f   Array.obj
 0001:00000146       _Java_java_lang_reflect_Array_setBoolean@20 10001146 f   Array.obj
 0001:0000016b       _Java_java_lang_reflect_Array_setByte@20 1000116b f   Array.obj
 0001:00000190       _Java_java_lang_reflect_Array_setChar@20 10001190 f   Array.obj
 0001:000001b7       _Java_java_lang_reflect_Array_setDouble@24 100011b7 f   Array.obj
 0001:000001de       _Java_java_lang_reflect_Array_setFloat@20 100011de f   Array.obj
 0001:00000207       _Java_java_lang_reflect_Array_setInt@20 10001207 f   Array.obj
 0001:00000226       _Java_java_lang_reflect_Array_setLong@24 10001226 f   Array.obj
 0001:00000243       _Java_java_lang_reflect_Array_setShort@20 10001243 f   Array.obj
 0001:0000026a       _Java_java_util_concurrent_atomic_AtomicLong_VMSupportsCS8@8 1000126a f   AtomicLong.obj
 0001:00000272       _Java_jdk_internal_loader_BootLoader_getSystemPackageLocation@12 10001272 f   BootLoader.obj
 0001:00000282       _Java_jdk_internal_loader_BootLoader_getSystemPackageNames@8 10001282 f   BootLoader.obj
 0001:0000028e       _Java_jdk_internal_loader_BootLoader_setBootLoaderUnnamedModule0@12 1000128e f   BootLoader.obj
 0001:0000029e       _Java_jdk_internal_misc_CDS_defineArchivedModules@16 1000129e f   CDS.obj
 0001:000002b2       _Java_jdk_internal_misc_CDS_dumpClassList@12 100012b2 f   CDS.obj
 0001:000002c2       _Java_jdk_internal_misc_CDS_dumpDynamicArchive@12 100012c2 f   CDS.obj
 0001:000002d2       _Java_jdk_internal_misc_CDS_getRandomSeedForDumping@8 100012d2 f   CDS.obj
 0001:000002da       _Java_jdk_internal_misc_CDS_initializeFromArchive@12 100012da f   CDS.obj
 0001:000002ea       _Java_jdk_internal_misc_CDS_isDumpingArchive0@8 100012ea f   CDS.obj
 0001:000002f6       _Java_jdk_internal_misc_CDS_isDumpingClassList0@8 100012f6 f   CDS.obj
 0001:00000302       _Java_jdk_internal_misc_CDS_isSharingEnabled0@8 10001302 f   CDS.obj
 0001:0000030e       _Java_jdk_internal_misc_CDS_logLambdaFormInvoker@12 1000130e f   CDS.obj
 0001:0000031e       _Java_java_lang_Class_forName0@24 1000131e f   Class.obj
 0001:0000043f       _Java_java_lang_Class_getPrimitiveClass@12 1000143f f   Class.obj
 0001:00000490       _Java_java_lang_Class_isAssignableFrom@12 10001490 f   Class.obj
 0001:000004ba       _Java_java_lang_Class_isInstance@12 100014ba f   Class.obj
 0001:000004dd       _Java_java_lang_Class_registerNatives@8 100014dd f   Class.obj
 0001:00000502       _Java_java_lang_ClassLoader_defineClass0@48 10001502 f   ClassLoader.obj
 0001:0000065e       _Java_java_lang_ClassLoader_defineClass1@36 1000165e f   ClassLoader.obj
 0001:000007db       _Java_java_lang_ClassLoader_defineClass2@36 100017db f   ClassLoader.obj
 0001:00000923       _Java_java_lang_ClassLoader_findBootstrapClass@12 10001923 f   ClassLoader.obj
 0001:000009af       _Java_java_lang_ClassLoader_findLoadedClass0@12 100019af f   ClassLoader.obj
 0001:000009c0       _Java_java_lang_ClassLoader_registerNatives@8 100019c0 f   ClassLoader.obj
 0001:00000a3b       _Java_java_io_Console_echo@12 10001a3b f   Console_md.obj
 0001:00000aab       _Java_java_io_Console_encoding@8 10001aab f   Console_md.obj
 0001:00000b1c       _Java_java_io_Console_istty@8 10001b1c f   Console_md.obj
 0001:00000b7c       ___local_stdio_printf_options 10001b7c f i Console_md.obj
 0001:00000b82       __vsnprintf_l              10001b82 f i Console_md.obj
 0001:00000bb5       _sprintf                   10001bb5 f i Console_md.obj
 0001:00000bcf       _Java_jdk_internal_reflect_ConstantPool_getClassAt0@16 10001bcf f   ConstantPool.obj
 0001:00000bd4       _Java_jdk_internal_reflect_ConstantPool_getClassAtIfLoaded0@16 10001bd4 f   ConstantPool.obj
 0001:00000bd9       _Java_jdk_internal_reflect_ConstantPool_getClassRefIndexAt0@16 10001bd9 f   ConstantPool.obj
 0001:00000bde       _Java_jdk_internal_reflect_ConstantPool_getDoubleAt0@16 10001bde f   ConstantPool.obj
 0001:00000be3       _Java_jdk_internal_reflect_ConstantPool_getFieldAt0@16 10001be3 f   ConstantPool.obj
 0001:00000be8       _Java_jdk_internal_reflect_ConstantPool_getFieldAtIfLoaded0@16 10001be8 f   ConstantPool.obj
 0001:00000bed       _Java_jdk_internal_reflect_ConstantPool_getFloatAt0@16 10001bed f   ConstantPool.obj
 0001:00000bf2       _Java_jdk_internal_reflect_ConstantPool_getIntAt0@16 10001bf2 f   ConstantPool.obj
 0001:00000bf7       _Java_jdk_internal_reflect_ConstantPool_getLongAt0@16 10001bf7 f   ConstantPool.obj
 0001:00000bfc       _Java_jdk_internal_reflect_ConstantPool_getMemberRefInfoAt0@16 10001bfc f   ConstantPool.obj
 0001:00000c01       _Java_jdk_internal_reflect_ConstantPool_getMethodAt0@16 10001c01 f   ConstantPool.obj
 0001:00000c06       _Java_jdk_internal_reflect_ConstantPool_getMethodAtIfLoaded0@16 10001c06 f   ConstantPool.obj
 0001:00000c0b       _Java_jdk_internal_reflect_ConstantPool_getNameAndTypeRefIndexAt0@16 10001c0b f   ConstantPool.obj
 0001:00000c10       _Java_jdk_internal_reflect_ConstantPool_getNameAndTypeRefInfoAt0@16 10001c10 f   ConstantPool.obj
 0001:00000c15       _Java_jdk_internal_reflect_ConstantPool_getSize0@12 10001c15 f   ConstantPool.obj
 0001:00000c1a       _Java_jdk_internal_reflect_ConstantPool_getStringAt0@16 10001c1a f   ConstantPool.obj
 0001:00000c1f       _Java_jdk_internal_reflect_ConstantPool_getTagAt0@16 10001c1f f   ConstantPool.obj
 0001:00000c24       _Java_jdk_internal_reflect_ConstantPool_getUTF8At0@16 10001c24 f   ConstantPool.obj
 0001:00000c29       _Java_java_lang_Double_doubleToRawLongBits@16 10001c29 f   Double.obj
 0001:00000c40       _Java_java_lang_Double_longBitsToDouble@16 10001c40 f   Double.obj
 0001:00000c58       _Java_java_lang_reflect_Executable_getParameters0@8 10001c58 f   Executable.obj
 0001:00000c5d       _Java_java_lang_reflect_Executable_getTypeAnnotationBytes0@8 10001c5d f   Executable.obj
 0001:00000c62       _Java_java_lang_reflect_Field_getTypeAnnotationBytes0@8 10001c62 f   Field.obj
 0001:00000c67       _Java_java_io_FileCleanable_cleanupClose0@20 10001c67 f   FileDescriptor_md.obj
 0001:00000c93       _Java_java_io_FileDescriptor_close0@8 10001c93 f   FileDescriptor_md.obj
 0001:00000ca5       _Java_java_io_FileDescriptor_getAppend@12 10001ca5 f   FileDescriptor_md.obj
 0001:00000caa       _Java_java_io_FileDescriptor_getHandle@12 10001caa f   FileDescriptor_md.obj
 0001:00000cd7       _Java_java_io_FileDescriptor_initIDs@8 10001cd7 f   FileDescriptor_md.obj
 0001:00000d3c       _Java_java_io_FileDescriptor_sync@8 10001d3c f   FileDescriptor_md.obj
 0001:00000d76       _Java_java_io_FileInputStream_available0@8 10001d76 f   FileInputStream.obj
 0001:00000df9       _Java_java_io_FileInputStream_initIDs@8 10001df9 f   FileInputStream.obj
 0001:00000e1c       _Java_java_io_FileInputStream_length0@8 10001e1c f   FileInputStream.obj
 0001:00000e7f       _Java_java_io_FileInputStream_open0@12 10001e7f f   FileInputStream.obj
 0001:00000e9e       _Java_java_io_FileInputStream_position0@8 10001e9e f   FileInputStream.obj
 0001:00000f05       _Java_java_io_FileInputStream_read0@8 10001f05 f   FileInputStream.obj
 0001:00000f1e       _Java_java_io_FileInputStream_readBytes@20 10001f1e f   FileInputStream.obj
 0001:00000f42       _Java_java_io_FileInputStream_skip0@16 10001f42 f   FileInputStream.obj
 0001:00000ffb       _Java_java_io_FileOutputStream_initIDs@8 10001ffb f   FileOutputStream_md.obj
 0001:0000101e       _Java_java_io_FileOutputStream_open0@16 1000201e f   FileOutputStream_md.obj
 0001:0000104e       _Java_java_io_FileOutputStream_write@16 1000204e f   FileOutputStream_md.obj
 0001:0000106f       _Java_java_io_FileOutputStream_writeBytes@24 1000206f f   FileOutputStream_md.obj
 0001:00001096       _Java_java_lang_Float_floatToRawIntBits@12 10002096 f   Float.obj
 0001:000010aa       _Java_java_lang_Float_intBitsToFloat@12 100020aa f   Float.obj
 0001:000010ba       _EnumCalendarInfoProc@16   100020ba f   HostLocaleProviderAdapter_md.obj
 0001:000010e9       _Java_sun_util_locale_provider_HostLocaleProviderAdapterImpl_getAmPmStrings@16 100020e9 f   HostLocaleProviderAdapter_md.obj
 0001:00001112       _Java_sun_util_locale_provider_HostLocaleProviderAdapterImpl_getCalendarDataValue@16 10002112 f   HostLocaleProviderAdapter_md.obj
 0001:0000117f       _Java_sun_util_locale_provider_HostLocaleProviderAdapterImpl_getCalendarDisplayStrings@24 1000217f f   HostLocaleProviderAdapter_md.obj
 0001:00001279       _Java_sun_util_locale_provider_HostLocaleProviderAdapterImpl_getCalendarID@12 10002279 f   HostLocaleProviderAdapter_md.obj
 0001:000012b4       _Java_sun_util_locale_provider_HostLocaleProviderAdapterImpl_getCurrencySymbol@16 100022b4 f   HostLocaleProviderAdapter_md.obj
 0001:00001351       _Java_sun_util_locale_provider_HostLocaleProviderAdapterImpl_getDateTimePattern@20 10002351 f   HostLocaleProviderAdapter_md.obj
 0001:00001447       _Java_sun_util_locale_provider_HostLocaleProviderAdapterImpl_getDecimalSeparator@16 10002447 f   HostLocaleProviderAdapter_md.obj
 0001:000014cd       _Java_sun_util_locale_provider_HostLocaleProviderAdapterImpl_getDefaultLocale@12 100024cd f   HostLocaleProviderAdapter_md.obj
 0001:00001525       _Java_sun_util_locale_provider_HostLocaleProviderAdapterImpl_getDisplayString@20 10002525 f   HostLocaleProviderAdapter_md.obj
 0001:000015f4       _Java_sun_util_locale_provider_HostLocaleProviderAdapterImpl_getEras@16 100025f4 f   HostLocaleProviderAdapter_md.obj
 0001:0000160f       _Java_sun_util_locale_provider_HostLocaleProviderAdapterImpl_getGroupingSeparator@16 1000260f f   HostLocaleProviderAdapter_md.obj
 0001:00001695       _Java_sun_util_locale_provider_HostLocaleProviderAdapterImpl_getInfinity@16 10002695 f   HostLocaleProviderAdapter_md.obj
 0001:00001732       _Java_sun_util_locale_provider_HostLocaleProviderAdapterImpl_getInternationalCurrencySymbol@16 10002732 f   HostLocaleProviderAdapter_md.obj
 0001:000017cf       _Java_sun_util_locale_provider_HostLocaleProviderAdapterImpl_getMinusSign@16 100027cf f   HostLocaleProviderAdapter_md.obj
 0001:00001855       _Java_sun_util_locale_provider_HostLocaleProviderAdapterImpl_getMonetaryDecimalSeparator@16 10002855 f   HostLocaleProviderAdapter_md.obj
 0001:000018db       _Java_sun_util_locale_provider_HostLocaleProviderAdapterImpl_getMonths@16 100028db f   HostLocaleProviderAdapter_md.obj
 0001:00001905       _Java_sun_util_locale_provider_HostLocaleProviderAdapterImpl_getNaN@16 10002905 f   HostLocaleProviderAdapter_md.obj
 0001:000019a2       _Java_sun_util_locale_provider_HostLocaleProviderAdapterImpl_getNumberPattern@16 100029a2 f   HostLocaleProviderAdapter_md.obj
 0001:00001a06       _Java_sun_util_locale_provider_HostLocaleProviderAdapterImpl_getPerMill@16 10002a06 f   HostLocaleProviderAdapter_md.obj
 0001:00001a8c       _Java_sun_util_locale_provider_HostLocaleProviderAdapterImpl_getPercent@16 10002a8c f   HostLocaleProviderAdapter_md.obj
 0001:00001b12       _Java_sun_util_locale_provider_HostLocaleProviderAdapterImpl_getShortMonths@16 10002b12 f   HostLocaleProviderAdapter_md.obj
 0001:00001b3c       _Java_sun_util_locale_provider_HostLocaleProviderAdapterImpl_getShortWeekdays@16 10002b3c f   HostLocaleProviderAdapter_md.obj
 0001:00001b66       _Java_sun_util_locale_provider_HostLocaleProviderAdapterImpl_getWeekdays@16 10002b66 f   HostLocaleProviderAdapter_md.obj
 0001:00001b90       _Java_sun_util_locale_provider_HostLocaleProviderAdapterImpl_getZeroDigit@16 10002b90 f   HostLocaleProviderAdapter_md.obj
 0001:00001c16       _Java_sun_util_locale_provider_HostLocaleProviderAdapterImpl_initialize@8 10002c16 f   HostLocaleProviderAdapter_md.obj
 0001:00001c95       _Java_sun_util_locale_provider_HostLocaleProviderAdapterImpl_isNativeDigit@12 10002c95 f   HostLocaleProviderAdapter_md.obj
 0001:00001cf2       _enumCalendarInfoWrapper   10002cf2 f   HostLocaleProviderAdapter_md.obj
 0001:00001d38       _getCalendarID             10002d38 f   HostLocaleProviderAdapter_md.obj
 0001:00001d84       _getCalendarInfoWrapper    10002d84 f   HostLocaleProviderAdapter_md.obj
 0001:00001dcc       _getErasImpl               10002dcc f   HostLocaleProviderAdapter_md.obj
 0001:00002005       _getFixPart                10003005 f   HostLocaleProviderAdapter_md.obj
 0001:000020a5       _getLocaleInfoWrapper      100030a5 f   HostLocaleProviderAdapter_md.obj
 0001:000020e4       _getNumberPart             100030e4 f   HostLocaleProviderAdapter_md.obj
 0001:00002254       _getNumberPattern          10003254 f   HostLocaleProviderAdapter_md.obj
 0001:000023cc       _replaceCalendarArrayElems 100033cc f   HostLocaleProviderAdapter_md.obj
 0001:00002537       _Java_java_lang_invoke_LambdaProxyClassArchive_addToArchive@36 10003537 f   LambdaProxyClassArchive.obj
 0001:0000255b       _Java_java_lang_invoke_LambdaProxyClassArchive_findFromArchive@32 1000355b f   LambdaProxyClassArchive.obj
 0001:0000257c       _Java_java_lang_Module_addExports0@20 1000357c f   Module.obj
 0001:00002594       _Java_java_lang_Module_addExportsToAll0@16 10003594 f   Module.obj
 0001:000025a8       _Java_java_lang_Module_addExportsToAllUnnamed0@16 100035a8 f   Module.obj
 0001:000025bc       _Java_java_lang_Module_addReads0@16 100035bc f   Module.obj
 0001:000025d0       _Java_java_lang_Module_defineModule0@28 100035d0 f   Module.obj
 0001:000025ee       _Java_jdk_internal_reflect_NativeConstructorAccessorImpl_newInstance0@16 100035ee f   NativeAccessors.obj
 0001:00002602       _Java_jdk_internal_reflect_NativeMethodAccessorImpl_invoke0@20 10003602 f   NativeAccessors.obj
 0001:0000261a       _Java_jdk_internal_loader_NativeLibraries_findBuiltinLib@12 1000361a f   NativeLibraries.obj
 0001:0000271f       _Java_jdk_internal_loader_NativeLibraries_findEntry0@16 1000371f f   NativeLibraries.obj
 0001:0000278b       _Java_jdk_internal_loader_NativeLibraries_load@28 1000378b f   NativeLibraries.obj
 0001:00002974       _Java_jdk_internal_loader_NativeLibraries_unload@28 10003974 f   NativeLibraries.obj
 0001:00002b1c       _Java_java_lang_NullPointerException_getExtendedNPEMessage@8 10003b1c f   NullPointerException.obj
 0001:00002b21       _Java_java_lang_Object_getClass@8 10003b21 f   Object.obj
 0001:00002b48       _Java_java_io_ObjectStreamClass_hasStaticInitializer@12 10003b48 f   ObjectStreamClass.obj
 0001:00002bf1       _Java_java_io_ObjectStreamClass_initNative@8 10003bf1 f   ObjectStreamClass.obj
 0001:00002c15       _Java_java_lang_ref_PhantomReference_refersTo0@12 10003c15 f   PhantomReference.obj
 0001:00002c1a       _Java_java_lang_ProcessEnvironment_environmentBlock@8 10003c1a f   ProcessEnvironment_md.obj
 0001:00002d16       _Java_java_lang_ProcessHandleImpl_00024Info_info0@16 10003d16 f   ProcessHandleImpl_win.obj
 0001:00002d63       _Java_java_lang_ProcessHandleImpl_00024Info_initIDs@8 10003d63 f   ProcessHandleImpl_win.obj
 0001:00002e1a       _Java_java_lang_ProcessHandleImpl_destroy0@28 10003e1a f   ProcessHandleImpl_win.obj
 0001:00002e6b       _Java_java_lang_ProcessHandleImpl_getCurrentPid0@8 10003e6b f   ProcessHandleImpl_win.obj
 0001:00002e76       _Java_java_lang_ProcessHandleImpl_getProcessPids0@28 10003e76 f   ProcessHandleImpl_win.obj
 0001:000030ee       _Java_java_lang_ProcessHandleImpl_initNative@8 100040ee f   ProcessHandleImpl_win.obj
 0001:000030f1       _Java_java_lang_ProcessHandleImpl_isAlive0@16 100040f1 f   ProcessHandleImpl_win.obj
 0001:00003143       _Java_java_lang_ProcessHandleImpl_parent0@24 10004143 f   ProcessHandleImpl_win.obj
 0001:00003275       _Java_java_lang_ProcessHandleImpl_waitForProcessExit0@20 10004275 f   ProcessHandleImpl_win.obj
 0001:0000369b       _Java_java_lang_ProcessImpl_closeHandle@16 1000469b f   ProcessImpl_md.obj
 0001:000036a8       _Java_java_lang_ProcessImpl_create@28 100046a8 f   ProcessImpl_md.obj
 0001:000037c7       _Java_java_lang_ProcessImpl_getExitCodeProcess@16 100047c7 f   ProcessImpl_md.obj
 0001:000037f2       _Java_java_lang_ProcessImpl_getProcessId0@16 100047f2 f   ProcessImpl_md.obj
 0001:000037ff       _Java_java_lang_ProcessImpl_getStillActive@8 100047ff f   ProcessImpl_md.obj
 0001:00003807       _Java_java_lang_ProcessImpl_isProcessAlive@16 10004807 f   ProcessImpl_md.obj
 0001:00003826       _Java_java_lang_ProcessImpl_openForAtomicAppend@12 10004826 f   ProcessImpl_md.obj
 0001:00003884       _Java_java_lang_ProcessImpl_terminateProcess@16 10004884 f   ProcessImpl_md.obj
 0001:00003893       _Java_java_lang_ProcessImpl_waitForInterruptibly@16 10004893 f   ProcessImpl_md.obj
 0001:000038cc       _Java_java_lang_ProcessImpl_waitForTimeoutInterruptibly@24 100048cc f   ProcessImpl_md.obj
 0001:00003906       __vswprintf_c_l            10004906 f i ProcessImpl_md.obj
 0001:000039b0       _os_error_message          100049b0 f   ProcessImpl_md.obj
 0001:00003d4d       _swprintf                  10004d4d f i ProcessImpl_md.obj
 0001:00003e50       _Java_java_io_RandomAccessFile_getFilePointer@8 10004e50 f   RandomAccessFile.obj
 0001:00003eb7       _Java_java_io_RandomAccessFile_initIDs@8 10004eb7 f   RandomAccessFile.obj
 0001:00003eda       _Java_java_io_RandomAccessFile_length@8 10004eda f   RandomAccessFile.obj
 0001:00003f3d       _Java_java_io_RandomAccessFile_open0@16 10004f3d f   RandomAccessFile.obj
 0001:00003f92       _Java_java_io_RandomAccessFile_read0@8 10004f92 f   RandomAccessFile.obj
 0001:00003fab       _Java_java_io_RandomAccessFile_readBytes@20 10004fab f   RandomAccessFile.obj
 0001:00003fcf       _Java_java_io_RandomAccessFile_seek0@16 10004fcf f   RandomAccessFile.obj
 0001:00004039       _Java_java_io_RandomAccessFile_setLength@16 10005039 f   RandomAccessFile.obj
 0001:000040de       _Java_java_io_RandomAccessFile_write0@12 100050de f   RandomAccessFile.obj
 0001:000040fd       _Java_java_io_RandomAccessFile_writeBytes@20 100050fd f   RandomAccessFile.obj
 0001:00004123       _Java_java_lang_ref_Reference_clear0@8 10005123 f   Reference.obj
 0001:00004128       _Java_java_lang_ref_Reference_getAndClearReferencePendingList@8 10005128 f   Reference.obj
 0001:00004134       _Java_java_lang_ref_Reference_hasReferencePendingList@8 10005134 f   Reference.obj
 0001:00004140       _Java_java_lang_ref_Reference_refersTo0@12 10005140 f   Reference.obj
 0001:00004145       _Java_java_lang_ref_Reference_waitForReferencePendingList@8 10005145 f   Reference.obj
 0001:00004151       _Java_jdk_internal_reflect_Reflection_areNestMates@16 10005151 f   Reflection.obj
 0001:00004165       _Java_jdk_internal_reflect_Reflection_getCallerClass@8 10005165 f   Reflection.obj
 0001:00004171       _Java_jdk_internal_reflect_Reflection_getClassAccessFlags@12 10005171 f   Reflection.obj
 0001:00004181       _Java_java_lang_Runtime_availableProcessors@8 10005181 f   Runtime.obj
 0001:00004189       _Java_java_lang_Runtime_freeMemory@8 10005189 f   Runtime.obj
 0001:00004191       _Java_java_lang_Runtime_gc@8 10005191 f   Runtime.obj
 0001:00004199       _Java_java_lang_Runtime_maxMemory@8 10005199 f   Runtime.obj
 0001:000041a1       _Java_java_lang_Runtime_totalMemory@8 100051a1 f   Runtime.obj
 0001:000041a9       _Java_java_lang_SecurityManager_getClassContext@8 100051a9 f   SecurityManager.obj
 0001:00004249       _Java_java_lang_Shutdown_beforeHalt@8 10005249 f   Shutdown.obj
 0001:00004251       _Java_java_lang_Shutdown_halt0@12 10005251 f   Shutdown.obj
 0001:0000425d       _Java_jdk_internal_misc_Signal_findSignal0@12 1000525d f   Signal.obj
 0001:000042b0       _Java_jdk_internal_misc_Signal_handle0@20 100052b0 f   Signal.obj
 0001:000042c1       _Java_jdk_internal_misc_Signal_raise0@12 100052c1 f   Signal.obj
 0001:000042cd       _Java_java_lang_StackStreamFactory_00024AbstractStackWalker_callStackWalk@32 100052cd f   StackStreamFactory.obj
 0001:000042f1       _Java_java_lang_StackStreamFactory_00024AbstractStackWalker_fetchStackFrames@36 100052f1 f   StackStreamFactory.obj
 0001:00004318       _Java_java_lang_StackStreamFactory_checkStackWalkModes@8 10005318 f   StackStreamFactory.obj
 0001:0000431d       _Java_java_lang_StackTraceElement_initStackTraceElement@16 1000531d f   StackTraceElement.obj
 0001:00004331       _Java_java_lang_StackTraceElement_initStackTraceElements@16 10005331 f   StackTraceElement.obj
 0001:00004345       _Java_java_lang_StrictMath_IEEEremainder@24 10005345 f   StrictMath.obj
 0001:0000436a       _Java_java_lang_StrictMath_acos@16 1000536a f   StrictMath.obj
 0001:00004381       _Java_java_lang_StrictMath_asin@16 10005381 f   StrictMath.obj
 0001:00004398       _Java_java_lang_StrictMath_atan2@24 10005398 f   StrictMath.obj
 0001:000043bd       _Java_java_lang_StrictMath_atan@16 100053bd f   StrictMath.obj
 0001:000043d4       _Java_java_lang_StrictMath_cos@16 100053d4 f   StrictMath.obj
 0001:000043eb       _Java_java_lang_StrictMath_cosh@16 100053eb f   StrictMath.obj
 0001:00004402       _Java_java_lang_StrictMath_expm1@16 10005402 f   StrictMath.obj
 0001:00004419       _Java_java_lang_StrictMath_log10@16 10005419 f   StrictMath.obj
 0001:00004430       _Java_java_lang_StrictMath_log1p@16 10005430 f   StrictMath.obj
 0001:00004447       _Java_java_lang_StrictMath_log@16 10005447 f   StrictMath.obj
 0001:0000445e       _Java_java_lang_StrictMath_sin@16 1000545e f   StrictMath.obj
 0001:00004475       _Java_java_lang_StrictMath_sinh@16 10005475 f   StrictMath.obj
 0001:0000448c       _Java_java_lang_StrictMath_sqrt@16 1000548c f   StrictMath.obj
 0001:000044a3       _Java_java_lang_StrictMath_tan@16 100054a3 f   StrictMath.obj
 0001:000044ba       _Java_java_lang_StrictMath_tanh@16 100054ba f   StrictMath.obj
 0001:000044d1       _Java_java_lang_StringUTF16_isBigEndian@8 100054d1 f   String.obj
 0001:000044d6       _Java_java_lang_String_intern@8 100054d6 f   String.obj
 0001:000044db       _Java_java_lang_System_identityHashCode@12 100054db f   System.obj
 0001:000044eb       _Java_java_lang_System_mapLibraryName@12 100054eb f   System.obj
 0001:000045d9       _Java_java_lang_System_registerNatives@8 100055d9 f   System.obj
 0001:000045f4       _Java_java_lang_System_setErr0@12 100055f4 f   System.obj
 0001:0000462a       _Java_java_lang_System_setIn0@12 1000562a f   System.obj
 0001:00004660       _Java_java_lang_System_setOut0@12 10005660 f   System.obj
 0001:00004696       _Java_jdk_internal_util_SystemProps_00024Raw_platformProperties@8 10005696 f   System.obj
 0001:00004d6b       _Java_jdk_internal_util_SystemProps_00024Raw_vmProperties@8 10005d6b f   System.obj
 0001:00004d9a       _Java_java_lang_Thread_clearInterruptEvent@8 10005d9a f   Thread.obj
 0001:00004da9       _Java_java_lang_Thread_registerNatives@8 10005da9 f   Thread.obj
 0001:00004dc4       _Java_java_lang_Throwable_fillInStackTrace@12 10005dc4 f   Throwable.obj
 0001:00004dd8       _Java_java_util_TimeZone_getSystemGMTOffsetID@8 10005dd8 f   TimeZone.obj
 0001:00004e02       _Java_java_util_TimeZone_getSystemTimeZoneID@12 10005e02 f   TimeZone.obj
 0001:00004ea1       _findJavaTZ_md             10005ea1 f   TimeZone_md.obj
 0001:00004f06       _getGMTOffsetID            10005f06 f   TimeZone_md.obj
 0001:000056d9       _Java_jdk_internal_misc_VM_getRuntimeArguments@8 100066d9 f   VM.obj
 0001:000056e5       _Java_jdk_internal_misc_VM_initialize@8 100066e5 f   VM.obj
 0001:00005700       _Java_jdk_internal_misc_VM_latestUserDefinedLoader0@8 10006700 f   VM.obj
 0001:0000570c       _Java_jdk_internal_vm_VMSupport_getVMTemporaryDirectory@8 1000670c f   VMSupport.obj
 0001:00005718       _Java_jdk_internal_vm_VMSupport_initAgentProperties@12 10006718 f   VMSupport.obj
 0001:00005728       _Java_jdk_internal_misc_VM_getgid@8 10006728 f   VM_md.obj
 0001:00005728       _Java_jdk_internal_misc_VM_getegid@8 10006728 f   VM_md.obj
 0001:00005728       _Java_jdk_internal_misc_VM_geteuid@8 10006728 f   VM_md.obj
 0001:00005728       _Java_jdk_internal_misc_VM_getuid@8 10006728 f   VM_md.obj
 0001:00005730       _Java_sun_io_Win32ErrorMode_setErrorMode@16 10006730 f   Win32ErrorMode.obj
 0001:0000573f       _Java_sun_security_provider_NativeSeedGenerator_nativeGenerateSeed@12 1000673f f   WinCAPISeedGenerator.obj
 0001:000057de       _Java_java_io_WinNTFileSystem_canonicalize0@12 100067de f   WinNTFileSystem_md.obj
 0001:0000591c       _Java_java_io_WinNTFileSystem_canonicalizeWithPrefix0@16 1000691c f   WinNTFileSystem_md.obj
 0001:00005a9a       _Java_java_io_WinNTFileSystem_checkAccess@16 10006a9a f   WinNTFileSystem_md.obj
 0001:00005afe       _Java_java_io_WinNTFileSystem_createDirectory@12 10006afe f   WinNTFileSystem_md.obj
 0001:00005b3e       _Java_java_io_WinNTFileSystem_createFileExclusively@12 10006b3e f   WinNTFileSystem_md.obj
 0001:00005bda       _Java_java_io_WinNTFileSystem_delete0@12 10006bda f   WinNTFileSystem_md.obj
 0001:00005c1f       _Java_java_io_WinNTFileSystem_getBooleanAttributes@12 10006c1f f   WinNTFileSystem_md.obj
 0001:00005c78       _Java_java_io_WinNTFileSystem_getDriveDirectory@12 10006c78 f   WinNTFileSystem_md.obj
 0001:00005cd7       _Java_java_io_WinNTFileSystem_getLastModifiedTime@12 10006cd7 f   WinNTFileSystem_md.obj
 0001:00005d89       _Java_java_io_WinNTFileSystem_getLength@12 10006d89 f   WinNTFileSystem_md.obj
 0001:00005ef3       _Java_java_io_WinNTFileSystem_getNameMax0@12 10006ef3 f   WinNTFileSystem_md.obj
 0001:00005f6a       _Java_java_io_WinNTFileSystem_getSpace0@16 10006f6a f   WinNTFileSystem_md.obj
 0001:00006035       _Java_java_io_WinNTFileSystem_initIDs@8 10007035 f   WinNTFileSystem_md.obj
 0001:00006096       _Java_java_io_WinNTFileSystem_list@12 10007096 f   WinNTFileSystem_md.obj
 0001:0000635b       _Java_java_io_WinNTFileSystem_listRoots0@8 1000735b f   WinNTFileSystem_md.obj
 0001:00006364       _Java_java_io_WinNTFileSystem_rename0@16 10007364 f   WinNTFileSystem_md.obj
 0001:000063c9       _Java_java_io_WinNTFileSystem_setLastModifiedTime@20 100073c9 f   WinNTFileSystem_md.obj
 0001:0000646d       _Java_java_io_WinNTFileSystem_setPermission@24 1000746d f   WinNTFileSystem_md.obj
 0001:00006523       _Java_java_io_WinNTFileSystem_setReadOnly@12 10007523 f   WinNTFileSystem_md.obj
 0001:00006603       _getFinalAttributes        10007603 f   WinNTFileSystem_md.obj
 0001:000066a7       _getFinalAttributesIfReparsePoint 100076a7 f   WinNTFileSystem_md.obj
 0001:00006a22       _wmemmove                  10007a22 f i WinNTFileSystem_md.obj
 0001:00006a3a       _JDK_Canonicalize          10007a3a f   canonicalize_md.obj
 0001:00006adb       _getPrefixed               10007adb f   canonicalize_md.obj
 0001:00006b50       _lastErrorReportable       10007b50 f   canonicalize_md.obj
 0001:00006b89       _wcanonicalize             10007b89 f   canonicalize_md.obj
 0001:00006e0d       _wcanonicalizeWithPrefix   10007e0d f   canonicalize_md.obj
 0001:00007028       _fixClassname              10008028 f   check_classname.obj
 0001:00007283       _verifyClassname           10008283 f   check_classname.obj
 0001:000072d2       _verifyFixClassname        100082d2 f   check_classname.obj
 0001:0000733f       _JNI_OnLoad@8              1000833f f   check_version.obj
 0001:00007376       _readBytes                 10008376 f   io_util.obj
 0001:000074ae       _readSingle                100084ae f   io_util.obj
 0001:0000750a       _throwFileNotFoundException 1000850a f   io_util.obj
 0001:0000757f       _writeBytes                1000857f f   io_util.obj
 0001:000076d9       _writeSingle               100086d9 f   io_util.obj
 0001:0000773c       _currentDir                1000873c f   io_util_md.obj
 0001:000077a0       _currentDirLength          100087a0 f   io_util_md.obj
 0001:0000783d       _fileDescriptorClose       1000883d f   io_util_md.obj
 0001:000078a1       _fileOpen                  100088a1 f   io_util_md.obj
 0001:0000791a       _fileToNTPath              1000891a f   io_util_md.obj
 0001:00007946       _getFD                     10008946 f   io_util_md.obj
 0001:0000797b       _handleAppend              1000897b f   io_util_md.obj
 0001:00007996       _handleAvailable           10008996 f   io_util_md.obj
 0001:00007a31       _handleGetLength           10008a31 f   io_util_md.obj
 0001:00007a56       _handleLseek@20            10008a56 f   io_util_md.obj
 0001:00007ad8       _handleRead                10008ad8 f   io_util_md.obj
 0001:00007b18       _handleSetLength           10008b18 f   io_util_md.obj
 0001:00007c22       _handleSync                10008c22 f   io_util_md.obj
 0001:00007c42       _handleWrite               10008c42 f   io_util_md.obj
 0001:00007c5d       _pathToNTPath              10008c5d f   io_util_md.obj
 0001:00007d71       _prefixAbpath              10008d71 f   io_util_md.obj
 0001:00007de0       _winFileHandleOpen         10008de0 f   io_util_md.obj
 0001:00007ee1       _GetJavaProperties         10008ee1 f   java_props_md.obj
 0001:00008474       _GetStringPlatform         10009474 f   java_props_md.obj
 0001:00008660       ___local_stdio_scanf_options 10009660 f i java_props_md.obj
 0001:00008666       __vsscanf_l                10009666 f i java_props_md.obj
 0001:00008769       _getEncodingFromLangID     10009769 f   java_props_md.obj
 0001:00008941       _getHomeFromShell32        10009941 f   java_props_md.obj
 0001:000089f4       _getJavaIDFromLangID       100099f4 f   java_props_md.obj
 0001:00008abc       _sscanf                    10009abc f i java_props_md.obj
 0001:00008ad4       _JDK_LoadSystemLibrary     10009ad4 f   jdk_util_md.obj
 0001:00008b8b       _jio_fprintf               10009b8b f   jio.obj
 0001:00008ba1       _jio_snprintf              10009ba1 f   jio.obj
 0001:00008bbb       _GetStringPlatformChars    10009bbb f   jni_util.obj
 0001:00008bcd       _InitializeEncoding        10009bcd f   jni_util.obj
 0001:00008d8e       _JNU_CallMethodByName      10009d8e f   jni_util.obj
 0001:00008dab       _JNU_CallMethodByNameV@24  10009dab f   jni_util.obj
 0001:00008f5d       _JNU_CallStaticMethodByName 10009f5d f   jni_util.obj
 0001:000090fe       _JNU_ClassString@4         1000a0fe f   jni_util.obj
 0001:0000914b       _JNU_CopyObjectArray@16    1000a14b f   jni_util.obj
 0001:0000919f       _JNU_GetEnv@8              1000a19f f   jni_util.obj
 0001:000091b9       _JNU_GetFieldByName@20     1000a1b9 f   jni_util.obj
 0001:00009307       _JNU_GetStaticFieldByName@20 1000a307 f   jni_util.obj
 0001:0000944b       _JNU_GetStringPlatformChars@12 1000a44b f   jni_util.obj
 0001:000094cb       _JNU_IsInstanceOfByName@12 1000a4cb f   jni_util.obj
 0001:00009513       _JNU_NewObjectByName       1000a513 f   jni_util.obj
 0001:0000956f       _JNU_NewStringPlatform@8   1000a56f f   jni_util.obj
 0001:00009620       _JNU_ReleaseStringPlatformChars@12 1000a620 f   jni_util.obj
 0001:0000962e       _JNU_SetFieldByName        1000a62e f   jni_util.obj
 0001:00009799       _JNU_ThrowArrayIndexOutOfBoundsException@8 1000a799 f   jni_util.obj
 0001:000097ae       _JNU_ThrowByName@12        1000a7ae f   jni_util.obj
 0001:000097d0       _JNU_ThrowByNameWithLastError@12 1000a7d0 f   jni_util.obj
 0001:00009853       _JNU_ThrowByNameWithMessageAndLastError@12 1000a853 f   jni_util.obj
 0001:000099da       _JNU_ThrowClassNotFoundException@8 1000a9da f   jni_util.obj
 0001:000099ef       _JNU_ThrowIOException@8    1000a9ef f   jni_util.obj
 0001:00009a04       _JNU_ThrowIOExceptionWithLastError@8 1000aa04 f   jni_util.obj
 0001:00009a19       _JNU_ThrowIllegalArgumentException@8 1000aa19 f   jni_util.obj
 0001:00009a2e       _JNU_ThrowInternalError@8  1000aa2e f   jni_util.obj
 0001:00009a43       _JNU_ThrowNullPointerException@8 1000aa43 f   jni_util.obj
 0001:00009a58       _JNU_ThrowOutOfMemoryError@8 1000aa58 f   jni_util.obj
 0001:00009a6d       _JNU_ToString@8            1000aa6d f   jni_util.obj
 0001:0000a360       _buildJniFunctionName      1000b360 f   jni_util_md.obj
 0001:0000a3e4       _getErrorString@12         1000b3e4 f   jni_util_md.obj
 0001:0000a40d       _getLastErrorString@8      1000b40d f   jni_util_md.obj
 0001:0000a490       _getProcessHandle          1000b490 f   jni_util_md.obj
 0001:0000a4a0       _jacos                     1000b4a0 f   fdlibm:w_acos.obj
 0001:0000a4c0       _jasin                     1000b4c0 f   fdlibm:w_asin.obj
 0001:0000a4e0       _jatan                     1000b4e0 f   fdlibm:s_atan.obj
 0001:0000a860       _jatan2                    1000b860 f   fdlibm:w_atan2.obj
 0001:0000a890       _jcos                      1000b890 f   fdlibm:s_cos.obj
 0001:0000aa60       _jsin                      1000ba60 f   fdlibm:s_sin.obj
 0001:0000ac30       _jtan                      1000bc30 f   fdlibm:s_tan.obj
 0001:0000ad10       _jcosh                     1000bd10 f   fdlibm:w_cosh.obj
 0001:0000ad30       _jsinh                     1000bd30 f   fdlibm:w_sinh.obj
 0001:0000ad50       _jtanh                     1000bd50 f   fdlibm:s_tanh.obj
 0001:0000af10       _jlog                      1000bf10 f   fdlibm:w_log.obj
 0001:0000af30       _jlog10                    1000bf30 f   fdlibm:w_log10.obj
 0001:0000af50       _jsqrt                     1000bf50 f   fdlibm:w_sqrt.obj
 0001:0000af70       _jremainder                1000bf70 f   fdlibm:w_remainder.obj
 0001:0000afa0       _jexpm1                    1000bfa0 f   fdlibm:s_expm1.obj
 0001:0000b4d0       _jlog1p                    1000c4d0 f   fdlibm:s_log1p.obj
 0001:0000b960       ___ieee754_acos            1000c960 f   fdlibm:e_acos.obj
 0001:0000bd70       ___ieee754_asin            1000cd70 f   fdlibm:e_asin.obj
 0001:0000c110       _jfabs                     1000d110 f   fdlibm:s_fabs.obj
 0001:0000c130       ___ieee754_atan2           1000d130 f   fdlibm:e_atan2.obj
 0001:0000c560       ___ieee754_rem_pio2        1000d560 f   fdlibm:e_rem_pio2.obj
 0001:0000cb70       ___kernel_sin              1000db70 f   fdlibm:k_sin.obj
 0001:0000cc80       ___kernel_cos              1000dc80 f   fdlibm:k_cos.obj
 0001:0000cdf0       ___kernel_tan              1000ddf0 f   fdlibm:k_tan.obj
 0001:0000d230       ___ieee754_cosh            1000e230 f   fdlibm:e_cosh.obj
 0001:0000d420       ___ieee754_sinh            1000e420 f   fdlibm:e_sinh.obj
 0001:0000d630       ___ieee754_log             1000e630 f   fdlibm:e_log.obj
 0001:0000da50       ___ieee754_log10           1000ea50 f   fdlibm:e_log10.obj
 0001:0000dbc0       ___ieee754_sqrt            1000ebc0 f   fdlibm:e_sqrt.obj
 0001:0000df40       ___ieee754_remainder       1000ef40 f   fdlibm:e_remainder.obj
 0001:0000e130       ___kernel_rem_pio2         1000f130 f   fdlibm:k_rem_pio2.obj
 0001:0000ef70       ___ieee754_exp             1000ff70 f   fdlibm:e_exp.obj
 0001:0000f290       ___ieee754_fmod            10010290 f   fdlibm:e_fmod.obj
 0001:0000f700       _jfloor                    10010700 f   fdlibm:s_floor.obj
 0001:0000f8b0       _scalbn                    100108b0 f   fdlibm:s_scalbn.obj
 0001:0000faa0       _copysign                  10010aa0 f   fdlibm:s_copysign.obj
 0001:0000fabe       _JVM_GetProtectionDomain@8 10010abe f   jvm:jvm.dll
 0001:0000fac4       _JVM_GetInheritedAccessControlContext@8 10010ac4 f   jvm:jvm.dll
 0001:0000faca       _JVM_GetStackAccessControlContext@8 10010aca f   jvm:jvm.dll
 0001:0000fad0       _JVM_GetArrayLength@8      10010ad0 f   jvm:jvm.dll
 0001:0000fad6       _JVM_GetArrayElement@12    10010ad6 f   jvm:jvm.dll
 0001:0000fadc       _JVM_GetPrimitiveArrayElement@16 10010adc f   jvm:jvm.dll
 0001:0000fae2       _JVM_SetArrayElement@16    10010ae2 f   jvm:jvm.dll
 0001:0000fae8       _JVM_SetPrimitiveArrayElement@24 10010ae8 f   jvm:jvm.dll
 0001:0000faee       _JVM_NewArray@12           10010aee f   jvm:jvm.dll
 0001:0000faf4       _JVM_NewMultiArray@12      10010af4 f   jvm:jvm.dll
 0001:0000fafa       _JVM_SupportsCX8@0         10010afa f   jvm:jvm.dll
 0001:0000fb00       _JVM_GetSystemPackage@8    10010b00 f   jvm:jvm.dll
 0001:0000fb06       _JVM_GetSystemPackages@4   10010b06 f   jvm:jvm.dll
 0001:0000fb0c       _JVM_SetBootLoaderUnnamedModule@8 10010b0c f   jvm:jvm.dll
 0001:0000fb12       _JVM_InitializeFromArchive@8 10010b12 f   jvm:jvm.dll
 0001:0000fb18       _JVM_IsCDSDumpingEnabled@4 10010b18 f   jvm:jvm.dll
 0001:0000fb1e       _JVM_IsSharingEnabled@4    10010b1e f   jvm:jvm.dll
 0001:0000fb24       _JVM_IsDumpingClassList@4  10010b24 f   jvm:jvm.dll
 0001:0000fb2a       _JVM_GetRandomSeedForDumping@0 10010b2a f   jvm:jvm.dll
 0001:0000fb30       _JVM_LogLambdaFormInvoker@8 10010b30 f   jvm:jvm.dll
 0001:0000fb36       _JVM_DumpClassListToFile@8 10010b36 f   jvm:jvm.dll
 0001:0000fb3c       _JVM_DumpDynamicArchive@8  10010b3c f   jvm:jvm.dll
 0001:0000fb42       _JVM_DefineArchivedModules@12 10010b42 f   jvm:jvm.dll
 0001:0000fb48       _JVM_InitClassName@8       10010b48 f   jvm:jvm.dll
 0001:0000fb4e       _JVM_GetClassInterfaces@8  10010b4e f   jvm:jvm.dll
 0001:0000fb54       _JVM_IsInterface@8         10010b54 f   jvm:jvm.dll
 0001:0000fb5a       _JVM_GetClassSigners@8     10010b5a f   jvm:jvm.dll
 0001:0000fb60       _JVM_SetClassSigners@12    10010b60 f   jvm:jvm.dll
 0001:0000fb66       _JVM_IsArrayClass@8        10010b66 f   jvm:jvm.dll
 0001:0000fb6c       _JVM_IsPrimitiveClass@8    10010b6c f   jvm:jvm.dll
 0001:0000fb72       _JVM_IsHiddenClass@8       10010b72 f   jvm:jvm.dll
 0001:0000fb78       _JVM_GetClassModifiers@8   10010b78 f   jvm:jvm.dll
 0001:0000fb7e       _JVM_GetDeclaredClasses@8  10010b7e f   jvm:jvm.dll
 0001:0000fb84       _JVM_GetDeclaringClass@8   10010b84 f   jvm:jvm.dll
 0001:0000fb8a       _JVM_GetSimpleBinaryName@8 10010b8a f   jvm:jvm.dll
 0001:0000fb90       _JVM_GetClassSignature@8   10010b90 f   jvm:jvm.dll
 0001:0000fb96       _JVM_GetClassAnnotations@8 10010b96 f   jvm:jvm.dll
 0001:0000fb9c       _JVM_GetClassTypeAnnotations@8 10010b9c f   jvm:jvm.dll
 0001:0000fba2       _JVM_GetClassDeclaredMethods@12 10010ba2 f   jvm:jvm.dll
 0001:0000fba8       _JVM_GetClassDeclaredFields@12 10010ba8 f   jvm:jvm.dll
 0001:0000fbae       _JVM_GetClassDeclaredConstructors@12 10010bae f   jvm:jvm.dll
 0001:0000fbb4       _JVM_GetNestHost@8         10010bb4 f   jvm:jvm.dll
 0001:0000fbba       _JVM_GetNestMembers@8      10010bba f   jvm:jvm.dll
 0001:0000fbc0       _JVM_IsRecord@8            10010bc0 f   jvm:jvm.dll
 0001:0000fbc6       _JVM_GetRecordComponents@8 10010bc6 f   jvm:jvm.dll
 0001:0000fbcc       _JVM_GetPermittedSubclasses@8 10010bcc f   jvm:jvm.dll
 0001:0000fbd2       _JVM_GetClassConstantPool@8 10010bd2 f   jvm:jvm.dll
 0001:0000fbd8       _JVM_DesiredAssertionStatus@12 10010bd8 f   jvm:jvm.dll
 0001:0000fbde       _JVM_GetEnclosingMethodInfo@8 10010bde f   jvm:jvm.dll
 0001:0000fbe4       _JVM_FindPrimitiveClass@8  10010be4 f   jvm:jvm.dll
 0001:0000fbea       _JVM_FindClassFromCaller@20 10010bea f   jvm:jvm.dll
 0001:0000fbf0       _JVM_AssertionStatusDirectives@8 10010bf0 f   jvm:jvm.dll
 0001:0000fbf6       _JVM_FindClassFromBootLoader@8 10010bf6 f   jvm:jvm.dll
 0001:0000fbfc       _JVM_FindLoadedClass@12    10010bfc f   jvm:jvm.dll
 0001:0000fc02       _JVM_DefineClassWithSource@28 10010c02 f   jvm:jvm.dll
 0001:0000fc08       _JVM_LookupDefineClass@36  10010c08 f   jvm:jvm.dll
 0001:0000fc0e       _JVM_ConstantPoolGetSize@12 10010c0e f   jvm:jvm.dll
 0001:0000fc14       _JVM_ConstantPoolGetClassAt@16 10010c14 f   jvm:jvm.dll
 0001:0000fc1a       _JVM_ConstantPoolGetClassAtIfLoaded@16 10010c1a f   jvm:jvm.dll
 0001:0000fc20       _JVM_ConstantPoolGetClassRefIndexAt@16 10010c20 f   jvm:jvm.dll
 0001:0000fc26       _JVM_ConstantPoolGetMethodAt@16 10010c26 f   jvm:jvm.dll
 0001:0000fc2c       _JVM_ConstantPoolGetMethodAtIfLoaded@16 10010c2c f   jvm:jvm.dll
 0001:0000fc32       _JVM_ConstantPoolGetFieldAt@16 10010c32 f   jvm:jvm.dll
 0001:0000fc38       _JVM_ConstantPoolGetFieldAtIfLoaded@16 10010c38 f   jvm:jvm.dll
 0001:0000fc3e       _JVM_ConstantPoolGetMemberRefInfoAt@16 10010c3e f   jvm:jvm.dll
 0001:0000fc44       _JVM_ConstantPoolGetNameAndTypeRefIndexAt@16 10010c44 f   jvm:jvm.dll
 0001:0000fc4a       _JVM_ConstantPoolGetNameAndTypeRefInfoAt@16 10010c4a f   jvm:jvm.dll
 0001:0000fc50       _JVM_ConstantPoolGetIntAt@16 10010c50 f   jvm:jvm.dll
 0001:0000fc56       _JVM_ConstantPoolGetLongAt@16 10010c56 f   jvm:jvm.dll
 0001:0000fc5c       _JVM_ConstantPoolGetFloatAt@16 10010c5c f   jvm:jvm.dll
 0001:0000fc62       _JVM_ConstantPoolGetDoubleAt@16 10010c62 f   jvm:jvm.dll
 0001:0000fc68       _JVM_ConstantPoolGetStringAt@16 10010c68 f   jvm:jvm.dll
 0001:0000fc6e       _JVM_ConstantPoolGetUTF8At@16 10010c6e f   jvm:jvm.dll
 0001:0000fc74       _JVM_ConstantPoolGetTagAt@16 10010c74 f   jvm:jvm.dll
 0001:0000fc7a       _JVM_GetMethodTypeAnnotations@8 10010c7a f   jvm:jvm.dll
 0001:0000fc80       _JVM_GetMethodParameters@8 10010c80 f   jvm:jvm.dll
 0001:0000fc86       _JVM_GetFieldTypeAnnotations@8 10010c86 f   jvm:jvm.dll
 0001:0000fc8c       _JVM_RegisterLambdaProxyClassForArchiving@32 10010c8c f   jvm:jvm.dll
 0001:0000fc92       _JVM_LookupLambdaProxyClassFromArchive@28 10010c92 f   jvm:jvm.dll
 0001:0000fc98       _JVM_DefineModule@24       10010c98 f   jvm:jvm.dll
 0001:0000fc9e       _JVM_AddModuleExports@16   10010c9e f   jvm:jvm.dll
 0001:0000fca4       _JVM_AddModuleExportsToAllUnnamed@12 10010ca4 f   jvm:jvm.dll
 0001:0000fcaa       _JVM_AddModuleExportsToAll@12 10010caa f   jvm:jvm.dll
 0001:0000fcb0       _JVM_AddReadsModule@12     10010cb0 f   jvm:jvm.dll
 0001:0000fcb6       _JVM_InvokeMethod@16       10010cb6 f   jvm:jvm.dll
 0001:0000fcbc       _JVM_NewInstanceFromConstructor@12 10010cbc f   jvm:jvm.dll
 0001:0000fcc2       _JVM_LoadLibrary@8         10010cc2 f   jvm:jvm.dll
 0001:0000fcc8       _JVM_UnloadLibrary@4       10010cc8 f   jvm:jvm.dll
 0001:0000fcce       _JVM_FindLibraryEntry@8    10010cce f   jvm:jvm.dll
 0001:0000fcd4       _JVM_IsSupportedJNIVersion@4 10010cd4 f   jvm:jvm.dll
 0001:0000fcda       _JVM_GetExtendedNPEMessage@8 10010cda f   jvm:jvm.dll
 0001:0000fce0       _JVM_PhantomReferenceRefersTo@12 10010ce0 f   jvm:jvm.dll
 0001:0000fce6       _JVM_GetThreadInterruptEvent@0 10010ce6 f   jvm:jvm.dll
 0001:0000fcec       _JVM_GetAndClearReferencePendingList@4 10010cec f   jvm:jvm.dll
 0001:0000fcf2       _JVM_HasReferencePendingList@4 10010cf2 f   jvm:jvm.dll
 0001:0000fcf8       _JVM_WaitForReferencePendingList@4 10010cf8 f   jvm:jvm.dll
 0001:0000fcfe       _JVM_ReferenceRefersTo@12  10010cfe f   jvm:jvm.dll
 0001:0000fd04       _JVM_ReferenceClear@8      10010d04 f   jvm:jvm.dll
 0001:0000fd0a       _JVM_GetCallerClass@4      10010d0a f   jvm:jvm.dll
 0001:0000fd10       _JVM_GetClassAccessFlags@8 10010d10 f   jvm:jvm.dll
 0001:0000fd16       _JVM_AreNestMates@12       10010d16 f   jvm:jvm.dll
 0001:0000fd1c       _JVM_GC@0                  10010d1c f   jvm:jvm.dll
 0001:0000fd22       _JVM_TotalMemory@0         10010d22 f   jvm:jvm.dll
 0001:0000fd28       _JVM_FreeMemory@0          10010d28 f   jvm:jvm.dll
 0001:0000fd2e       _JVM_MaxMemory@0           10010d2e f   jvm:jvm.dll
 0001:0000fd34       _JVM_ActiveProcessorCount@0 10010d34 f   jvm:jvm.dll
 0001:0000fd3a       _JVM_GetClassContext@4     10010d3a f   jvm:jvm.dll
 0001:0000fd40       _JVM_BeforeHalt@0          10010d40 f   jvm:jvm.dll
 0001:0000fd46       _JVM_Halt@4                10010d46 f   jvm:jvm.dll
 0001:0000fd4c       _JVM_RegisterSignal@8      10010d4c f   jvm:jvm.dll
 0001:0000fd52       _JVM_RaiseSignal@4         10010d52 f   jvm:jvm.dll
 0001:0000fd58       _JVM_FindSignal@4          10010d58 f   jvm:jvm.dll
 0001:0000fd5e       _JVM_CallStackWalk@32      10010d5e f   jvm:jvm.dll
 0001:0000fd64       _JVM_MoreStackWalk@36      10010d64 f   jvm:jvm.dll
 0001:0000fd6a       _JVM_InitStackTraceElementArray@12 10010d6a f   jvm:jvm.dll
 0001:0000fd70       _JVM_InitStackTraceElement@12 10010d70 f   jvm:jvm.dll
 0001:0000fd76       _JVM_InternString@8        10010d76 f   jvm:jvm.dll
 0001:0000fd7c       _JVM_CurrentTimeMillis@8   10010d7c f   jvm:jvm.dll
 0001:0000fd82       _JVM_NanoTime@8            10010d82 f   jvm:jvm.dll
 0001:0000fd88       _JVM_ArrayCopy@28          10010d88 f   jvm:jvm.dll
 0001:0000fd8e       _JVM_IHashCode@8           10010d8e f   jvm:jvm.dll
 0001:0000fd94       _JVM_GetProperties@4       10010d94 f   jvm:jvm.dll
 0001:0000fd9a       _JVM_StartThread@8         10010d9a f   jvm:jvm.dll
 0001:0000fda0       _JVM_StopThread@12         10010da0 f   jvm:jvm.dll
 0001:0000fda6       _JVM_IsThreadAlive@8       10010da6 f   jvm:jvm.dll
 0001:0000fdac       _JVM_SuspendThread@8       10010dac f   jvm:jvm.dll
 0001:0000fdb2       _JVM_ResumeThread@8        10010db2 f   jvm:jvm.dll
 0001:0000fdb8       _JVM_SetThreadPriority@12  10010db8 f   jvm:jvm.dll
 0001:0000fdbe       _JVM_Yield@8               10010dbe f   jvm:jvm.dll
 0001:0000fdc4       _JVM_Sleep@16              10010dc4 f   jvm:jvm.dll
 0001:0000fdca       _JVM_CurrentThread@8       10010dca f   jvm:jvm.dll
 0001:0000fdd0       _JVM_Interrupt@8           10010dd0 f   jvm:jvm.dll
 0001:0000fdd6       _JVM_HoldsLock@12          10010dd6 f   jvm:jvm.dll
 0001:0000fddc       _JVM_GetAllThreads@8       10010ddc f   jvm:jvm.dll
 0001:0000fde2       _JVM_SetNativeThreadName@12 10010de2 f   jvm:jvm.dll
 0001:0000fde8       _JVM_DumpThreads@12        10010de8 f   jvm:jvm.dll
 0001:0000fdee       _JVM_FillInStackTrace@8    10010dee f   jvm:jvm.dll
 0001:0000fdf4       _JVM_GetNanoTimeAdjustment@16 10010df4 f   jvm:jvm.dll
 0001:0000fdfa       _JVM_GetVmArguments@4      10010dfa f   jvm:jvm.dll
 0001:0000fe00       _JVM_LatestUserDefinedLoader@4 10010e00 f   jvm:jvm.dll
 0001:0000fe06       _JVM_InitAgentProperties@8 10010e06 f   jvm:jvm.dll
 0001:0000fe0c       _JVM_GetTemporaryDirectory@4 10010e0c f   jvm:jvm.dll
 0001:0000fe12       _jio_vsnprintf             10010e12 f   jvm:jvm.dll
 0001:0000fe18       _jio_vfprintf              10010e18 f   jvm:jvm.dll
 0001:0000fe1e       __imp_load__SHGetFolderPathW@20 10010e1e f   shell32:SHELL32.dll
 0001:0000fe28       __tailMerge_shell32_dll    10010e28     shell32:SHELL32.dll
 0001:0000fe39       __imp_load__SHGetKnownFolderPath@16 10010e39 f   shell32:SHELL32.dll
 0001:0000fe43       _SHGetKnownFolderPath@16   10010e43 f   shell32:SHELL32.dll
 0001:0000fe49       ?DloadAcquireSectionWriteAccess@@YGXXZ 10010e49 f i delayimp:delayhlp.obj
 0001:0000fe7c       ?DloadGetSRWLockFunctionPointers@@YGEXZ 10010e7c f i delayimp:delayhlp.obj
 0001:0000feef       ?DloadLock@@YGXXZ          10010eef f i delayimp:delayhlp.obj
 0001:0000ff2e       ?DloadMakePermanentImageCommit@@YGXPAXK@Z 10010f2e f i delayimp:delayhlp.obj
 0001:0000ff9d       ?DloadObtainSection@@YGPAXPAK0@Z 10010f9d f i delayimp:delayhlp.obj
 0001:00010018       ?DloadProtectSection@@YGXKPAK@Z 10011018 f i delayimp:delayhlp.obj
 0001:00010086       ?DloadReleaseSectionWriteAccess@@YGXXZ 10011086 f i delayimp:delayhlp.obj
 0001:000100bc       ?DloadUnlock@@YGXXZ        100110bc f i delayimp:delayhlp.obj
 0001:000100e8       ___delayLoadHelper2@8      100110e8 f   delayimp:delayhlp.obj
 0001:00010357       _ConvertSidToStringSidW@8  10011357 f   advapi32:ADVAPI32.dll
 0001:0001035d       _GetFileVersionInfoSizeW@8 1001135d f   version:VERSION.dll
 0001:00010363       _GetFileVersionInfoW@16    10011363 f   version:VERSION.dll
 0001:00010369       _VerQueryValueW@16         10011369 f   version:VERSION.dll
 0001:0001036f       @__security_check_cookie@4 1001136f f   MSVCRT:secchk.obj
 0001:00010380       ___raise_securityfailure   10011380 f   MSVCRT:gs_report.obj
 0001:000103a8       ___report_gsfailure        100113a8 f   MSVCRT:gs_report.obj
 0001:000104a1       ___report_rangecheckfailure 100114a1 f   MSVCRT:gs_report.obj
 0001:000104ad       ___report_securityfailure  100114ad f   MSVCRT:gs_report.obj
 0001:00010580       __alldiv                   10011580 f   MSVCRT:lldiv.obj
 0001:00010630       __allmul                   10011630 f   MSVCRT:llmul.obj
 0001:00010670       __aulldiv                  10011670 f   MSVCRT:ulldiv.obj
 0001:000106e0       __chkstk                   100116e0 f   MSVCRT:chkstk.obj
 0001:000106e0       __alloca_probe             100116e0 f   MSVCRT:chkstk.obj
 0001:00010710       __SEH_prolog4_GS           10011710 f   MSVCRT:sehprolg4gs.obj
 0001:00010757       __SEH_epilog4_GS           10011757 f   MSVCRT:sehprolg4gs.obj
 0001:00010768       __except_handler4          10011768 f   MSVCRT:chandler4gs.obj
 0001:00010ad7       __DllMainCRTStartup@12     10011ad7 f   MSVCRT:dll_dllmain.obj
 0001:00010afa       @_guard_check_icall_nop@4  10011afa f i MSVCRT:guard_support.obj
 0001:00010b00       __SEH_prolog4              10011b00 f   MSVCRT:sehprolg4.obj
 0001:00010b44       __SEH_epilog4              10011b44 f   MSVCRT:sehprolg4.obj
 0001:00010ba5       ___security_init_cookie    10011ba5 f   MSVCRT:gs_support.obj
 0001:00010bf0       _DllMain@12                10011bf0 f   MSVCRT:dll_dllmain_stub.obj
 0001:00010c12       ?__scrt_initialize_type_info@@YAXXZ 10011c12 f   MSVCRT:tncleanup.obj
 0001:00010c1e       ?__scrt_uninitialize_type_info@@YAXXZ 10011c1e f   MSVCRT:tncleanup.obj
 0001:00010c2a       ___scrt_initialize_default_local_stdio_options 10011c2a f   MSVCRT:default_local_stdio_options.obj
 0001:00010c8b       ___scrt_acquire_startup_lock 10011c8b f   MSVCRT:utility.obj
 0001:00010cbd       ___scrt_dllmain_after_initialize_c 10011cbd f   MSVCRT:utility.obj
 0001:00010ce8       ___scrt_dllmain_before_initialize_c 10011ce8 f   MSVCRT:utility.obj
 0001:00010cf6       ___scrt_dllmain_crt_thread_attach 10011cf6 f   MSVCRT:utility.obj
 0001:00010d15       ___scrt_dllmain_crt_thread_detach 10011d15 f   MSVCRT:utility.obj
 0001:00010d22       ___scrt_dllmain_exception_filter 10011d22 f   MSVCRT:utility.obj
 0001:00010d56       ___scrt_dllmain_uninitialize_c 10011d56 f   MSVCRT:utility.obj
 0001:00010d79       ___scrt_dllmain_uninitialize_critical 10011d79 f   MSVCRT:utility.obj
 0001:00010d86       ___scrt_initialize_crt     10011d86 f   MSVCRT:utility.obj
 0001:00010dbf       ___scrt_initialize_onexit_tables 10011dbf f   MSVCRT:utility.obj
 0001:00010e46       ___scrt_is_nonwritable_in_current_image 10011e46 f   MSVCRT:utility.obj
 0001:00010eda       ___scrt_release_startup_lock 10011eda f   MSVCRT:utility.obj
 0001:00010ef7       ___scrt_uninitialize_crt   10011ef7 f   MSVCRT:utility.obj
 0001:00010f1f       ___scrt_get_dyn_tls_init_callback 10011f1f f   MSVCRT:dyn_tls_init.obj
 0001:00010f27       ___scrt_fastfail           10011f27 f   MSVCRT:utility_desktop.obj
 0001:00011041       __crt_debugger_hook        10012041 f   MSVCRT:utility_desktop.obj
 0001:00011049       __RTC_Initialize           10012049 f   MSVCRT:initsect.obj
 0001:00011075       __RTC_Terminate            10012075 f   MSVCRT:initsect.obj
 0001:000110a1       ___isa_available_init      100120a1 f   MSVCRT:cpu_disp.obj
 0001:00011271       __get_startup_argv_mode    10012271 f   MSVCRT:argv_mode.obj
 0001:00011275       ___scrt_is_ucrt_dll_in_use 10012275 f   MSVCRT:ucrt_detection.obj
 0001:00011281       _CreateToolhelp32Snapshot@8 10012281 f   kernel32:KERNEL32.dll
 0001:00011287       _Process32First@8          10012287 f   kernel32:KERNEL32.dll
 0001:0001128d       _Process32Next@8           1001228d f   kernel32:KERNEL32.dll
 0001:00011293       _IsProcessorFeaturePresent@4 10012293 f   kernel32:KERNEL32.dll
 0001:00011299       _memset                    10012299 f   vcruntime:VCRUNTIME140.dll
 0001:0001129f       _memcmp                    1001229f f   vcruntime:VCRUNTIME140.dll
 0001:000112a5       _memmove                   100122a5 f   vcruntime:VCRUNTIME140.dll
 0001:000112ab       _wcsrchr                   100122ab f   vcruntime:VCRUNTIME140.dll
 0001:000112b1       _wcschr                    100122b1 f   vcruntime:VCRUNTIME140.dll
 0001:000112b7       _strrchr                   100122b7 f   vcruntime:VCRUNTIME140.dll
 0001:000112bd       __except_handler4_common   100122bd f   vcruntime:VCRUNTIME140.dll
 0001:000112c3       ___std_type_info_destroy_list 100122c3 f   vcruntime:VCRUNTIME140.dll
 0001:000112c9       _strcpy                    100122c9 f   ucrt:api-ms-win-crt-string-l1-1-0.dll
 0001:000112cf       _strlen                    100122cf f   ucrt:api-ms-win-crt-string-l1-1-0.dll
 0001:000112d5       _strcat                    100122d5 f   ucrt:api-ms-win-crt-string-l1-1-0.dll
 0001:000112db       _strcmp                    100122db f   ucrt:api-ms-win-crt-string-l1-1-0.dll
 0001:000112e1       __initterm                 100122e1 f   ucrt:api-ms-win-crt-runtime-l1-1-0.dll
 0001:000112e7       __initterm_e               100122e7 f   ucrt:api-ms-win-crt-runtime-l1-1-0.dll
 0001:000112ed       __seh_filter_dll           100122ed f   ucrt:api-ms-win-crt-runtime-l1-1-0.dll
 0001:000112f3       __configure_narrow_argv    100122f3 f   ucrt:api-ms-win-crt-runtime-l1-1-0.dll
 0001:000112f9       __initialize_narrow_environment 100122f9 f   ucrt:api-ms-win-crt-runtime-l1-1-0.dll
 0001:000112ff       __initialize_onexit_table  100122ff f   ucrt:api-ms-win-crt-runtime-l1-1-0.dll
 0001:00011305       __execute_onexit_table     10012305 f   ucrt:api-ms-win-crt-runtime-l1-1-0.dll
 0001:0001130b       __cexit                    1001230b f   ucrt:api-ms-win-crt-runtime-l1-1-0.dll
 0001:00011311       __filter_x86_sse2_floating_point_exception_default 10012311 f   MSVCRT:x86_exception_filter.obj
 0001:00011311       __filter_x86_sse2_floating_point_exception 10012311 f   MSVCRT:x86_exception_filter.obj
 0001:00011389       ___acrt_thread_attach      10012389 f   MSVCRT:ucrt_stubs.obj
 0001:00011389       ___scrt_stub_for_acrt_uninitialize 10012389 f   MSVCRT:ucrt_stubs.obj
 0001:00011389       ___scrt_stub_for_acrt_initialize 10012389 f   MSVCRT:ucrt_stubs.obj
 0001:00011389       ___vcrt_initialize         10012389 f   MSVCRT:ucrt_stubs.obj
 0001:00011389       ___acrt_initialize         10012389 f   MSVCRT:ucrt_stubs.obj
 0001:00011389       ___acrt_uninitialize       10012389 f   MSVCRT:ucrt_stubs.obj
 0001:00011389       ___vcrt_uninitialize       10012389 f   MSVCRT:ucrt_stubs.obj
 0001:00011389       ___scrt_stub_for_acrt_uninitialize_critical 10012389 f   MSVCRT:ucrt_stubs.obj
 0001:00011389       ___acrt_uninitialize_critical 10012389 f   MSVCRT:ucrt_stubs.obj
 0001:00011389       ___vcrt_thread_attach      10012389 f   MSVCRT:ucrt_stubs.obj
 0001:00011389       ___vcrt_uninitialize_critical 10012389 f   MSVCRT:ucrt_stubs.obj
 0001:00011389       ___scrt_stub_for_acrt_thread_attach 10012389 f   MSVCRT:ucrt_stubs.obj
 0001:00011389       ___scrt_stub_for_acrt_thread_detach 10012389 f   MSVCRT:ucrt_stubs.obj
 0001:00011389       ___acrt_thread_detach      10012389 f   MSVCRT:ucrt_stubs.obj
 0001:00011389       ___vcrt_thread_detach      10012389 f   MSVCRT:ucrt_stubs.obj
 0001:0001138c       ___scrt_stub_for_is_c_termination_complete 1001238c f   MSVCRT:ucrt_stubs.obj
 0001:0001138c       __is_c_termination_complete 1001238c f   MSVCRT:ucrt_stubs.obj
 0002:00000000       __imp__OpenProcessToken@12 10013000     advapi32:ADVAPI32.dll
 0002:00000004       __imp__GetTokenInformation@20 10013004     advapi32:ADVAPI32.dll
 0002:00000008       __imp__LookupAccountSidW@28 10013008     advapi32:ADVAPI32.dll
 0002:0000000c       __imp__ConvertSidToStringSidW@8 1001300c     advapi32:ADVAPI32.dll
 0002:00000010       __imp__RegCloseKey@4       10013010     advapi32:ADVAPI32.dll
 0002:00000014       __imp__RegEnumKeyExA@32    10013014     advapi32:ADVAPI32.dll
 0002:00000018       __imp__RegOpenKeyExA@20    10013018     advapi32:ADVAPI32.dll
 0002:0000001c       __imp__RegOpenKeyExW@20    1001301c     advapi32:ADVAPI32.dll
 0002:00000020       __imp__RegQueryInfoKeyA@48 10013020     advapi32:ADVAPI32.dll
 0002:00000024       __imp__RegQueryValueExA@24 10013024     advapi32:ADVAPI32.dll
 0002:00000028       __imp__RegQueryValueExW@24 10013028     advapi32:ADVAPI32.dll
 0002:0000002c       __imp__CryptAcquireContextA@20 1001302c     advapi32:ADVAPI32.dll
 0002:00000030       __imp__CryptReleaseContext@8 10013030     advapi32:ADVAPI32.dll
 0002:00000034       __imp__CryptGenRandom@12   10013034     advapi32:ADVAPI32.dll
 0002:00000038       __imp__GetUserNameW@8      10013038     advapi32:ADVAPI32.dll
 0002:0000003c       \177ADVAPI32_NULL_THUNK_DATA 1001303c     advapi32:ADVAPI32.dll
 0002:00000040       __imp__GetStdHandle@4      10013040     kernel32:KERNEL32.dll
 0002:00000044       __imp__GetFileType@4       10013044     kernel32:KERNEL32.dll
 0002:00000048       __imp__GetConsoleCP@0      10013048     kernel32:KERNEL32.dll
 0002:0000004c       __imp__GetConsoleMode@8    1001304c     kernel32:KERNEL32.dll
 0002:00000050       __imp__IsDebuggerPresent@0 10013050     kernel32:KERNEL32.dll
 0002:00000054       __imp__InitializeSListHead@4 10013054     kernel32:KERNEL32.dll
 0002:00000058       __imp__DisableThreadLibraryCalls@4 10013058     kernel32:KERNEL32.dll
 0002:0000005c       __imp__GetSystemTimeAsFileTime@4 1001305c     kernel32:KERNEL32.dll
 0002:00000060       __imp__GetCurrentThreadId@0 10013060     kernel32:KERNEL32.dll
 0002:00000064       __imp__QueryPerformanceCounter@4 10013064     kernel32:KERNEL32.dll
 0002:00000068       __imp__GetCurrentProcess@0 10013068     kernel32:KERNEL32.dll
 0002:0000006c       __imp__SetUnhandledExceptionFilter@4 1001306c     kernel32:KERNEL32.dll
 0002:00000070       __imp__UnhandledExceptionFilter@4 10013070     kernel32:KERNEL32.dll
 0002:00000074       __imp__LoadLibraryExA@12   10013074     kernel32:KERNEL32.dll
 0002:00000078       __imp__GetModuleHandleW@4  10013078     kernel32:KERNEL32.dll
 0002:0000007c       __imp__FreeLibrary@4       1001307c     kernel32:KERNEL32.dll
 0002:00000080       __imp__VirtualQuery@12     10013080     kernel32:KERNEL32.dll
 0002:00000084       __imp__VirtualProtect@16   10013084     kernel32:KERNEL32.dll
 0002:00000088       __imp__RaiseException@16   10013088     kernel32:KERNEL32.dll
 0002:0000008c       __imp__FormatMessageA@28   1001308c     kernel32:KERNEL32.dll
 0002:00000090       __imp__LoadLibraryA@4      10013090     kernel32:KERNEL32.dll
 0002:00000094       __imp__GetSystemDirectoryA@8 10013094     kernel32:KERNEL32.dll
 0002:00000098       __imp__GetACP@0            10013098     kernel32:KERNEL32.dll
 0002:0000009c       __imp__IsValidCodePage@4   1001309c     kernel32:KERNEL32.dll
 0002:000000a0       __imp__GetNativeSystemInfo@4 100130a0     kernel32:KERNEL32.dll
 0002:000000a4       __imp__GetVersionExA@4     100130a4     kernel32:KERNEL32.dll
 0002:000000a8       __imp__GetWindowsDirectoryA@8 100130a8     kernel32:KERNEL32.dll
 0002:000000ac       __imp__GetSystemDirectoryW@8 100130ac     kernel32:KERNEL32.dll
 0002:000000b0       __imp__GetSystemInfo@4     100130b0     kernel32:KERNEL32.dll
 0002:000000b4       __imp__IsProcessorFeaturePresent@4 100130b4     kernel32:KERNEL32.dll
 0002:000000b8       __imp__GetTempPathW@8      100130b8     kernel32:KERNEL32.dll
 0002:000000bc       __imp__GetCurrentDirectoryW@8 100130bc     kernel32:KERNEL32.dll
 0002:000000c0       __imp__PeekConsoleInputA@16 100130c0     kernel32:KERNEL32.dll
 0002:000000c4       __imp__GetNumberOfConsoleInputEvents@8 100130c4     kernel32:KERNEL32.dll
 0002:000000c8       __imp__PeekNamedPipe@24    100130c8     kernel32:KERNEL32.dll
 0002:000000cc       __imp__WriteFile@20        100130cc     kernel32:KERNEL32.dll
 0002:000000d0       __imp__SetFilePointerEx@20 100130d0     kernel32:KERNEL32.dll
 0002:000000d4       __imp__SetFileInformationByHandle@16 100130d4     kernel32:KERNEL32.dll
 0002:000000d8       __imp__ReadFile@20         100130d8     kernel32:KERNEL32.dll
 0002:000000dc       __imp__GetFileSizeEx@8     100130dc     kernel32:KERNEL32.dll
 0002:000000e0       __imp__GetDriveTypeW@4     100130e0     kernel32:KERNEL32.dll
 0002:000000e4       __imp__FlushFileBuffers@4  100130e4     kernel32:KERNEL32.dll
 0002:000000e8       __imp__GetModuleHandleExW@12 100130e8     kernel32:KERNEL32.dll
 0002:000000ec       __imp__DeviceIoControl@32  100130ec     kernel32:KERNEL32.dll
 0002:000000f0       __imp__SetLastError@4      100130f0     kernel32:KERNEL32.dll
 0002:000000f4       __imp__SetFileTime@16      100130f4     kernel32:KERNEL32.dll
 0002:000000f8       __imp__SetFileAttributesW@8 100130f8     kernel32:KERNEL32.dll
 0002:000000fc       __imp__RemoveDirectoryW@4  100130fc     kernel32:KERNEL32.dll
 0002:00000100       __imp__GetVolumePathNameW@12 10013100     kernel32:KERNEL32.dll
 0002:00000104       __imp__GetVolumeInformationW@32 10013104     kernel32:KERNEL32.dll
 0002:00000108       __imp__GetLogicalDrives@0  10013108     kernel32:KERNEL32.dll
 0002:0000010c       __imp__GetFullPathNameW@16 1001310c     kernel32:KERNEL32.dll
 0002:00000110       __imp__GetFileTime@16      10013110     kernel32:KERNEL32.dll
 0002:00000114       __imp__GetFileInformationByHandle@8 10013114     kernel32:KERNEL32.dll
 0002:00000118       __imp__GetFileAttributesExW@12 10013118     kernel32:KERNEL32.dll
 0002:0000011c       __imp__GetFileAttributesW@4 1001311c     kernel32:KERNEL32.dll
 0002:00000120       __imp__GetDiskFreeSpaceExW@16 10013120     kernel32:KERNEL32.dll
 0002:00000124       __imp__FindNextFileW@8     10013124     kernel32:KERNEL32.dll
 0002:00000128       __imp__FindFirstFileW@8    10013128     kernel32:KERNEL32.dll
 0002:0000012c       __imp__FindClose@4         1001312c     kernel32:KERNEL32.dll
 0002:00000130       __imp__DeleteFileW@4       10013130     kernel32:KERNEL32.dll
 0002:00000134       __imp__CreateDirectoryW@8  10013134     kernel32:KERNEL32.dll
 0002:00000138       __imp__SetErrorMode@4      10013138     kernel32:KERNEL32.dll
 0002:0000013c       __imp__GetUserGeoID@4      1001313c     kernel32:KERNEL32.dll
 0002:00000140       __imp__GetGeoInfoA@20      10013140     kernel32:KERNEL32.dll
 0002:00000144       __imp__GetLocaleInfoA@16   10013144     kernel32:KERNEL32.dll
 0002:00000148       __imp__MultiByteToWideChar@24 10013148     kernel32:KERNEL32.dll
 0002:0000014c       __imp__GetDynamicTimeZoneInformation@4 1001314c     kernel32:KERNEL32.dll
 0002:00000150       __imp__GetTimeZoneInformation@4 10013150     kernel32:KERNEL32.dll
 0002:00000154       __imp__ResetEvent@4        10013154     kernel32:KERNEL32.dll
 0002:00000158       __imp__GetConsoleWindow@0  10013158     kernel32:KERNEL32.dll
 0002:0000015c       __imp__WideCharToMultiByte@32 1001315c     kernel32:KERNEL32.dll
 0002:00000160       __imp__FormatMessageW@28   10013160     kernel32:KERNEL32.dll
 0002:00000164       __imp__GetProcessId@4      10013164     kernel32:KERNEL32.dll
 0002:00000168       __imp__CreateProcessW@40   10013168     kernel32:KERNEL32.dll
 0002:0000016c       __imp__CreatePipe@16       1001316c     kernel32:KERNEL32.dll
 0002:00000170       __imp__SetHandleInformation@12 10013170     kernel32:KERNEL32.dll
 0002:00000174       __imp__GetHandleInformation@8 10013174     kernel32:KERNEL32.dll
 0002:00000178       __imp__CreateFileW@28      10013178     kernel32:KERNEL32.dll
 0002:0000017c       __imp__Process32Next@8     1001317c     kernel32:KERNEL32.dll
 0002:00000180       __imp__Process32First@8    10013180     kernel32:KERNEL32.dll
 0002:00000184       __imp__CreateToolhelp32Snapshot@8 10013184     kernel32:KERNEL32.dll
 0002:00000188       __imp__QueryFullProcessImageNameW@16 10013188     kernel32:KERNEL32.dll
 0002:0000018c       __imp__LocalFree@4         1001318c     kernel32:KERNEL32.dll
 0002:00000190       __imp__OpenProcess@12      10013190     kernel32:KERNEL32.dll
 0002:00000194       __imp__GetExitCodeProcess@8 10013194     kernel32:KERNEL32.dll
 0002:00000198       __imp__TerminateProcess@8  10013198     kernel32:KERNEL32.dll
 0002:0000019c       __imp__GetCurrentProcessId@0 1001319c     kernel32:KERNEL32.dll
 0002:000001a0       __imp__GetProcessTimes@20  100131a0     kernel32:KERNEL32.dll
 0002:000001a4       __imp__WaitForMultipleObjects@16 100131a4     kernel32:KERNEL32.dll
 0002:000001a8       __imp__GetLastError@0      100131a8     kernel32:KERNEL32.dll
 0002:000001ac       __imp__FreeEnvironmentStringsW@4 100131ac     kernel32:KERNEL32.dll
 0002:000001b0       __imp__FreeEnvironmentStringsA@4 100131b0     kernel32:KERNEL32.dll
 0002:000001b4       __imp__GetEnvironmentStringsW@0 100131b4     kernel32:KERNEL32.dll
 0002:000001b8       __imp__GetEnvironmentStrings@0 100131b8     kernel32:KERNEL32.dll
 0002:000001bc       __imp__GetUserDefaultLCID@0 100131bc     kernel32:KERNEL32.dll
 0002:000001c0       __imp__GetUserDefaultUILanguage@0 100131c0     kernel32:KERNEL32.dll
 0002:000001c4       __imp__GetProcAddress@8    100131c4     kernel32:KERNEL32.dll
 0002:000001c8       __imp__GetModuleHandleA@4  100131c8     kernel32:KERNEL32.dll
 0002:000001cc       __imp__CloseHandle@4       100131cc     kernel32:KERNEL32.dll
 0002:000001d0       __imp__SetConsoleMode@8    100131d0     kernel32:KERNEL32.dll
 0002:000001d4       \177KERNEL32_NULL_THUNK_DATA 100131d4     kernel32:KERNEL32.dll
 0002:000001d8       __imp__memset              100131d8     vcruntime:VCRUNTIME140.dll
 0002:000001dc       __imp__memcmp              100131dc     vcruntime:VCRUNTIME140.dll
 0002:000001e0       __imp__memmove             100131e0     vcruntime:VCRUNTIME140.dll
 0002:000001e4       __imp____std_type_info_destroy_list 100131e4     vcruntime:VCRUNTIME140.dll
 0002:000001e8       __imp___except_handler4_common 100131e8     vcruntime:VCRUNTIME140.dll
 0002:000001ec       __imp__wcsrchr             100131ec     vcruntime:VCRUNTIME140.dll
 0002:000001f0       __imp__wcschr              100131f0     vcruntime:VCRUNTIME140.dll
 0002:000001f4       __imp__strrchr             100131f4     vcruntime:VCRUNTIME140.dll
 0002:000001f8       \177VCRUNTIME140_NULL_THUNK_DATA 100131f8     vcruntime:VCRUNTIME140.dll
 0002:000001fc       __imp__GetFileVersionInfoW@16 100131fc     version:VERSION.dll
 0002:00000200       __imp__VerQueryValueW@16   10013200     version:VERSION.dll
 0002:00000204       __imp__GetFileVersionInfoSizeW@8 10013204     version:VERSION.dll
 0002:00000208       \177VERSION_NULL_THUNK_DATA 10013208     version:VERSION.dll
 0002:0000020c       __imp__atoi                1001320c     ucrt:api-ms-win-crt-convert-l1-1-0.dll
 0002:00000210       __imp___itoa_s             10013210     ucrt:api-ms-win-crt-convert-l1-1-0.dll
 0002:00000214       __imp__wcstombs            10013214     ucrt:api-ms-win-crt-convert-l1-1-0.dll
 0002:00000218       \177api-ms-win-crt-convert-l1-1-0_NULL_THUNK_DATA 10013218     ucrt:api-ms-win-crt-convert-l1-1-0.dll
 0002:0000021c       __imp___wgetdcwd           1001321c     ucrt:api-ms-win-crt-environment-l1-1-0.dll
 0002:00000220       __imp___wgetcwd            10013220     ucrt:api-ms-win-crt-environment-l1-1-0.dll
 0002:00000224       __imp___wgetenv            10013224     ucrt:api-ms-win-crt-environment-l1-1-0.dll
 0002:00000228       \177api-ms-win-crt-environment-l1-1-0_NULL_THUNK_DATA 10013228     ucrt:api-ms-win-crt-environment-l1-1-0.dll
 0002:0000022c       __imp___wfullpath          1001322c     ucrt:api-ms-win-crt-filesystem-l1-1-0.dll
 0002:00000230       __imp___wrename            10013230     ucrt:api-ms-win-crt-filesystem-l1-1-0.dll
 0002:00000234       \177api-ms-win-crt-filesystem-l1-1-0_NULL_THUNK_DATA 10013234     ucrt:api-ms-win-crt-filesystem-l1-1-0.dll
 0002:00000238       __imp__realloc             10013238     ucrt:api-ms-win-crt-heap-l1-1-0.dll
 0002:0000023c       __imp__malloc              1001323c     ucrt:api-ms-win-crt-heap-l1-1-0.dll
 0002:00000240       __imp__free                10013240     ucrt:api-ms-win-crt-heap-l1-1-0.dll
 0002:00000244       \177api-ms-win-crt-heap-l1-1-0_NULL_THUNK_DATA 10013244     ucrt:api-ms-win-crt-heap-l1-1-0.dll
 0002:00000248       __imp___initialize_onexit_table 10013248     ucrt:api-ms-win-crt-runtime-l1-1-0.dll
 0002:0000024c       __imp___initialize_narrow_environment 1001324c     ucrt:api-ms-win-crt-runtime-l1-1-0.dll
 0002:00000250       __imp___configure_narrow_argv 10013250     ucrt:api-ms-win-crt-runtime-l1-1-0.dll
 0002:00000254       __imp___execute_onexit_table 10013254     ucrt:api-ms-win-crt-runtime-l1-1-0.dll
 0002:00000258       __imp___initterm_e         10013258     ucrt:api-ms-win-crt-runtime-l1-1-0.dll
 0002:0000025c       __imp___initterm           1001325c     ucrt:api-ms-win-crt-runtime-l1-1-0.dll
 0002:00000260       __imp__strerror_s          10013260     ucrt:api-ms-win-crt-runtime-l1-1-0.dll
 0002:00000264       __imp___cexit              10013264     ucrt:api-ms-win-crt-runtime-l1-1-0.dll
 0002:00000268       __imp___errno              10013268     ucrt:api-ms-win-crt-runtime-l1-1-0.dll
 0002:0000026c       __imp___seh_filter_dll     1001326c     ucrt:api-ms-win-crt-runtime-l1-1-0.dll
 0002:00000270       \177api-ms-win-crt-runtime-l1-1-0_NULL_THUNK_DATA 10013270     ucrt:api-ms-win-crt-runtime-l1-1-0.dll
 0002:00000274       __imp____stdio_common_vswprintf 10013274     ucrt:api-ms-win-crt-stdio-l1-1-0.dll
 0002:00000278       __imp__fopen               10013278     ucrt:api-ms-win-crt-stdio-l1-1-0.dll
 0002:0000027c       __imp____stdio_common_vsscanf 1001327c     ucrt:api-ms-win-crt-stdio-l1-1-0.dll
 0002:00000280       __imp____acrt_iob_func     10013280     ucrt:api-ms-win-crt-stdio-l1-1-0.dll
 0002:00000284       __imp__fclose              10013284     ucrt:api-ms-win-crt-stdio-l1-1-0.dll
 0002:00000288       __imp__fgets               10013288     ucrt:api-ms-win-crt-stdio-l1-1-0.dll
 0002:0000028c       __imp____stdio_common_vsprintf 1001328c     ucrt:api-ms-win-crt-stdio-l1-1-0.dll
 0002:00000290       \177api-ms-win-crt-stdio-l1-1-0_NULL_THUNK_DATA 10013290     ucrt:api-ms-win-crt-stdio-l1-1-0.dll
 0002:00000294       __imp__iswctype            10013294     ucrt:api-ms-win-crt-string-l1-1-0.dll
 0002:00000298       __imp__wcsncmp             10013298     ucrt:api-ms-win-crt-string-l1-1-0.dll
 0002:0000029c       __imp___wcsupr             1001329c     ucrt:api-ms-win-crt-string-l1-1-0.dll
 0002:000002a0       __imp__towupper            100132a0     ucrt:api-ms-win-crt-string-l1-1-0.dll
 0002:000002a4       __imp__wcsncat             100132a4     ucrt:api-ms-win-crt-string-l1-1-0.dll
 0002:000002a8       __imp__strcmp              100132a8     ucrt:api-ms-win-crt-string-l1-1-0.dll
 0002:000002ac       __imp__strcat              100132ac     ucrt:api-ms-win-crt-string-l1-1-0.dll
 0002:000002b0       __imp__strncpy             100132b0     ucrt:api-ms-win-crt-string-l1-1-0.dll
 0002:000002b4       __imp__wcscat              100132b4     ucrt:api-ms-win-crt-string-l1-1-0.dll
 0002:000002b8       __imp__strlen              100132b8     ucrt:api-ms-win-crt-string-l1-1-0.dll
 0002:000002bc       __imp__strcpy              100132bc     ucrt:api-ms-win-crt-string-l1-1-0.dll
 0002:000002c0       __imp__wcslen              100132c0     ucrt:api-ms-win-crt-string-l1-1-0.dll
 0002:000002c4       __imp__wcscpy              100132c4     ucrt:api-ms-win-crt-string-l1-1-0.dll
 0002:000002c8       __imp__wcscmp              100132c8     ucrt:api-ms-win-crt-string-l1-1-0.dll
 0002:000002cc       __imp___wcsdup             100132cc     ucrt:api-ms-win-crt-string-l1-1-0.dll
 0002:000002d0       __imp__wcscat_s            100132d0     ucrt:api-ms-win-crt-string-l1-1-0.dll
 0002:000002d4       __imp___strdup             100132d4     ucrt:api-ms-win-crt-string-l1-1-0.dll
 0002:000002d8       \177api-ms-win-crt-string-l1-1-0_NULL_THUNK_DATA 100132d8     ucrt:api-ms-win-crt-string-l1-1-0.dll
 0002:000002dc       __imp__JVM_WaitForReferencePendingList@4 100132dc     jvm:jvm.dll
 0002:000002e0       __imp__JVM_HasReferencePendingList@4 100132e0     jvm:jvm.dll
 0002:000002e4       __imp__JVM_GetAndClearReferencePendingList@4 100132e4     jvm:jvm.dll
 0002:000002e8       __imp__JVM_GetThreadInterruptEvent@0 100132e8     jvm:jvm.dll
 0002:000002ec       __imp__JVM_PhantomReferenceRefersTo@12 100132ec     jvm:jvm.dll
 0002:000002f0       __imp__JVM_GetExtendedNPEMessage@8 100132f0     jvm:jvm.dll
 0002:000002f4       __imp__JVM_IsSupportedJNIVersion@4 100132f4     jvm:jvm.dll
 0002:000002f8       __imp__JVM_FindLibraryEntry@8 100132f8     jvm:jvm.dll
 0002:000002fc       __imp__JVM_UnloadLibrary@4 100132fc     jvm:jvm.dll
 0002:00000300       __imp__JVM_LoadLibrary@8   10013300     jvm:jvm.dll
 0002:00000304       __imp__JVM_NewInstanceFromConstructor@12 10013304     jvm:jvm.dll
 0002:00000308       __imp__JVM_InvokeMethod@16 10013308     jvm:jvm.dll
 0002:0000030c       __imp__JVM_AddReadsModule@12 1001330c     jvm:jvm.dll
 0002:00000310       __imp__JVM_AddModuleExportsToAll@12 10013310     jvm:jvm.dll
 0002:00000314       __imp__JVM_AddModuleExportsToAllUnnamed@12 10013314     jvm:jvm.dll
 0002:00000318       __imp__JVM_AddModuleExports@16 10013318     jvm:jvm.dll
 0002:0000031c       __imp__JVM_DefineModule@24 1001331c     jvm:jvm.dll
 0002:00000320       __imp__JVM_LookupLambdaProxyClassFromArchive@28 10013320     jvm:jvm.dll
 0002:00000324       __imp__JVM_RegisterLambdaProxyClassForArchiving@32 10013324     jvm:jvm.dll
 0002:00000328       __imp__JVM_GetFieldTypeAnnotations@8 10013328     jvm:jvm.dll
 0002:0000032c       __imp__JVM_GetMethodParameters@8 1001332c     jvm:jvm.dll
 0002:00000330       __imp__JVM_GetMethodTypeAnnotations@8 10013330     jvm:jvm.dll
 0002:00000334       __imp__JVM_ConstantPoolGetTagAt@16 10013334     jvm:jvm.dll
 0002:00000338       __imp__JVM_ConstantPoolGetUTF8At@16 10013338     jvm:jvm.dll
 0002:0000033c       __imp__JVM_ConstantPoolGetStringAt@16 1001333c     jvm:jvm.dll
 0002:00000340       __imp__JVM_ConstantPoolGetDoubleAt@16 10013340     jvm:jvm.dll
 0002:00000344       __imp__JVM_ConstantPoolGetFloatAt@16 10013344     jvm:jvm.dll
 0002:00000348       __imp__JVM_ConstantPoolGetLongAt@16 10013348     jvm:jvm.dll
 0002:0000034c       __imp__JVM_ConstantPoolGetIntAt@16 1001334c     jvm:jvm.dll
 0002:00000350       __imp__JVM_ConstantPoolGetNameAndTypeRefInfoAt@16 10013350     jvm:jvm.dll
 0002:00000354       __imp__JVM_ConstantPoolGetNameAndTypeRefIndexAt@16 10013354     jvm:jvm.dll
 0002:00000358       __imp__JVM_ConstantPoolGetMemberRefInfoAt@16 10013358     jvm:jvm.dll
 0002:0000035c       __imp__JVM_ConstantPoolGetFieldAtIfLoaded@16 1001335c     jvm:jvm.dll
 0002:00000360       __imp__JVM_ConstantPoolGetFieldAt@16 10013360     jvm:jvm.dll
 0002:00000364       __imp__JVM_ConstantPoolGetMethodAtIfLoaded@16 10013364     jvm:jvm.dll
 0002:00000368       __imp__JVM_ConstantPoolGetMethodAt@16 10013368     jvm:jvm.dll
 0002:0000036c       __imp__JVM_ConstantPoolGetClassRefIndexAt@16 1001336c     jvm:jvm.dll
 0002:00000370       __imp__JVM_ConstantPoolGetClassAtIfLoaded@16 10013370     jvm:jvm.dll
 0002:00000374       __imp__JVM_ConstantPoolGetClassAt@16 10013374     jvm:jvm.dll
 0002:00000378       __imp__JVM_ConstantPoolGetSize@12 10013378     jvm:jvm.dll
 0002:0000037c       __imp__JVM_LookupDefineClass@36 1001337c     jvm:jvm.dll
 0002:00000380       __imp__JVM_DefineClassWithSource@28 10013380     jvm:jvm.dll
 0002:00000384       __imp__JVM_FindLoadedClass@12 10013384     jvm:jvm.dll
 0002:00000388       __imp__JVM_FindClassFromBootLoader@8 10013388     jvm:jvm.dll
 0002:0000038c       __imp__JVM_AssertionStatusDirectives@8 1001338c     jvm:jvm.dll
 0002:00000390       __imp__JVM_FindClassFromCaller@20 10013390     jvm:jvm.dll
 0002:00000394       __imp__JVM_FindPrimitiveClass@8 10013394     jvm:jvm.dll
 0002:00000398       __imp__JVM_StartThread@8   10013398     jvm:jvm.dll
 0002:0000039c       __imp__JVM_GetProtectionDomain@8 1001339c     jvm:jvm.dll
 0002:000003a0       __imp__JVM_GetClassConstantPool@8 100133a0     jvm:jvm.dll
 0002:000003a4       __imp__JVM_GetPermittedSubclasses@8 100133a4     jvm:jvm.dll
 0002:000003a8       __imp__JVM_GetRecordComponents@8 100133a8     jvm:jvm.dll
 0002:000003ac       __imp__JVM_IsRecord@8      100133ac     jvm:jvm.dll
 0002:000003b0       __imp__JVM_GetNestMembers@8 100133b0     jvm:jvm.dll
 0002:000003b4       __imp__JVM_GetNestHost@8   100133b4     jvm:jvm.dll
 0002:000003b8       __imp__JVM_GetClassDeclaredConstructors@12 100133b8     jvm:jvm.dll
 0002:000003bc       __imp__JVM_GetClassDeclaredFields@12 100133bc     jvm:jvm.dll
 0002:000003c0       __imp__JVM_ReferenceRefersTo@12 100133c0     jvm:jvm.dll
 0002:000003c4       __imp__JVM_GetClassTypeAnnotations@8 100133c4     jvm:jvm.dll
 0002:000003c8       __imp__JVM_GetClassAnnotations@8 100133c8     jvm:jvm.dll
 0002:000003cc       __imp__JVM_GetClassSignature@8 100133cc     jvm:jvm.dll
 0002:000003d0       __imp__JVM_GetSimpleBinaryName@8 100133d0     jvm:jvm.dll
 0002:000003d4       __imp__JVM_GetDeclaringClass@8 100133d4     jvm:jvm.dll
 0002:000003d8       __imp__JVM_GetDeclaredClasses@8 100133d8     jvm:jvm.dll
 0002:000003dc       __imp__JVM_GetClassModifiers@8 100133dc     jvm:jvm.dll
 0002:000003e0       __imp__JVM_IsHiddenClass@8 100133e0     jvm:jvm.dll
 0002:000003e4       __imp__JVM_IsPrimitiveClass@8 100133e4     jvm:jvm.dll
 0002:000003e8       __imp__JVM_IsArrayClass@8  100133e8     jvm:jvm.dll
 0002:000003ec       __imp__JVM_SetClassSigners@12 100133ec     jvm:jvm.dll
 0002:000003f0       __imp__JVM_GetClassSigners@8 100133f0     jvm:jvm.dll
 0002:000003f4       __imp__JVM_IsInterface@8   100133f4     jvm:jvm.dll
 0002:000003f8       __imp__JVM_GetClassInterfaces@8 100133f8     jvm:jvm.dll
 0002:000003fc       __imp__JVM_InitClassName@8 100133fc     jvm:jvm.dll
 0002:00000400       __imp__JVM_DefineArchivedModules@12 10013400     jvm:jvm.dll
 0002:00000404       __imp__JVM_DumpDynamicArchive@8 10013404     jvm:jvm.dll
 0002:00000408       __imp__JVM_DumpClassListToFile@8 10013408     jvm:jvm.dll
 0002:0000040c       __imp__JVM_LogLambdaFormInvoker@8 1001340c     jvm:jvm.dll
 0002:00000410       __imp__JVM_GetRandomSeedForDumping@0 10013410     jvm:jvm.dll
 0002:00000414       __imp__JVM_IsDumpingClassList@4 10013414     jvm:jvm.dll
 0002:00000418       __imp__JVM_IsSharingEnabled@4 10013418     jvm:jvm.dll
 0002:0000041c       __imp__JVM_IsCDSDumpingEnabled@4 1001341c     jvm:jvm.dll
 0002:00000420       __imp__JVM_InitializeFromArchive@8 10013420     jvm:jvm.dll
 0002:00000424       __imp__JVM_SetBootLoaderUnnamedModule@8 10013424     jvm:jvm.dll
 0002:00000428       __imp__JVM_GetSystemPackages@4 10013428     jvm:jvm.dll
 0002:0000042c       __imp__JVM_GetSystemPackage@8 1001342c     jvm:jvm.dll
 0002:00000430       __imp__JVM_SupportsCX8@0   10013430     jvm:jvm.dll
 0002:00000434       __imp__JVM_NewMultiArray@12 10013434     jvm:jvm.dll
 0002:00000438       __imp__JVM_NewArray@12     10013438     jvm:jvm.dll
 0002:0000043c       __imp__JVM_StopThread@12   1001343c     jvm:jvm.dll
 0002:00000440       __imp__JVM_IsThreadAlive@8 10013440     jvm:jvm.dll
 0002:00000444       __imp__JVM_ReferenceClear@8 10013444     jvm:jvm.dll
 0002:00000448       __imp__JVM_GetCallerClass@4 10013448     jvm:jvm.dll
 0002:0000044c       __imp__JVM_GetClassAccessFlags@8 1001344c     jvm:jvm.dll
 0002:00000450       __imp__JVM_AreNestMates@12 10013450     jvm:jvm.dll
 0002:00000454       __imp__JVM_GC@0            10013454     jvm:jvm.dll
 0002:00000458       __imp__JVM_TotalMemory@0   10013458     jvm:jvm.dll
 0002:0000045c       __imp__JVM_FreeMemory@0    1001345c     jvm:jvm.dll
 0002:00000460       __imp__JVM_MaxMemory@0     10013460     jvm:jvm.dll
 0002:00000464       __imp__JVM_ActiveProcessorCount@0 10013464     jvm:jvm.dll
 0002:00000468       __imp__JVM_GetClassContext@4 10013468     jvm:jvm.dll
 0002:0000046c       __imp__JVM_BeforeHalt@0    1001346c     jvm:jvm.dll
 0002:00000470       __imp__JVM_Halt@4          10013470     jvm:jvm.dll
 0002:00000474       __imp__JVM_RegisterSignal@8 10013474     jvm:jvm.dll
 0002:00000478       __imp__JVM_RaiseSignal@4   10013478     jvm:jvm.dll
 0002:0000047c       __imp__JVM_FindSignal@4    1001347c     jvm:jvm.dll
 0002:00000480       __imp__JVM_CallStackWalk@32 10013480     jvm:jvm.dll
 0002:00000484       __imp__JVM_MoreStackWalk@36 10013484     jvm:jvm.dll
 0002:00000488       __imp__JVM_SetPrimitiveArrayElement@24 10013488     jvm:jvm.dll
 0002:0000048c       __imp__JVM_SuspendThread@8 1001348c     jvm:jvm.dll
 0002:00000490       __imp__JVM_ResumeThread@8  10013490     jvm:jvm.dll
 0002:00000494       __imp__JVM_InitStackTraceElementArray@12 10013494     jvm:jvm.dll
 0002:00000498       __imp__JVM_InitStackTraceElement@12 10013498     jvm:jvm.dll
 0002:0000049c       __imp__JVM_InternString@8  1001349c     jvm:jvm.dll
 0002:000004a0       __imp__JVM_SetThreadPriority@12 100134a0     jvm:jvm.dll
 0002:000004a4       __imp__JVM_Yield@8         100134a4     jvm:jvm.dll
 0002:000004a8       __imp__JVM_CurrentTimeMillis@8 100134a8     jvm:jvm.dll
 0002:000004ac       __imp__JVM_Sleep@16        100134ac     jvm:jvm.dll
 0002:000004b0       __imp__JVM_SetArrayElement@16 100134b0     jvm:jvm.dll
 0002:000004b4       __imp__JVM_GetPrimitiveArrayElement@16 100134b4     jvm:jvm.dll
 0002:000004b8       __imp__JVM_NanoTime@8      100134b8     jvm:jvm.dll
 0002:000004bc       __imp__JVM_ArrayCopy@28    100134bc     jvm:jvm.dll
 0002:000004c0       __imp__JVM_GetArrayElement@12 100134c0     jvm:jvm.dll
 0002:000004c4       __imp__JVM_GetArrayLength@8 100134c4     jvm:jvm.dll
 0002:000004c8       __imp__JVM_GetStackAccessControlContext@8 100134c8     jvm:jvm.dll
 0002:000004cc       __imp__JVM_CurrentThread@8 100134cc     jvm:jvm.dll
 0002:000004d0       __imp__JVM_IHashCode@8     100134d0     jvm:jvm.dll
 0002:000004d4       __imp__JVM_Interrupt@8     100134d4     jvm:jvm.dll
 0002:000004d8       __imp__JVM_HoldsLock@12    100134d8     jvm:jvm.dll
 0002:000004dc       __imp__JVM_GetAllThreads@8 100134dc     jvm:jvm.dll
 0002:000004e0       __imp__JVM_SetNativeThreadName@12 100134e0     jvm:jvm.dll
 0002:000004e4       __imp__JVM_DumpThreads@12  100134e4     jvm:jvm.dll
 0002:000004e8       __imp__JVM_FillInStackTrace@8 100134e8     jvm:jvm.dll
 0002:000004ec       __imp__JVM_GetNanoTimeAdjustment@16 100134ec     jvm:jvm.dll
 0002:000004f0       __imp__JVM_GetVmArguments@4 100134f0     jvm:jvm.dll
 0002:000004f4       __imp__JVM_LatestUserDefinedLoader@4 100134f4     jvm:jvm.dll
 0002:000004f8       __imp__JVM_InitAgentProperties@8 100134f8     jvm:jvm.dll
 0002:000004fc       __imp__JVM_GetTemporaryDirectory@4 100134fc     jvm:jvm.dll
 0002:00000500       __imp__jio_vsnprintf       10013500     jvm:jvm.dll
 0002:00000504       __imp__jio_vfprintf        10013504     jvm:jvm.dll
 0002:00000508       __imp__JVM_GetClassDeclaredMethods@12 10013508     jvm:jvm.dll
 0002:0000050c       __imp__JVM_GetProperties@4 1001350c     jvm:jvm.dll
 0002:00000510       __imp__JVM_GetInheritedAccessControlContext@8 10013510     jvm:jvm.dll
 0002:00000514       __imp__JVM_GetEnclosingMethodInfo@8 10013514     jvm:jvm.dll
 0002:00000518       __imp__JVM_DesiredAssertionStatus@12 10013518     jvm:jvm.dll
 0002:0000051c       \177jvm_NULL_THUNK_DATA    1001351c     jvm:jvm.dll
 0002:00000520       ___guard_check_icall_fptr  10013520     MSVCRT:guard_support.obj
 0002:00000524       ___xc_a                    10013524     MSVCRT:initializers.obj
 0002:00000528       ___xc_z                    10013528     MSVCRT:initializers.obj
 0002:0000052c       ___xi_a                    1001352c     MSVCRT:initializers.obj
 0002:00000530       ___xi_z                    10013530     MSVCRT:initializers.obj
 0002:00000534       ___xp_a                    10013534     MSVCRT:initializers.obj
 0002:00000538       ___xp_z                    10013538     MSVCRT:initializers.obj
 0002:0000053c       ___xt_a                    1001353c     MSVCRT:initializers.obj
 0002:00000540       ___xt_z                    10013540     MSVCRT:initializers.obj
 0002:00000550       ??_C@_0O@LMKLDNGH@initClassName@ 10013550     Class.obj
 0002:00000560       ??_C@_0BF@FOHFOJOB@?$CI?$CJLjava?1lang?1String?$DL@ 10013560     Class.obj
 0002:00000578       ??_C@_0O@BCDKKCAE@getSuperclass@ 10013578     Class.obj
 0002:00000588       ??_C@_0BE@IIFEGCLG@?$CI?$CJLjava?1lang?1Class?$DL@ 10013588     Class.obj
 0002:0000059c       ??_C@_0P@FLDOEJHK@getInterfaces0@ 1001359c     Class.obj
 0002:000005ac       ??_C@_0BF@BNKCIMJP@?$CI?$CJ?$FLLjava?1lang?1Class?$DL@ 100135ac     Class.obj
 0002:000005c4       ??_C@_0M@NAJCIFFF@isInterface@ 100135c4     Class.obj
 0002:000005d0       ??_C@_03MMPFGPID@?$CI?$CJZ@ 100135d0     Class.obj
 0002:000005d4       ??_C@_0L@NOPNAKKC@getSigners@ 100135d4     Class.obj
 0002:000005e0       ??_C@_0BG@PFDHKCPA@?$CI?$CJ?$FLLjava?1lang?1Object?$DL@ 100135e0     Class.obj
 0002:000005f8       ??_C@_0L@MANCLNOL@setSigners@ 100135f8     Class.obj
 0002:00000604       ??_C@_0BH@JBNAJHIH@?$CI?$FLLjava?1lang?1Object?$DL?$CJV@ 10013604     Class.obj
 0002:0000061c       ??_C@_07LJDBDAGJ@isArray@  1001361c     Class.obj
 0002:00000624       ??_C@_08POGCNBGK@isHidden@ 10013624     Class.obj
 0002:00000630       ??_C@_0M@DJOEILEB@isPrimitive@ 10013630     Class.obj
 0002:0000063c       ??_C@_0N@MKAAFCEB@getModifiers@ 1001363c     Class.obj
 0002:0000064c       ??_C@_03KNBKCOBB@?$CI?$CJI@ 1001364c     Class.obj
 0002:00000650       ??_C@_0BD@BEKBHNDA@getDeclaredFields0@ 10013650     Class.obj
 0002:00000664       ??_C@_0BO@KFNILMGC@?$CIZ?$CJ?$FLLjava?1lang?1reflect?1Field?$DL@ 10013664     Class.obj
 0002:00000684       ??_C@_0BE@LOILJEHC@getDeclaredMethods0@ 10013684     Class.obj
 0002:00000698       ??_C@_0BP@IIIKNIKA@?$CIZ?$CJ?$FLLjava?1lang?1reflect?1Method?$DL@ 10013698     Class.obj
 0002:000006b8       ??_C@_0BJ@KLPKFLFA@getDeclaredConstructors0@ 100136b8     Class.obj
 0002:000006d4       ??_C@_0CE@FDMOFPI@?$CIZ?$CJ?$FLLjava?1lang?1reflect?1Construc@ 100136d4     Class.obj
 0002:000006f8       ??_C@_0BF@CGNPOFHG@getProtectionDomain0@ 100136f8     Class.obj
 0002:00000710       ??_C@_0CD@LEMBAENN@?$CI?$CJLjava?1security?1ProtectionDoma@ 10013710     Class.obj
 0002:00000734       ??_C@_0BE@CIFNAIBM@getDeclaredClasses0@ 10013734     Class.obj
 0002:00000748       ??_C@_0BD@NHPDOJGF@getDeclaringClass0@ 10013748     Class.obj
 0002:0000075c       ??_C@_0BF@ODCBBOMF@getSimpleBinaryName0@ 1001375c     Class.obj
 0002:00000774       ??_C@_0BF@KFMFPKNK@getGenericSignature0@ 10013774     Class.obj
 0002:0000078c       ??_C@_0BC@CDJDGCDH@getRawAnnotations@ 1001378c     Class.obj
 0002:000007a0       ??_C@_04LHPAGAEF@?$CI?$CJ?$FLB@ 100137a0     Class.obj
 0002:000007a8       ??_C@_0BA@DLHKEBGM@getConstantPool@ 100137a8     Class.obj
 0002:000007b8       ??_C@_0CG@OKGFDDJA@?$CI?$CJLjdk?1internal?1reflect?1Constan@ 100137b8     Class.obj
 0002:000007e0       ??_C@_0BI@EOEBGMEG@desiredAssertionStatus0@ 100137e0     Class.obj
 0002:000007f8       ??_C@_0BF@CBMAAKJJ@?$CILjava?1lang?1Class?$DL?$CJZ@ 100137f8     Class.obj
 0002:00000810       ??_C@_0BE@OLDEPMPN@getEnclosingMethod0@ 10013810     Class.obj
 0002:00000824       ??_C@_0BG@CNILIFMJ@getRawTypeAnnotations@ 10013824     Class.obj
 0002:0000083c       ??_C@_0N@NMCDFPDB@getNestHost0@ 1001383c     Class.obj
 0002:0000084c       ??_C@_0BA@DLOACIFG@getNestMembers0@ 1001384c     Class.obj
 0002:0000085c       ??_C@_0BF@GFGGJCDB@getRecordComponents0@ 1001385c     Class.obj
 0002:00000874       ??_C@_0CH@JOFOJHIB@?$CI?$CJ?$FLLjava?1lang?1reflect?1RecordCom@ 10013874     Class.obj
 0002:0000089c       ??_C@_09PCIIHAKK@isRecord0@ 1001389c     Class.obj
 0002:000008a8       ??_C@_0BI@GAOMCNP@getPermittedSubclasses0@ 100138a8     Class.obj
 0002:000008c0       ??_C@_0BD@EELMJMNJ@retrieveDirectives@ 100138c0     ClassLoader.obj
 0002:000008d4       ??_C@_0CI@FCANAINE@?$CI?$CJLjava?1lang?1AssertionStatusDir@ 100138d4     ClassLoader.obj
 0002:000008fc       ??_C@_04BOOCJOME@ms?$CFd@  100138fc     Console_md.obj
 0002:00000904       ??_C@_05EGJIMALK@UTF?98@   10013904     Console_md.obj
 0002:0000090c       ??_C@_04LDGHIPEL@cp?$CFd@  1001390c     Console_md.obj
 0002:00000914       ??_C@_0BG@NEFMNKJA@GetConsoleMode?5failed@ 10013914     Console_md.obj
 0002:0000092c       ??_C@_0BG@CBAKADNB@SetConsoleMode?5failed@ 1001392c     Console_md.obj
 0002:00000944       ??_C@_01JPJNBJEM@I@        10013944     FileDescriptor_md.obj
 0002:00000948       ??_C@_02ENHFDPNM@fd@       10013948     FileDescriptor_md.obj
 0002:0000094c       ??_C@_01LELAEKIP@J@        1001394c     FileDescriptor_md.obj
 0002:00000950       ??_C@_06NCGDPKCC@handle@   10013950     FileDescriptor_md.obj
 0002:00000958       ??_C@_01POHCFINO@Z@        10013958     FileDescriptor_md.obj
 0002:0000095c       ??_C@_06PCICMFGG@append@   1001395c     FileDescriptor_md.obj
 0002:00000964       ??_C@_0M@IALGLCNJ@sync?5failed@ 10013964     FileDescriptor_md.obj
 0002:00000970       ??_C@_0BM@MBMINGIL@java?1io?1SyncFailedException@ 10013970     FileDescriptor_md.obj
 0002:0000098c       ??_C@_0N@NOKLILHD@close?5failed@ 1001398c     FileDescriptor_md.obj
 0002:0000099c       ??_C@_0BJ@BDFOFHPL@Ljava?1io?1FileDescriptor?$DL@ 1001399c     FileInputStream.obj
 0002:000009b8       ??_C@_0O@KLFONINF@Stream?5Closed@ 100139b8     FileInputStream.obj
 0002:000009c8       ??_C@_0BB@CEBOPAFI@GetLength?5failed@ 100139c8     FileInputStream.obj
 0002:000009dc       ??_C@_0M@HPFDGGMC@Seek?5failed@ 100139dc     FileInputStream.obj
 0002:000009e8       ??_C@_0L@FCLNKJKA@Seek?5error@ 100139e8     FileInputStream.obj
 0002:000009f4       ??_C@_11LOCGONAA@@         100139f4     HostLocaleProviderAdapter_md.obj
 0002:000009f8       ??_C@_13BMLCKOLB@?$PP?$KE@ 100139f8     HostLocaleProviderAdapter_md.obj
 0002:000009fc       ??_C@_15GMICKCJK@?$PP?$KE?$AA?5@ 100139fc     HostLocaleProviderAdapter_md.obj
 0002:00000a04       ??_C@_13EJFHHPOP@?$AA?$CF@ 10013a04     HostLocaleProviderAdapter_md.obj
 0002:00000a08       ??_C@_15LJGOGFOH@?$AA?$CF?$AA?5@ 10013a08     HostLocaleProviderAdapter_md.obj
 0002:00000a10       ??_C@_13LLDNKHDC@?$AA?$CI@ 10013a10     HostLocaleProviderAdapter_md.obj
 0002:00000a14       ??_C@_13IMODFHAA@?$AA?9@   10013a14     HostLocaleProviderAdapter_md.obj
 0002:00000a18       ??_C@_15FFDNOHIK@?$AA?9?$AA?5@ 10013a18     HostLocaleProviderAdapter_md.obj
 0002:00000a20       ??_C@_15GHMLFHFF@?$AA?$CI?$PP?$KE@ 10013a20     HostLocaleProviderAdapter_md.obj
 0002:00000a28       ??_C@_15DHAGMGOG@?$AA?9?$PP?$KE@ 10013a28     HostLocaleProviderAdapter_md.obj
 0002:00000a30       ??_C@_15JOOIHKEH@?$PP?$KE?$AA?9@ 10013a30     HostLocaleProviderAdapter_md.obj
 0002:00000a38       ??_C@_17NKBBKLNH@?$AA?9?$PP?$KE?$AA?5@ 10013a38     HostLocaleProviderAdapter_md.obj
 0002:00000a40       ??_C@_17OBCOLLDF@?$PP?$KE?$AA?5?$AA?9@ 10013a40     HostLocaleProviderAdapter_md.obj
 0002:00000a48       ??_C@_17JCPBKFLD@?$AA?$CI?$PP?$KE?$AA?5@ 10013a48     HostLocaleProviderAdapter_md.obj
 0002:00000a50       ??_C@_15GCODBHLI@?$AA?9?$AA?$CF@ 10013a50     HostLocaleProviderAdapter_md.obj
 0002:00000a58       ??_C@_15ELAELNDK@?$AA?$CF?$AA?9@ 10013a58     HostLocaleProviderAdapter_md.obj
 0002:00000a60       ??_C@_17PPNGMKK@?$AA?9?$AA?$CF?$AA?5@ 10013a60     HostLocaleProviderAdapter_md.obj
 0002:00000a68       ??_C@_17HOLPDOHB@?$AA?$CF?$AA?5?$AA?9@ 10013a68     HostLocaleProviderAdapter_md.obj
 0002:00000a70       ??_C@_15ILJINFDI@?$AA?5?$PP?$KE@ 10013a70     HostLocaleProviderAdapter_md.obj
 0002:00000a78       ??_C@_15NOHNAEGG@?$AA?5?$AA?$CF@ 10013a78     HostLocaleProviderAdapter_md.obj
 0002:00000a80       ??_C@_13DIBMAFH@?$AA?$CJ@  10013a80     HostLocaleProviderAdapter_md.obj
 0002:00000a84       ??_C@_13HOIJIPNN@?$AA?5@   10013a84     HostLocaleProviderAdapter_md.obj
 0002:00000a88       ??_C@_15BLMJCMIJ@?$AA?5?$AA?9@ 10013a88     HostLocaleProviderAdapter_md.obj
 0002:00000a90       ??_C@_15BBIKONBA@?$PP?$KE?$AA?$CJ@ 10013a90     HostLocaleProviderAdapter_md.obj
 0002:00000a98       ??_C@_17LDHOGGNL@?$AA?5?$PP?$KE?$AA?9@ 10013a98     HostLocaleProviderAdapter_md.obj
 0002:00000aa0       ??_C@_17DNALNMHF@?$AA?9?$AA?5?$PP?$KE@ 10013aa0     HostLocaleProviderAdapter_md.obj
 0002:00000aa8       ??_C@_17DMBMPBIM@?$AA?5?$PP?$KE?$AA?$CJ@ 10013aa8     HostLocaleProviderAdapter_md.obj
 0002:00000ab0       ??_C@_17GGJCKBKG@?$AA?5?$AA?$CF?$AA?9@ 10013ab0     HostLocaleProviderAdapter_md.obj
 0002:00000ab8       ??_C@_17GIOOANCL@?$AA?9?$AA?5?$AA?$CF@ 10013ab8     HostLocaleProviderAdapter_md.obj
 0002:00000ac0       ??_C@_0BA@ONOKGCMP@GetLocaleInfoEx@ 10013ac0     HostLocaleProviderAdapter_md.obj
 0002:00000ad0       ??_C@_0N@MDJJJHMB@kernel32?4dll@ 10013ad0     HostLocaleProviderAdapter_md.obj
 0002:00000ae0       ??_C@_0BC@NJJJJEJP@GetCalendarInfoEx@ 10013ae0     HostLocaleProviderAdapter_md.obj
 0002:00000af4       ??_C@_0BF@IALNPCBG@EnumCalendarInfoExEx@ 10013af4     HostLocaleProviderAdapter_md.obj
 0002:00000b0c       ??_C@_0BI@FKAGBMCL@memory?5allocation?5error@ 10013b0c     HostLocaleProviderAdapter_md.obj
 0002:00000b24       ??_C@_0BB@FLFAIHG@java?1lang?1String@ 10013b24     HostLocaleProviderAdapter_md.obj
 0002:00000b38       ??_C@_17PINHLBBM@?$AAu?$AAn?$AAd@ 10013b38     HostLocaleProviderAdapter_md.obj
 0002:00000b40       ??_C@_15MNPNEAIF@?$AAe?$AAn@ 10013b40     HostLocaleProviderAdapter_md.obj
 0002:00000b48       ??_C@_13PJJBFPED@?$AA?$DL@ 10013b48     HostLocaleProviderAdapter_md.obj
 0002:00000b4c       ??_C@_13DEFPDAGF@?$AA?0@   10013b4c     HostLocaleProviderAdapter_md.obj
 0002:00000b50       ??_C@_0DG@ILJBJODK@jdk?1internal?1loader?1NativeLibra@ 10013b50     NativeLibraries.obj
 0002:00000b88       ??_C@_0L@FFGJFOPI@jniVersion@ 10013b88     NativeLibraries.obj
 0002:00000b94       ??_C@_0O@CNBBEDNA@_JNI_OnLoad?$EA8@ 10013b94     NativeLibraries.obj
 0002:00000ba4       ??_C@_0L@OIKEFKEO@JNI_OnLoad@ 10013ba4     NativeLibraries.obj
 0002:00000bb0       ??_C@_0BA@LDELBKAG@_JNI_OnUnload?$EA8@ 10013bb0     NativeLibraries.obj
 0002:00000bc0       ??_C@_0N@LLELHEHJ@JNI_OnUnload@ 10013bc0     NativeLibraries.obj
 0002:00000bd0       ??_C@_0CO@NLJCNFHA@unsupported?5JNI?5version?50x?$CF08X?5@ 10013bd0     NativeLibraries.obj
 0002:00000c00       ??_C@_0BP@JABHMODJ@java?1lang?1UnsatisfiedLinkError@ 10013c00     NativeLibraries.obj
 0002:00000c1f       ??_C@_00CNPNBAHC@@         10013c1f     NativeLibraries.obj
 0002:00000c20       ??_C@_04HLONOPDM@?4dll@    10013c20     NativeLibraries.obj
 0002:00000c28       ??_C@_0CB@CKDHIJCP@NULL?5filename?5for?5native?5librar@ 10013c28     NativeLibraries.obj
 0002:00000c4c       ??_C@_0BM@LKJNLDJK@java?1lang?1NoSuchMethodError@ 10013c4c     ObjectStreamClass.obj
 0002:00000c68       ??_C@_03GAEACAIP@?$CI?$CJV@ 10013c68     ObjectStreamClass.obj
 0002:00000c6c       ??_C@_08JOGLKNJI@?$DMclinit?$DO@ 10013c6c     ObjectStreamClass.obj
 0002:00000c78       ??_C@_05GBDANG@?$CI?$FLB?$CJV@ 10013c78     ProcessEnvironment_md.obj
 0002:00000c80       ??_C@_06FALKBLGB@?$DMinit?$DO@ 10013c80     ProcessEnvironment_md.obj
 0002:00000c88       ??_C@_0BN@PKAKOFME@GetEnvironmentStrings?5failed@ 10013c88     ProcessEnvironment_md.obj
 0002:00000ca8       ??_C@_0BD@JFADHEFE@Ljava?1lang?1String?$DL@ 10013ca8     ProcessHandleImpl_win.obj
 0002:00000cbc       ??_C@_07KMMNMMFF@command@  10013cbc     ProcessHandleImpl_win.obj
 0002:00000cc4       ??_C@_0M@EELMKCHN@commandLine@ 10013cc4     ProcessHandleImpl_win.obj
 0002:00000cd0       ??_C@_0BE@KHJCLGPN@?$FLLjava?1lang?1String?$DL@ 10013cd0     ProcessHandleImpl_win.obj
 0002:00000ce4       ??_C@_09PBNAMLIK@arguments@ 10013ce4     ProcessHandleImpl_win.obj
 0002:00000cf0       ??_C@_09MJNIPNBH@totalTime@ 10013cf0     ProcessHandleImpl_win.obj
 0002:00000cfc       ??_C@_09IIHJADCI@startTime@ 10013cfc     ProcessHandleImpl_win.obj
 0002:00000d08       ??_C@_04CCHAHKJA@user@     10013d08     ProcessHandleImpl_win.obj
 0002:00000d10       ??_C@_0BD@OOONFEIA@GetExitCodeProcess@ 10013d10     ProcessHandleImpl_win.obj
 0002:00000d24       ??_C@_0BL@IONOAEOO@java?1lang?1RuntimeException@ 10013d24     ProcessHandleImpl_win.obj
 0002:00000d40       ??_C@_0BH@LBENJJIP@WaitForMultipleObjects@ 10013d40     ProcessHandleImpl_win.obj
 0002:00000d58       ??_C@_0BH@DJKIHHBP@snapshot?5not?5available@ 10013d58     ProcessHandleImpl_win.obj
 0002:00000d70       ??_C@_0BG@LPMGLOAP@array?5sizes?5not?5equal@ 10013d70     ProcessHandleImpl_win.obj
 0002:00000d88       ??_C@_0BE@JIDLIKOL@GetTokenInformation@ 10013d88     ProcessHandleImpl_win.obj
 0002:00000d9c       ??_C@_13FPGAJAPJ@?$AA?2@   10013d9c     ProcessHandleImpl_win.obj
 0002:00000da0       ??_C@_1CA@BNEMBNGE@?$AA?$CF?$AAs?$AA?5?$AAe?$AAr?$AAr?$AAo?$AAr?$AA?$DN?$AA?$CF?$AAd?$AA?0?$AA?5?$AA?$CF?$AAs@ 10013da0     ProcessImpl_md.obj
 0002:00000dc0       ??_C@_1CI@OBOFAJOJ@?$AA?$CF?$AAs?$AA?5?$AAf?$AAa?$AAi?$AAl?$AAe?$AAd?$AA?0?$AA?5?$AAe?$AAr?$AAr?$AAo@ 10013dc0     ProcessImpl_md.obj
 0002:00000de8       ??_C@_0CM@EAKDBECK@Secondary?5error?5while?5OS?5messag@ 10013de8     ProcessImpl_md.obj
 0002:00000e14       ??_C@_1BG@HKMEIOD@?$AAC?$AAr?$AAe?$AAa?$AAt?$AAe?$AAP?$AAi?$AAp?$AAe@ 10013e14     ProcessImpl_md.obj
 0002:00000e2c       ??_C@_1BM@MMIOBBBF@?$AAC?$AAr?$AAe?$AAa?$AAt?$AAe?$AAP?$AAr?$AAo?$AAc?$AAe?$AAs?$AAs@ 10013e2c     ProcessImpl_md.obj
 0002:00000e48       ??_C@_1CG@LCLEBLIK@?$AAG?$AAe?$AAt?$AAE?$AAx?$AAi?$AAt?$AAC?$AAo?$AAd?$AAe?$AAP?$AAr?$AAo?$AAc@ 10013e48     ProcessImpl_md.obj
 0002:00000e70       ??_C@_1CO@PLEHGDKC@?$AAW?$AAa?$AAi?$AAt?$AAF?$AAo?$AAr?$AAM?$AAu?$AAl?$AAt?$AAi?$AAp?$AAl?$AAe@ 10013e70     ProcessImpl_md.obj
 0002:00000ea0       ??_C@_0M@GPOOGHPH@CreateFileW@ 10013ea0     ProcessImpl_md.obj
 0002:00000eac       ??_C@_0BF@HDGNMJHD@Negative?5seek?5offset@ 10013eac     RandomAccessFile.obj
 0002:00000ec4       ??_C@_0BB@GOOEHMBA@setLength?5failed@ 10013ec4     RandomAccessFile.obj
 0002:00000ed8       ??_C@_0BK@FOJCHAGK@java?1lang?1SecurityManager@ 10013ed8     SecurityManager.obj
 0002:00000ef4       ??_C@_0M@PBLAKOBI@initialized@ 10013ef4     SecurityManager.obj
 0002:00000f00       ??_C@_0BM@MPFHLPCE@java?1lang?1SecurityException@ 10013f00     SecurityManager.obj
 0002:00000f1c       ??_C@_0CC@HPKFBHGI@security?5manager?5not?5initialize@ 10013f1c     SecurityManager.obj
 0002:00000f40       ??_C@_04MEMAJGDJ@name@     10013f40     Signal.obj
 0002:00000f48       ??_C@_0BC@JMDLHMGP@currentTimeMillis@ 10013f48     System.obj
 0002:00000f5c       ??_C@_03IGDHHNNC@?$CI?$CJJ@ 10013f5c     System.obj
 0002:00000f60       ??_C@_08GAAFINGG@nanoTime@ 10013f60     System.obj
 0002:00000f6c       ??_C@_09EEHNOAG@arraycopy@ 10013f6c     System.obj
 0002:00000f78       ??_C@_0CL@DPOGMIND@?$CILjava?1lang?1Object?$DLILjava?1lang?1@ 10013f78     System.obj
 0002:00000fa4       ??_C@_02MLODCJFF@32@       10013fa4     System.obj
 0002:00000fa8       ??_C@_0BG@GPDHLGHH@Ljava?1io?1InputStream?$DL@ 10013fa8     System.obj
 0002:00000fc0       ??_C@_02LMMGJAGL@in@       10013fc0     System.obj
 0002:00000fc4       ??_C@_0BG@FPECDKGJ@Ljava?1io?1PrintStream?$DL@ 10013fc4     System.obj
 0002:00000fdc       ??_C@_03KEJHNBPP@out@      10013fdc     System.obj
 0002:00000fe0       ??_C@_03JIDPIAJI@err@      10013fe0     System.obj
 0002:00000fe4       ??_C@_0O@OLOAHEKB@name?5too?5long@ 10013fe4     System.obj
 0002:00000ff4       ??_C@_06MGHKGFHF@start0@   10013ff4     Thread.obj
 0002:00000ffc       ??_C@_05CHCLNOMK@stop0@    10013ffc     Thread.obj
 0002:00001004       ??_C@_0BG@JLFLBLJI@?$CILjava?1lang?1Object?$DL?$CJV@ 10014004     Thread.obj
 0002:0000101c       ??_C@_07BOOHCBLM@isAlive@  1001401c     Thread.obj
 0002:00001024       ??_C@_08PIHJGBMA@suspend0@ 10014024     Thread.obj
 0002:00001030       ??_C@_07EJLENFAP@resume0@  10014030     Thread.obj
 0002:00001038       ??_C@_0N@GOFHJCMI@setPriority0@ 10014038     Thread.obj
 0002:00001048       ??_C@_04PFANPMCN@?$CII?$CJV@ 10014048     Thread.obj
 0002:00001050       ??_C@_05LKJGIMLP@yield@    10014050     Thread.obj
 0002:00001058       ??_C@_05PCJCMMHD@sleep@    10014058     Thread.obj
 0002:00001060       ??_C@_04OHLIFDMD@?$CIJ?$CJV@ 10014060     Thread.obj
 0002:00001068       ??_C@_0O@GIDKOGNF@currentThread@ 10014068     Thread.obj
 0002:00001078       ??_C@_0BF@GLBLFFEM@?$CI?$CJLjava?1lang?1Thread?$DL@ 10014078     Thread.obj
 0002:00001090       ??_C@_0L@KOCFLKPP@interrupt0@ 10014090     Thread.obj
 0002:0000109c       ??_C@_09BKEKKKBN@holdsLock@ 1001409c     Thread.obj
 0002:000010a8       ??_C@_0BG@DHOOFEJE@?$CILjava?1lang?1Object?$DL?$CJZ@ 100140a8     Thread.obj
 0002:000010c0       ??_C@_0L@MBENOCKD@getThreads@ 100140c0     Thread.obj
 0002:000010cc       ??_C@_0BG@CJDMDLMO@?$CI?$CJ?$FLLjava?1lang?1Thread?$DL@ 100140cc     Thread.obj
 0002:000010e4       ??_C@_0M@ECOKKOKF@dumpThreads@ 100140e4     Thread.obj
 0002:000010f0       ??_C@_0DF@ELFIABCA@?$CI?$FLLjava?1lang?1Thread?$DL?$CJ?$FL?$FLLjava?1la@ 100140f0     Thread.obj
 0002:00001128       ??_C@_0O@LPHHHNKJ@setNativeName@ 10014128     Thread.obj
 0002:00001138       ??_C@_0BG@IKDDPPGD@?$CILjava?1lang?1String?$DL?$CJV@ 10014138     Thread.obj
 0002:00001150       ??_C@_1BK@BOBBLECB@?$AAS?$AAt?$AAa?$AAn?$AAd?$AAa?$AAr?$AAd?$AAN?$AAa?$AAm?$AAe@ 10014150     TimeZone_md.obj
 0002:0000116c       ??_C@_0N@PEHDGIGO@StandardName@ 1001416c     TimeZone_md.obj
 0002:0000117c       ??_C@_17GFIDPLDA@?$AAS?$AAt?$AAd@ 1001417c     TimeZone_md.obj
 0002:00001184       ??_C@_03FFGKOOIA@Std@      10014184     TimeZone_md.obj
 0002:00001188       ??_C@_0P@EKMDNJBA@GMT?$CFc?$CF02d?3?$CF02d@ 10014188     TimeZone_md.obj
 0002:00001198       ??_C@_03HOONMGKE@GMT@      10014198     TimeZone_md.obj
 0002:0000119c       ??_C@_0DF@OCPBGDJE@System?2CurrentControlSet?2Contro@ 1001419c     TimeZone_md.obj
 0002:000011d4       ??_C@_0BM@HEGPJGEC@DynamicDaylightTimeDisabled@ 100141d4     TimeZone_md.obj
 0002:000011f0       ??_C@_0BA@GCKJIEGO@TimeZoneKeyName@ 100141f0     TimeZone_md.obj
 0002:00001200       ??_C@_0DI@LLEGOPFO@SOFTWARE?2Microsoft?2Windows?5NT?2C@ 10014200     TimeZone_md.obj
 0002:00001238       ??_C@_0DF@JEJGGGGH@SOFTWARE?2Microsoft?2Windows?2Curr@ 10014238     TimeZone_md.obj
 0002:00001270       ??_C@_03NKEEOHDM@TZI@      10014270     TimeZone_md.obj
 0002:00001274       ??_C@_0BA@PBEHAGHA@?2lib?2tzmappings@ 10014274     TimeZone_md.obj
 0002:00001284       ??_C@_01KDCPPGHE@r@        10014284     TimeZone_md.obj
 0002:00001288       ??_C@_0BA@PMGFJNJD@can?8t?5open?5?$CFs?4?6@ 10014288     TimeZone_md.obj
 0002:00001298       ??_C@_0BG@MJJAMJBB@premature?5end?5of?5line@ 10014298     TimeZone_md.obj
 0002:000012b0       ??_C@_0BN@NFCIANLB@illegal?5null?5character?5found@ 100142b0     TimeZone_md.obj
 0002:000012d0       ??_C@_0CE@OJDILIEN@illegal?5non?9newline?5character?5f@ 100142d0     TimeZone_md.obj
 0002:000012f4       ??_C@_03MMKGDKGA@001@      100142f4     TimeZone_md.obj
 0002:000012f8       ??_C@_0DO@EINJANBE@Illegal?5format?5in?5tzmappings?5fi@ 100142f8     TimeZone_md.obj
 0002:00001338       ??_C@_0P@DOCHMBNE@ActiveTimeBias@ 10014338     TimeZone_md.obj
 0002:00001348       ??_C@_0BG@FPHJJCID@getNanoTimeAdjustment@ 10014348     VM.obj
 0002:00001360       ??_C@_04BMPAOJO@?$CIJ?$CJJ@ 10014360     VM.obj
 0002:00001368       ??_C@_04JCEIFDIJ@J2SE@     10014368     WinCAPISeedGenerator.obj
 0002:00001370       ??_C@_0N@IOFABHFH@java?1io?1File@ 10014370     WinNTFileSystem_md.obj
 0002:00001380       ??_C@_04LNEJFJGI@path@     10014380     WinNTFileSystem_md.obj
 0002:00001388       ??_C@_0BK@PDKDDAF@GetFinalPathNameByHandleW@ 10014388     WinNTFileSystem_md.obj
 0002:000013a4       ??_C@_0CA@NIIGFDJD@native?5memory?5allocation?5failed@ 100143a4     WinNTFileSystem_md.obj
 0002:000013c4       ??_C@_0N@NMICNPLE@Bad?5pathname@ 100143c4     WinNTFileSystem_md.obj
 0002:000013d4       ??_C@_17LIAKHCCP@?$AAC?$AAO?$AAN@ 100143d4     WinNTFileSystem_md.obj
 0002:000013dc       ??_C@_17PFHGFFKC@?$AAP?$AAR?$AAN@ 100143dc     WinNTFileSystem_md.obj
 0002:000013e4       ??_C@_17CNBAFMOM@?$AAA?$AAU?$AAX@ 100143e4     WinNTFileSystem_md.obj
 0002:000013ec       ??_C@_17CLELIOII@?$AAN?$AAU?$AAL@ 100143ec     WinNTFileSystem_md.obj
 0002:000013f4       ??_C@_17KKLPNNMB@?$AAC?$AAO?$AAM@ 100143f4     WinNTFileSystem_md.obj
 0002:000013fc       ??_C@_17KMAOGHDG@?$AAL?$AAP?$AAT@ 100143fc     WinNTFileSystem_md.obj
 0002:00001404       ??_C@_0BE@LONNMHBH@Could?5not?5open?5file@ 10014404     WinNTFileSystem_md.obj
 0002:00001418       ??_C@_13BBDEGPLJ@?$AA?$CK@ 10014418     WinNTFileSystem_md.obj
 0002:0000141c       ??_C@_15PKPONJIK@?$AA?2?$AA?$CK@ 1001441c     WinNTFileSystem_md.obj
 0002:00001424       ??_C@_13JOFGPIOO@?$AA?4@   10014424     WinNTFileSystem_md.obj
 0002:00001428       ??_C@_15DDHGOCBH@?$AA?4?$AA?4@ 10014428     WinNTFileSystem_md.obj
 0002:00001430       ??_C@_0CH@PNOGCBMH@Could?5not?5get?5maximum?5component@ 10014430     WinNTFileSystem_md.obj
 0002:00001458       ??_C@_19BKJMDJK@?$AA?2?$AA?2?$AA?4?$AA?2@ 10014458     canonicalize_md.obj
 0002:00001464       ??_C@_1BC@FBJNHMLC@?$AA?2?$AA?2?$AA?$DP?$AA?2?$AAU?$AAN?$AAC?$AA?$AA@ 10014464     canonicalize_md.obj
 0002:00001478       ??_C@_1M@DJNCMBIG@?$AA?2?$AA?2?$AA?$DP?$AA?2?$AA?$AA@ 10014478     canonicalize_md.obj
 0002:00001484       ??_C@_0L@BHPPDFMA@Read?5error@ 10014484     io_util.obj
 0002:00001490       ??_C@_0CE@JOEPHHFN@java?1lang?1IndexOutOfBoundsExcep@ 10014490     io_util.obj
 0002:000014b4       ??_C@_0M@PJBDJJDJ@Write?5error@ 100144b4     io_util.obj
 0002:000014c0       ??_C@_0CI@HEGLGDKJ@?$CILjava?1lang?1String?$DLLjava?1lang?1S@ 100144c0     io_util.obj
 0002:000014e8       ??_C@_0BO@FDOOLAPO@java?1io?1FileNotFoundException@ 100144e8     io_util.obj
 0002:00001508       ??_C@_03LIOLIPAH@GBK@      10014508     java_props_md.obj
 0002:0000150c       ??_C@_07DNCGDNOG@GB18030@  1001450c     java_props_md.obj
 0002:00001514       ??_C@_05PCINFEFG@MS950@    10014514     java_props_md.obj
 0002:0000151c       ??_C@_0P@JHCFFHNK@MS950_HKSCS_XP@ 1001451c     java_props_md.obj
 0002:0000152c       ??_C@_0BH@NKFNLGAB@?2FONTS?2SimSun18030?4ttc@ 1001452c     java_props_md.obj
 0002:00001544       ??_C@_01JOAMLHOP@?9@       10014544     java_props_md.obj
 0002:00001548       ??_C@_04LFKJOHGN@ia64@     10014548     java_props_md.obj
 0002:00001550       ??_C@_05MDLPDLNO@amd64@    10014550     java_props_md.obj
 0002:00001558       ??_C@_0DO@DIFICBBG@pentium_pro?$CLmmx?5pentium_pro?5pen@ 10014558     java_props_md.obj
 0002:00001598       ??_C@_0CC@BIODACBF@pentium_pro?5pentium?5i486?5i386?5i@ 10014598     java_props_md.obj
 0002:000015bc       ??_C@_0CC@PPFBHJAM@pentium?$CLmmx?5pentium?5i486?5i386?5i@ 100145bc     java_props_md.obj
 0002:000015e0       ??_C@_0BG@CMPGKFGL@pentium?5i486?5i386?5i86@ 100145e0     java_props_md.obj
 0002:000015f8       ??_C@_0O@MAAOGNKJ@i486?5i386?5i86@ 100145f8     java_props_md.obj
 0002:00001608       ??_C@_08IPFADFGF@i386?5i86@ 10014608     java_props_md.obj
 0002:00001614       ??_C@_0BH@NIHCMEPJ@?$CF?$CK?$FLa?9z?2?9?$FN?$CF1?$FLA?9Z?$FN?$CF?$FLa?9z?$FN@ 10014614     java_props_md.obj
 0002:0000162c       ??_C@_02LFNMGJAP@en@       1001462c     java_props_md.obj
 0002:00001630       ??_C@_02PLFPMECB@US@       10014630     java_props_md.obj
 0002:00001634       ??_C@_02BFDMMJOC@nb@       10014634     java_props_md.obj
 0002:00001638       ??_C@_02KAJCLHKP@no@       10014638     java_props_md.obj
 0002:0000163c       ??_C@_02NFLNFON@NO@        1001463c     java_props_md.obj
 0002:00001640       ??_C@_02LJIJIGOO@nn@       10014640     java_props_md.obj
 0002:00001644       ??_C@_02BBMDGADK@NY@       10014644     java_props_md.obj
 0002:00001648       ??_C@_0O@BAKIPCDE@?2kernel32?4dll@ 10014648     java_props_md.obj
 0002:00001658       ??_C@_1BM@JEABEHHA@?$AA?2?$AAk?$AAe?$AAr?$AAn?$AAe?$AAl?$AA3?$AA2?$AA?4?$AAd?$AAl?$AAl@ 10014658     java_props_md.obj
 0002:00001674       ??_C@_0L@NEBNHFIE@Windows?595@ 10014674     java_props_md.obj
 0002:00001680       ??_C@_0L@GBLDALMJ@Windows?598@ 10014680     java_props_md.obj
 0002:0000168c       ??_C@_0L@DNFOOIFM@Windows?5Me@ 1001468c     java_props_md.obj
 0002:00001698       ??_C@_0BF@KOJMMOAG@Windows?59X?5?$CIunknown?$CJ@ 10014698     java_props_md.obj
 0002:000016b0       ??_C@_0L@PJEFFBLH@Windows?5NT@ 100146b0     java_props_md.obj
 0002:000016bc       ??_C@_0N@MEKDBOKB@Windows?52000@ 100146bc     java_props_md.obj
 0002:000016cc       ??_C@_0L@IFICELHB@Windows?5XP@ 100146cc     java_props_md.obj
 0002:000016d8       ??_C@_0N@OPIOENGC@Windows?52003@ 100146d8     java_props_md.obj
 0002:000016e8       ??_C@_0BF@GMBBPJFL@Windows?5NT?5?$CIunknown?$CJ@ 100146e8     java_props_md.obj
 0002:00001700       ??_C@_0O@IFKHFILP@Windows?5Vista@ 10014700     java_props_md.obj
 0002:00001710       ??_C@_09GOHFIPMO@Windows?57@ 10014710     java_props_md.obj
 0002:0000171c       ??_C@_09OJONJDAB@Windows?58@ 1001471c     java_props_md.obj
 0002:00001728       ??_C@_0M@IEJDHGAK@Windows?58?41@ 10014728     java_props_md.obj
 0002:00001734       ??_C@_0BE@GHBPPLPA@Windows?5Server?52008@ 10014734     java_props_md.obj
 0002:00001748       ??_C@_0BH@ONPOEHKF@Windows?5Server?52008?5R2@ 10014748     java_props_md.obj
 0002:00001760       ??_C@_0BE@JMDCHJEN@Windows?5Server?52012@ 10014760     java_props_md.obj
 0002:00001774       ??_C@_0BH@GMBCIMKB@Windows?5Server?52012?5R2@ 10014774     java_props_md.obj
 0002:0000178c       ??_C@_0L@LOGCOBDI@Windows?511@ 1001478c     java_props_md.obj
 0002:00001798       ??_C@_0L@KHHJNAHJ@Windows?510@ 10014798     java_props_md.obj
 0002:000017a4       ??_C@_0BE@JOHEMHBE@Windows?5Server?52022@ 100147a4     java_props_md.obj
 0002:000017b8       ??_C@_0BE@HPMGKAIG@Windows?5Server?52019@ 100147b8     java_props_md.obj
 0002:000017cc       ??_C@_0BE@PIFOLMEJ@Windows?5Server?52016@ 100147cc     java_props_md.obj
 0002:000017e0       ??_C@_0BC@JFKFADHL@Windows?5?$CIunknown?$CJ@ 100147e0     java_props_md.obj
 0002:000017f4       ??_C@_05KBEOJPB@?$CFd?4?$CFd@ 100147f4     java_props_md.obj
 0002:000017fc       ??_C@_03NDFEINMN@x86@      100147fc     java_props_md.obj
 0002:00001800       ??_C@_06LADGIEOA@little@   10014800     java_props_md.obj
 0002:00001808       ??_C@_1BC@GGLDBIGJ@?$AAU?$AAS?$AAE?$AAR?$AAN?$AAA?$AAM?$AAE@ 10014808     java_props_md.obj
 0002:0000181c       ??_C@_1BA@KDMGPDJH@?$AAu?$AAn?$AAk?$AAn?$AAo?$AAw?$AAn@ 1001481c     java_props_md.obj
 0002:0000182c       ??_C@_17BJPFHBEJ@?$AAC?$AA?3?$AA?2@ 1001482c     java_props_md.obj
 0002:00001834       ??_C@_0M@JNHAKOPM@MS950_HKSCS@ 10014834     java_props_md.obj
 0002:00001840       ??_C@_0O@KBEEOPPB@UnicodeLittle@ 10014840     java_props_md.obj
 0002:00001850       ??_C@_01KICIPPFI@?2@       10014850     java_props_md.obj
 0002:00001854       ??_C@_01ICJEACDI@?$DL@     10014854     java_props_md.obj
 0002:00001858       ??_C@_02PCIJFNDE@?$AN?6@   10014858     java_props_md.obj
 0002:0000185c       ??_C@_0BP@GJLHLAKJ@java?1lang?1NullPointerException@ 1001485c     jni_util.obj
 0002:0000187c       ??_C@_0CJ@ODBKFPOB@java?1lang?1ArrayIndexOutOfBounds@ 1001487c     jni_util.obj
 0002:000018a8       ??_C@_0BL@ENCPOIKC@java?1lang?1OutOfMemoryError@ 100148a8     jni_util.obj
 0002:000018c4       ??_C@_0CD@MOHADDFA@java?1lang?1IllegalArgumentExcept@ 100148c4     jni_util.obj
 0002:000018e8       ??_C@_0BI@NBLNIHIB@java?1lang?1InternalError@ 100148e8     jni_util.obj
 0002:00001900       ??_C@_0CB@KCPANAMN@java?1lang?1ClassNotFoundExceptio@ 10014900     jni_util.obj
 0002:00001924       ??_C@_0BE@EBAPEBGJ@java?1io?1IOException@ 10014924     jni_util.obj
 0002:00001938       ??_C@_05DNDNCJEB@?5?$CI?$CFs?$CJ@ 10014938     jni_util.obj
 0002:00001940       ??_C@_0CH@NCPCFFHJ@?$CILjava?1lang?1String?$DL?$CJLjava?1lang?1@ 10014940     jni_util.obj
 0002:00001968       ??_C@_06CMLIEHFC@concat@   10014968     jni_util.obj
 0002:00001970       ??_C@_0BH@GDIHDDN@no?5further?5information@ 10014970     jni_util.obj
 0002:00001988       ??_C@_0CO@NPADHBGE@JNU_CallStaticMethodByName?3?5ill@ 10014988     jni_util.obj
 0002:000019b8       ??_C@_0CJ@MELNKLJP@JNU_CallMethodByNameV?3?5illegal?5@ 100149b8     jni_util.obj
 0002:000019e4       ??_C@_0BG@CGIGLAGP@?$CILjava?1lang?1String?$DL?$CJZ@ 100149e4     jni_util.obj
 0002:000019fc       ??_C@_0M@CPFODPBC@isSupported@ 100149fc     jni_util.obj
 0002:00001a08       ??_C@_0BJ@ECKJLLIP@java?1nio?1charset?1Charset@ 10014a08     jni_util.obj
 0002:00001a24       ??_C@_06FEGJKAJG@8859_1@   10014a24     jni_util.obj
 0002:00001a2c       ??_C@_09KEDHCKDI@ISO8859?91@ 10014a2c     jni_util.obj
 0002:00001a38       ??_C@_09PDECJGAG@ISO8859_1@ 10014a38     jni_util.obj
 0002:00001a44       ??_C@_0L@GJIJNDEK@ISO?98859?91@ 10014a44     jni_util.obj
 0002:00001a50       ??_C@_09BGDIBLML@ISO646?9US@ 10014a50     jni_util.obj
 0002:00001a5c       ??_C@_06BFOBJALC@Cp1252@   10014a5c     jni_util.obj
 0002:00001a64       ??_C@_08MIMKAGHL@utf?916le@ 10014a64     jni_util.obj
 0002:00001a70       ??_C@_0BM@KEODIIBN@platform?5encoding?5undefined@ 10014a70     jni_util.obj
 0002:00001a8c       ??_C@_0BH@BOKGLNMJ@?$CILjava?1lang?1String?$DL?$CJ?$FLB@ 10014a8c     jni_util.obj
 0002:00001aa4       ??_C@_08LJNJGADH@getBytes@ 10014aa4     jni_util.obj
 0002:00001ab0       ??_C@_0BI@KCGPNIE@?$CI?$FLBLjava?1lang?1String?$DL?$CJV@ 10014ab0     jni_util.obj
 0002:00001ac8       ??_C@_01HMGJMAIH@B@        10014ac8     jni_util.obj
 0002:00001acc       ??_C@_05DMGOLBNP@coder@    10014acc     jni_util.obj
 0002:00001ad4       ??_C@_02KCBIMKDL@?$FLB@    10014ad4     jni_util.obj
 0002:00001ad8       ??_C@_05MFEJDJP@value@     10014ad8     jni_util.obj
 0002:00001ae0       ??_C@_0CC@PDGFIJNH@platform?5encoding?5not?5initializ@ 10014ae0     jni_util.obj
 0002:00001b04       ??_C@_04HIBGFPH@NULL@      10014b04     jni_util.obj
 0002:00001b0c       ??_C@_08JCDFGHAO@toString@ 10014b0c     jni_util.obj
 0002:00001b18       ??_C@_0CG@ENHAICHD@JNU_GetFieldByName?3?5illegal?5sig@ 10014b18     jni_util.obj
 0002:00001b40       ??_C@_0CG@PKMPNPAI@JNU_SetFieldByName?3?5illegal?5sig@ 10014b40     jni_util.obj
 0002:00001b68       ??_C@_0CM@FFECHOAH@JNU_GetStaticFieldByName?3?5illeg@ 10014b68     jni_util.obj
 0002:00001b94       ??_C@_01IDAFKMJL@_@        10014b94     jni_util_md.obj
 0002:00001b98       __real@3ff8000000000000    10014b98     fdlibm:s_atan.obj
 0002:00001ba0       __real@4000000000000000    10014ba0     fdlibm:s_atan.obj
 0002:00001ba8       __real@bff0000000000000    10014ba8     fdlibm:s_atan.obj
 0002:00001bb0       __xmm@80000000000000008000000000000000 10014bb0     fdlibm:s_atan.obj
 0002:00001bc0       __real@3fe0000000000000    10014bc0     fdlibm:s_expm1.obj
 0002:00001bc8       __real@4008000000000000    10014bc8     fdlibm:s_expm1.obj
 0002:00001bd0       __real@4018000000000000    10014bd0     fdlibm:s_expm1.obj
 0002:00001bd8       __real@bfd0000000000000    10014bd8     fdlibm:s_expm1.obj
 0002:00001be0       __real@bfe0000000000000    10014be0     fdlibm:s_expm1.obj
 0002:00001be8       __real@c000000000000000    10014be8     fdlibm:s_expm1.obj
 0002:00001bf0       __real@3fe5555555555555    10014bf0     fdlibm:s_log1p.obj
 0002:00001bf8       __real@3ff0000000000000    10014bf8     fdlibm:s_log1p.obj
 0002:00001c00       __real@0000000000000000    10014c00     fdlibm:e_acos.obj
 0002:00001c08       __real@c008000000000000    10014c08     fdlibm:e_atan2.obj
 0002:00001c10       __real@3fd2000000000000    10014c10     fdlibm:k_cos.obj
 0002:00001c18       __real@3fd5555555555555    10014c18     fdlibm:e_log.obj
 0002:00001c20       __real@3fc0000000000000    10014c20     fdlibm:k_rem_pio2.obj
 0002:00001c28       __real@4020000000000000    10014c28     fdlibm:k_rem_pio2.obj
 0002:00001c30       __sz_SHELL32_dll           10014c30     shell32:SHELL32.dll
 0002:00001c3c       _FOLDERID_Profile          10014c3c     shell32:shguid.obj
 0002:00001c4c       ??_C@_1BK@DBDEIDLH@?$AAK?$AAE?$AAR?$AAN?$AAE?$AAL?$AA3?$AA2?$AA?4?$AAD?$AAL?$AAL@ 10014c4c     delayimp:delayhlp.obj
 0002:00001c68       ??_C@_0BI@OMNLIJDB@AcquireSRWLockExclusive@ 10014c68     delayimp:delayhlp.obj
 0002:00001c80       ??_C@_0BI@HMIEPCNJ@ReleaseSRWLockExclusive@ 10014c80     delayimp:delayhlp.obj
 0002:00001c98       ___pfnDliNotifyHook2       10014c98     delayimp:delayhk2.obj
 0002:00001c9c       ___pfnDliFailureHook2      10014c9c     delayimp:delayhk1.obj
 0002:00001ca8       __pDefaultRawDllMain       10014ca8     MSVCRT:dll_dllmain.obj
 0002:00001ca8       __pRawDllMain              10014ca8     MSVCRT:dll_dllmain.obj
 0002:00001cb0       __load_config_used         10014cb0     MSVCRT:loadcfg.obj
 0002:00001dd8       ___safe_se_handler_table   10014dd8     <linker-defined>
 0002:000020d8       ___rtc_iaa                 100150d8     MSVCRT:initsect.obj
 0002:000020dc       ___rtc_izz                 100150dc     MSVCRT:initsect.obj
 0002:000020e0       ___rtc_taa                 100150e0     MSVCRT:initsect.obj
 0002:000020e4       ___rtc_tzz                 100150e4     MSVCRT:initsect.obj
 0002:0000218c       __DELAY_IMPORT_DESCRIPTOR_shell32_dll 1001518c     shell32:SHELL32.dll
 0002:000021ac       __NULL_DELAY_IMPORT_DESCRIPTOR 100151ac     shell32:SHELL32.dll
 0002:000021d4       \177SHELL32_NULL_THUNK_DATA_DLN 100151d4     shell32:SHELL32.dll
 0002:00002208       \177SHELL32_NULL_THUNK_DATA_DLB 10015208     shell32:SHELL32.dll
 0002:00006378       __IMPORT_DESCRIPTOR_jvm    10019378     jvm:jvm.dll
 0002:0000638c       __IMPORT_DESCRIPTOR_ADVAPI32 1001938c     advapi32:ADVAPI32.dll
 0002:000063a0       __IMPORT_DESCRIPTOR_VERSION 100193a0     version:VERSION.dll
 0002:000063b4       __IMPORT_DESCRIPTOR_KERNEL32 100193b4     kernel32:KERNEL32.dll
 0002:000063c8       __IMPORT_DESCRIPTOR_VCRUNTIME140 100193c8     vcruntime:VCRUNTIME140.dll
 0002:000063dc       __IMPORT_DESCRIPTOR_api-ms-win-crt-heap-l1-1-0 100193dc     ucrt:api-ms-win-crt-heap-l1-1-0.dll
 0002:000063f0       __IMPORT_DESCRIPTOR_api-ms-win-crt-stdio-l1-1-0 100193f0     ucrt:api-ms-win-crt-stdio-l1-1-0.dll
 0002:00006404       __IMPORT_DESCRIPTOR_api-ms-win-crt-string-l1-1-0 10019404     ucrt:api-ms-win-crt-string-l1-1-0.dll
 0002:00006418       __IMPORT_DESCRIPTOR_api-ms-win-crt-convert-l1-1-0 10019418     ucrt:api-ms-win-crt-convert-l1-1-0.dll
 0002:0000642c       __IMPORT_DESCRIPTOR_api-ms-win-crt-runtime-l1-1-0 1001942c     ucrt:api-ms-win-crt-runtime-l1-1-0.dll
 0002:00006440       __IMPORT_DESCRIPTOR_api-ms-win-crt-filesystem-l1-1-0 10019440     ucrt:api-ms-win-crt-filesystem-l1-1-0.dll
 0002:00006454       __IMPORT_DESCRIPTOR_api-ms-win-crt-environment-l1-1-0 10019454     ucrt:api-ms-win-crt-environment-l1-1-0.dll
 0002:00006468       __NULL_IMPORT_DESCRIPTOR   10019468     jvm:jvm.dll
 0003:00000168       _monthsType                1001c168     HostLocaleProviderAdapter_md.obj
 0003:0000019c       _sMonthsType               1001c19c     HostLocaleProviderAdapter_md.obj
 0003:000001d0       _wDaysType                 1001c1d0     HostLocaleProviderAdapter_md.obj
 0003:000001ec       _sWDaysType                1001c1ec     HostLocaleProviderAdapter_md.obj
 0003:00000208       _ampmType                  1001c208     HostLocaleProviderAdapter_md.obj
 0003:00000210       _fixes                     1001c210     HostLocaleProviderAdapter_md.obj
 0003:00000da0       __fltused                  1001cda0     MSVCRT:fltused.obj
 0003:00000da4       ___security_cookie_complement 1001cda4     MSVCRT:gs_cookie.obj
 0003:00000da8       ___security_cookie         1001cda8     MSVCRT:gs_cookie.obj
 0003:00000db0       ___scrt_native_dllmain_reason 1001cdb0     MSVCRT:utility.obj
 0003:00000db4       ___isa_enabled             1001cdb4     MSVCRT:cpu_disp.obj
 0003:00000db8       ___scrt_ucrt_dll_is_in_use 1001cdb8     MSVCRT:ucrt_stubs.obj
 0003:00000dbc       __imp__SHGetKnownFolderPath@16 1001cdbc     shell32:SHELL32.dll
 0003:00000dc0       __imp__SHGetFolderPathW@20 1001cdc0     shell32:SHELL32.dll
 0003:00000dc4       \177SHELL32_NULL_THUNK_DATA_DLA 1001cdc4     shell32:SHELL32.dll
 0003:00000dc8       _initialized               1001cdc8     HostLocaleProviderAdapter_md.obj
 0003:00000ed0       __hmod__SHELL32_dll        1001ced0     shell32:SHELL32.dll
 0003:00000ed4       ?DloadKernel32@@3PAUHINSTANCE__@@A 1001ced4     delayimp:delayhlp.obj
 0003:00000ed8       ?DloadAcquireSRWLockExclusive@@3P6GXPAK@ZA 1001ced8     delayimp:delayhlp.obj
 0003:00000edc       ?DloadReleaseSRWLockExclusive@@3P6GXPAK@ZA 1001cedc     delayimp:delayhlp.obj
 0003:00000ee0       ?DloadSrwLock@@3KA         1001cee0     delayimp:delayhlp.obj
 0003:00000ee4       ?DloadSectionLockCount@@3KA 1001cee4     delayimp:delayhlp.obj
 0003:00000ee8       ?DloadSectionOldProtection@@3KA 1001cee8     delayimp:delayhlp.obj
 0003:00000eec       ?DloadSectionCommitPermanent@@3KA 1001ceec     delayimp:delayhlp.obj
 0003:00001210       ?__type_info_root_node@@3U__type_info_node@@A 1001d210     MSVCRT:tncleanup.obj
 0003:00001218       ___scrt_current_native_startup_state 1001d218     MSVCRT:utility.obj
 0003:0000121c       ___scrt_native_startup_lock 1001d21c     MSVCRT:utility.obj
 0003:0000123c       ___scrt_debugger_hook_flag 1001d23c     MSVCRT:utility_desktop.obj
 0003:00001240       ___isa_available           1001d240     MSVCRT:cpu_disp.obj
 0003:00001244       ___favor                   1001d244     MSVCRT:cpu_disp.obj
 0003:00001248       ?_OptionsStorage@?1??__local_stdio_scanf_options@@9@9 1001d248     <common>
 0003:00001250       _raf_fd                    1001d250     <common>
 0003:00001254       _pEnumCalendarInfoExEx     1001d254     <common>
 0003:00001258       _pGetCalendarInfoEx        1001d258     <common>
 0003:0000125c       _pGetLocaleInfoEx          1001d25c     <common>
 0003:00001260       _fos_fd                    1001d260     <common>
 0003:00001264       _fis_fd                    1001d264     <common>
 0003:00001268       _IO_append_fdID            1001d268     <common>
 0003:0000126c       _IO_handle_fdID            1001d26c     <common>
 0003:00001270       _IO_fd_fdID                1001d270     <common>
 0003:00001278       ?_OptionsStorage@?1??__local_stdio_printf_options@@9@9 1001d278     <common>
 0003:00001280       ___dyn_tls_init_callback   1001d280     <common>

 entry point at        0001:00010ad7

 Static symbols

 0000:fffdf000       .debug$S                   10000000     java.exp
 0000:fffdf000       .debug$S                   10000000     vcruntime:VCRUNTIME140.dll
 0000:fffdf000       .debug$S                   10000000     vcruntime:VCRUNTIME140.dll
 0000:fffdf000       .debug$S                   10000000     vcruntime:VCRUNTIME140.dll
 0000:fffdf000       .debug$S                   10000000     vcruntime:VCRUNTIME140.dll
 0000:fffdf000       .debug$S                   10000000     vcruntime:VCRUNTIME140.dll
 0000:fffdf000       .debug$S                   10000000     vcruntime:VCRUNTIME140.dll
 0000:fffdf000       .debug$S                   10000000     vcruntime:VCRUNTIME140.dll
 0000:fffdf000       .debug$S                   10000000     vcruntime:VCRUNTIME140.dll
 0000:fffdf000       .debug$S                   10000000     vcruntime:VCRUNTIME140.dll
 0000:fffdf000       .debug$S                   10000000     vcruntime:VCRUNTIME140.dll
 0000:fffdf000       .debug$S                   10000000     ucrt:api-ms-win-crt-convert-l1-1-0.dll
 0000:fffdf000       .debug$S                   10000000     ucrt:api-ms-win-crt-convert-l1-1-0.dll
 0000:fffdf000       .debug$S                   10000000     ucrt:api-ms-win-crt-convert-l1-1-0.dll
 0000:fffdf000       .debug$S                   10000000     ucrt:api-ms-win-crt-environment-l1-1-0.dll
 0000:fffdf000       .debug$S                   10000000     ucrt:api-ms-win-crt-environment-l1-1-0.dll
 0000:fffdf000       .debug$S                   10000000     ucrt:api-ms-win-crt-environment-l1-1-0.dll
 0000:fffdf000       .debug$S                   10000000     ucrt:api-ms-win-crt-filesystem-l1-1-0.dll
 0000:fffdf000       .debug$S                   10000000     ucrt:api-ms-win-crt-filesystem-l1-1-0.dll
 0000:fffdf000       .debug$S                   10000000     ucrt:api-ms-win-crt-filesystem-l1-1-0.dll
 0000:fffdf000       .debug$S                   10000000     ucrt:api-ms-win-crt-heap-l1-1-0.dll
 0000:fffdf000       .debug$S                   10000000     ucrt:api-ms-win-crt-heap-l1-1-0.dll
 0000:fffdf000       .debug$S                   10000000     ucrt:api-ms-win-crt-heap-l1-1-0.dll
 0000:fffdf000       .debug$S                   10000000     ucrt:api-ms-win-crt-runtime-l1-1-0.dll
 0000:fffdf000       .debug$S                   10000000     ucrt:api-ms-win-crt-runtime-l1-1-0.dll
 0000:fffdf000       .debug$S                   10000000     ucrt:api-ms-win-crt-runtime-l1-1-0.dll
 0000:fffdf000       .debug$S                   10000000     ucrt:api-ms-win-crt-runtime-l1-1-0.dll
 0000:fffdf000       .debug$S                   10000000     ucrt:api-ms-win-crt-runtime-l1-1-0.dll
 0000:fffdf000       .debug$S                   10000000     ucrt:api-ms-win-crt-runtime-l1-1-0.dll
 0000:fffdf000       .debug$S                   10000000     ucrt:api-ms-win-crt-runtime-l1-1-0.dll
 0000:fffdf000       .debug$S                   10000000     ucrt:api-ms-win-crt-runtime-l1-1-0.dll
 0000:fffdf000       .debug$S                   10000000     ucrt:api-ms-win-crt-runtime-l1-1-0.dll
 0000:fffdf000       .debug$S                   10000000     ucrt:api-ms-win-crt-runtime-l1-1-0.dll
 0000:fffdf000       .debug$S                   10000000     ucrt:api-ms-win-crt-runtime-l1-1-0.dll
 0000:fffdf000       .debug$S                   10000000     ucrt:api-ms-win-crt-runtime-l1-1-0.dll
 0000:fffdf000       .debug$S                   10000000     ucrt:api-ms-win-crt-runtime-l1-1-0.dll
 0000:fffdf000       .debug$S                   10000000     ucrt:api-ms-win-crt-runtime-l1-1-0.dll
 0000:fffdf000       .debug$S                   10000000     ucrt:api-ms-win-crt-stdio-l1-1-0.dll
 0000:fffdf000       .debug$S                   10000000     ucrt:api-ms-win-crt-stdio-l1-1-0.dll
 0000:fffdf000       .debug$S                   10000000     ucrt:api-ms-win-crt-stdio-l1-1-0.dll
 0000:fffdf000       .debug$S                   10000000     ucrt:api-ms-win-crt-stdio-l1-1-0.dll
 0000:fffdf000       .debug$S                   10000000     ucrt:api-ms-win-crt-stdio-l1-1-0.dll
 0000:fffdf000       .debug$S                   10000000     ucrt:api-ms-win-crt-stdio-l1-1-0.dll
 0000:fffdf000       .debug$S                   10000000     ucrt:api-ms-win-crt-stdio-l1-1-0.dll
 0000:fffdf000       .debug$S                   10000000     ucrt:api-ms-win-crt-string-l1-1-0.dll
 0000:fffdf000       .debug$S                   10000000     ucrt:api-ms-win-crt-string-l1-1-0.dll
 0000:fffdf000       .debug$S                   10000000     ucrt:api-ms-win-crt-string-l1-1-0.dll
 0000:fffdf000       .debug$S                   10000000     ucrt:api-ms-win-crt-string-l1-1-0.dll
 0000:fffdf000       .debug$S                   10000000     ucrt:api-ms-win-crt-string-l1-1-0.dll
 0000:fffdf000       .debug$S                   10000000     ucrt:api-ms-win-crt-string-l1-1-0.dll
 0000:fffdf000       .debug$S                   10000000     ucrt:api-ms-win-crt-string-l1-1-0.dll
 0000:fffdf000       .debug$S                   10000000     ucrt:api-ms-win-crt-string-l1-1-0.dll
 0000:fffdf000       .debug$S                   10000000     ucrt:api-ms-win-crt-string-l1-1-0.dll
 0000:fffdf000       .debug$S                   10000000     ucrt:api-ms-win-crt-string-l1-1-0.dll
 0000:fffdf000       .debug$S                   10000000     ucrt:api-ms-win-crt-string-l1-1-0.dll
 0000:fffdf000       .debug$S                   10000000     ucrt:api-ms-win-crt-string-l1-1-0.dll
 0000:fffdf000       .debug$S                   10000000     ucrt:api-ms-win-crt-string-l1-1-0.dll
 0000:fffdf000       .debug$S                   10000000     ucrt:api-ms-win-crt-string-l1-1-0.dll
 0000:fffdf000       .debug$S                   10000000     ucrt:api-ms-win-crt-string-l1-1-0.dll
 0000:fffdf000       .debug$S                   10000000     ucrt:api-ms-win-crt-string-l1-1-0.dll
 0000:fffdf000       .debug$S                   10000000     ucrt:api-ms-win-crt-string-l1-1-0.dll
 0000:fffdf000       .debug$S                   10000000     advapi32:ADVAPI32.dll
 0000:fffdf000       .debug$S                   10000000     advapi32:ADVAPI32.dll
 0000:fffdf000       .debug$S                   10000000     advapi32:ADVAPI32.dll
 0000:fffdf000       .debug$S                   10000000     advapi32:ADVAPI32.dll
 0000:fffdf000       .debug$S                   10000000     advapi32:ADVAPI32.dll
 0000:fffdf000       .debug$S                   10000000     advapi32:ADVAPI32.dll
 0000:fffdf000       .debug$S                   10000000     advapi32:ADVAPI32.dll
 0000:fffdf000       .debug$S                   10000000     advapi32:ADVAPI32.dll
 0000:fffdf000       .debug$S                   10000000     advapi32:ADVAPI32.dll
 0000:fffdf000       .debug$S                   10000000     advapi32:ADVAPI32.dll
 0000:fffdf000       .debug$S                   10000000     advapi32:ADVAPI32.dll
 0000:fffdf000       .debug$S                   10000000     advapi32:ADVAPI32.dll
 0000:fffdf000       .debug$S                   10000000     advapi32:ADVAPI32.dll
 0000:fffdf000       .debug$S                   10000000     advapi32:ADVAPI32.dll
 0000:fffdf000       .debug$S                   10000000     advapi32:ADVAPI32.dll
 0000:fffdf000       .debug$S                   10000000     kernel32:KERNEL32.dll
 0000:fffdf000       .debug$S                   10000000     kernel32:KERNEL32.dll
 0000:fffdf000       .debug$S                   10000000     kernel32:KERNEL32.dll
 0000:fffdf000       .debug$S                   10000000     kernel32:KERNEL32.dll
 0000:fffdf000       .debug$S                   10000000     kernel32:KERNEL32.dll
 0000:fffdf000       .debug$S                   10000000     kernel32:KERNEL32.dll
 0000:fffdf000       .debug$S                   10000000     kernel32:KERNEL32.dll
 0000:fffdf000       .debug$S                   10000000     kernel32:KERNEL32.dll
 0000:fffdf000       .debug$S                   10000000     kernel32:KERNEL32.dll
 0000:fffdf000       .debug$S                   10000000     kernel32:KERNEL32.dll
 0000:fffdf000       .debug$S                   10000000     kernel32:KERNEL32.dll
 0000:fffdf000       .debug$S                   10000000     kernel32:KERNEL32.dll
 0000:fffdf000       .debug$S                   10000000     kernel32:KERNEL32.dll
 0000:fffdf000       .debug$S                   10000000     kernel32:KERNEL32.dll
 0000:fffdf000       .debug$S                   10000000     kernel32:KERNEL32.dll
 0000:fffdf000       .debug$S                   10000000     kernel32:KERNEL32.dll
 0000:fffdf000       .debug$S                   10000000     kernel32:KERNEL32.dll
 0000:fffdf000       .debug$S                   10000000     kernel32:KERNEL32.dll
 0000:fffdf000       .debug$S                   10000000     kernel32:KERNEL32.dll
 0000:fffdf000       .debug$S                   10000000     kernel32:KERNEL32.dll
 0000:fffdf000       .debug$S                   10000000     kernel32:KERNEL32.dll
 0000:fffdf000       .debug$S                   10000000     kernel32:KERNEL32.dll
 0000:fffdf000       .debug$S                   10000000     kernel32:KERNEL32.dll
 0000:fffdf000       .debug$S                   10000000     kernel32:KERNEL32.dll
 0000:fffdf000       .debug$S                   10000000     kernel32:KERNEL32.dll
 0000:fffdf000       .debug$S                   10000000     kernel32:KERNEL32.dll
 0000:fffdf000       .debug$S                   10000000     kernel32:KERNEL32.dll
 0000:fffdf000       .debug$S                   10000000     kernel32:KERNEL32.dll
 0000:fffdf000       .debug$S                   10000000     kernel32:KERNEL32.dll
 0000:fffdf000       .debug$S                   10000000     kernel32:KERNEL32.dll
 0000:fffdf000       .debug$S                   10000000     kernel32:KERNEL32.dll
 0000:fffdf000       .debug$S                   10000000     kernel32:KERNEL32.dll
 0000:fffdf000       .debug$S                   10000000     kernel32:KERNEL32.dll
 0000:fffdf000       .debug$S                   10000000     kernel32:KERNEL32.dll
 0000:fffdf000       .debug$S                   10000000     kernel32:KERNEL32.dll
 0000:fffdf000       .debug$S                   10000000     kernel32:KERNEL32.dll
 0000:fffdf000       .debug$S                   10000000     kernel32:KERNEL32.dll
 0000:fffdf000       .debug$S                   10000000     kernel32:KERNEL32.dll
 0000:fffdf000       .debug$S                   10000000     kernel32:KERNEL32.dll
 0000:fffdf000       .debug$S                   10000000     kernel32:KERNEL32.dll
 0000:fffdf000       .debug$S                   10000000     kernel32:KERNEL32.dll
 0000:fffdf000       .debug$S                   10000000     kernel32:KERNEL32.dll
 0000:fffdf000       .debug$S                   10000000     kernel32:KERNEL32.dll
 0000:fffdf000       .debug$S                   10000000     kernel32:KERNEL32.dll
 0000:fffdf000       .debug$S                   10000000     kernel32:KERNEL32.dll
 0000:fffdf000       .debug$S                   10000000     kernel32:KERNEL32.dll
 0000:fffdf000       .debug$S                   10000000     kernel32:KERNEL32.dll
 0000:fffdf000       .debug$S                   10000000     kernel32:KERNEL32.dll
 0000:fffdf000       .debug$S                   10000000     kernel32:KERNEL32.dll
 0000:fffdf000       .debug$S                   10000000     kernel32:KERNEL32.dll
 0000:fffdf000       .debug$S                   10000000     kernel32:KERNEL32.dll
 0000:fffdf000       .debug$S                   10000000     kernel32:KERNEL32.dll
 0000:fffdf000       .debug$S                   10000000     kernel32:KERNEL32.dll
 0000:fffdf000       .debug$S                   10000000     kernel32:KERNEL32.dll
 0000:fffdf000       .debug$S                   10000000     kernel32:KERNEL32.dll
 0000:fffdf000       .debug$S                   10000000     kernel32:KERNEL32.dll
 0000:fffdf000       .debug$S                   10000000     kernel32:KERNEL32.dll
 0000:fffdf000       .debug$S                   10000000     kernel32:KERNEL32.dll
 0000:fffdf000       .debug$S                   10000000     kernel32:KERNEL32.dll
 0000:fffdf000       .debug$S                   10000000     kernel32:KERNEL32.dll
 0000:fffdf000       .debug$S                   10000000     kernel32:KERNEL32.dll
 0000:fffdf000       .debug$S                   10000000     kernel32:KERNEL32.dll
 0000:fffdf000       .debug$S                   10000000     kernel32:KERNEL32.dll
 0000:fffdf000       .debug$S                   10000000     kernel32:KERNEL32.dll
 0000:fffdf000       .debug$S                   10000000     kernel32:KERNEL32.dll
 0000:fffdf000       .debug$S                   10000000     kernel32:KERNEL32.dll
 0000:fffdf000       .debug$S                   10000000     kernel32:KERNEL32.dll
 0000:fffdf000       .debug$S                   10000000     kernel32:KERNEL32.dll
 0000:fffdf000       .debug$S                   10000000     kernel32:KERNEL32.dll
 0000:fffdf000       .debug$S                   10000000     kernel32:KERNEL32.dll
 0000:fffdf000       .debug$S                   10000000     kernel32:KERNEL32.dll
 0000:fffdf000       .debug$S                   10000000     kernel32:KERNEL32.dll
 0000:fffdf000       .debug$S                   10000000     kernel32:KERNEL32.dll
 0000:fffdf000       .debug$S                   10000000     kernel32:KERNEL32.dll
 0000:fffdf000       .debug$S                   10000000     kernel32:KERNEL32.dll
 0000:fffdf000       .debug$S                   10000000     kernel32:KERNEL32.dll
 0000:fffdf000       .debug$S                   10000000     kernel32:KERNEL32.dll
 0000:fffdf000       .debug$S                   10000000     kernel32:KERNEL32.dll
 0000:fffdf000       .debug$S                   10000000     kernel32:KERNEL32.dll
 0000:fffdf000       .debug$S                   10000000     kernel32:KERNEL32.dll
 0000:fffdf000       .debug$S                   10000000     kernel32:KERNEL32.dll
 0000:fffdf000       .debug$S                   10000000     kernel32:KERNEL32.dll
 0000:fffdf000       .debug$S                   10000000     kernel32:KERNEL32.dll
 0000:fffdf000       .debug$S                   10000000     kernel32:KERNEL32.dll
 0000:fffdf000       .debug$S                   10000000     kernel32:KERNEL32.dll
 0000:fffdf000       .debug$S                   10000000     kernel32:KERNEL32.dll
 0000:fffdf000       .debug$S                   10000000     kernel32:KERNEL32.dll
 0000:fffdf000       .debug$S                   10000000     kernel32:KERNEL32.dll
 0000:fffdf000       .debug$S                   10000000     kernel32:KERNEL32.dll
 0000:fffdf000       .debug$S                   10000000     kernel32:KERNEL32.dll
 0000:fffdf000       .debug$S                   10000000     kernel32:KERNEL32.dll
 0000:fffdf000       .debug$S                   10000000     kernel32:KERNEL32.dll
 0000:fffdf000       .debug$S                   10000000     kernel32:KERNEL32.dll
 0000:fffdf000       .debug$S                   10000000     kernel32:KERNEL32.dll
 0000:fffdf000       .debug$S                   10000000     kernel32:KERNEL32.dll
 0000:fffdf000       .debug$S                   10000000     kernel32:KERNEL32.dll
 0000:fffdf000       .debug$S                   10000000     kernel32:KERNEL32.dll
 0000:fffdf000       .debug$S                   10000000     kernel32:KERNEL32.dll
 0000:fffdf000       .debug$S                   10000000     kernel32:KERNEL32.dll
 0000:fffdf000       .debug$S                   10000000     kernel32:KERNEL32.dll
 0000:fffdf000       .debug$S                   10000000     kernel32:KERNEL32.dll
 0000:fffdf000       .debug$S                   10000000     kernel32:KERNEL32.dll
 0000:fffdf000       .debug$S                   10000000     kernel32:KERNEL32.dll
 0000:fffdf000       .debug$S                   10000000     kernel32:KERNEL32.dll
 0000:fffdf000       .debug$S                   10000000     kernel32:KERNEL32.dll
 0000:fffdf000       .debug$S                   10000000     shell32:SHELL32.dll
 0000:fffdf000       .debug$S                   10000000     shell32:SHELL32.dll
 0000:fffdf000       .debug$S                   10000000     version:VERSION.dll
 0000:fffdf000       .debug$S                   10000000     version:VERSION.dll
 0000:fffdf000       .debug$S                   10000000     version:VERSION.dll
 0000:fffdf000       .debug$S                   10000000     jvm:jvm.dll
 0000:fffdf000       .debug$S                   10000000     jvm:jvm.dll
 0000:fffdf000       .debug$S                   10000000     jvm:jvm.dll
 0000:fffdf000       .debug$S                   10000000     jvm:jvm.dll
 0000:fffdf000       .debug$S                   10000000     jvm:jvm.dll
 0000:fffdf000       .debug$S                   10000000     jvm:jvm.dll
 0000:fffdf000       .debug$S                   10000000     jvm:jvm.dll
 0000:fffdf000       .debug$S                   10000000     jvm:jvm.dll
 0000:fffdf000       .debug$S                   10000000     jvm:jvm.dll
 0000:fffdf000       .debug$S                   10000000     jvm:jvm.dll
 0000:fffdf000       .debug$S                   10000000     jvm:jvm.dll
 0000:fffdf000       .debug$S                   10000000     jvm:jvm.dll
 0000:fffdf000       .debug$S                   10000000     jvm:jvm.dll
 0000:fffdf000       .debug$S                   10000000     jvm:jvm.dll
 0000:fffdf000       .debug$S                   10000000     jvm:jvm.dll
 0000:fffdf000       .debug$S                   10000000     jvm:jvm.dll
 0000:fffdf000       .debug$S                   10000000     jvm:jvm.dll
 0000:fffdf000       .debug$S                   10000000     jvm:jvm.dll
 0000:fffdf000       .debug$S                   10000000     jvm:jvm.dll
 0000:fffdf000       .debug$S                   10000000     jvm:jvm.dll
 0000:fffdf000       .debug$S                   10000000     jvm:jvm.dll
 0000:fffdf000       .debug$S                   10000000     jvm:jvm.dll
 0000:fffdf000       .debug$S                   10000000     jvm:jvm.dll
 0000:fffdf000       .debug$S                   10000000     jvm:jvm.dll
 0000:fffdf000       .debug$S                   10000000     jvm:jvm.dll
 0000:fffdf000       .debug$S                   10000000     jvm:jvm.dll
 0000:fffdf000       .debug$S                   10000000     jvm:jvm.dll
 0000:fffdf000       .debug$S                   10000000     jvm:jvm.dll
 0000:fffdf000       .debug$S                   10000000     jvm:jvm.dll
 0000:fffdf000       .debug$S                   10000000     jvm:jvm.dll
 0000:fffdf000       .debug$S                   10000000     jvm:jvm.dll
 0000:fffdf000       .debug$S                   10000000     jvm:jvm.dll
 0000:fffdf000       .debug$S                   10000000     jvm:jvm.dll
 0000:fffdf000       .debug$S                   10000000     jvm:jvm.dll
 0000:fffdf000       .debug$S                   10000000     jvm:jvm.dll
 0000:fffdf000       .debug$S                   10000000     jvm:jvm.dll
 0000:fffdf000       .debug$S                   10000000     jvm:jvm.dll
 0000:fffdf000       .debug$S                   10000000     jvm:jvm.dll
 0000:fffdf000       .debug$S                   10000000     jvm:jvm.dll
 0000:fffdf000       .debug$S                   10000000     jvm:jvm.dll
 0000:fffdf000       .debug$S                   10000000     jvm:jvm.dll
 0000:fffdf000       .debug$S                   10000000     jvm:jvm.dll
 0000:fffdf000       .debug$S                   10000000     jvm:jvm.dll
 0000:fffdf000       .debug$S                   10000000     jvm:jvm.dll
 0000:fffdf000       .debug$S                   10000000     jvm:jvm.dll
 0000:fffdf000       .debug$S                   10000000     jvm:jvm.dll
 0000:fffdf000       .debug$S                   10000000     jvm:jvm.dll
 0000:fffdf000       .debug$S                   10000000     jvm:jvm.dll
 0000:fffdf000       .debug$S                   10000000     jvm:jvm.dll
 0000:fffdf000       .debug$S                   10000000     jvm:jvm.dll
 0000:fffdf000       .debug$S                   10000000     jvm:jvm.dll
 0000:fffdf000       .debug$S                   10000000     jvm:jvm.dll
 0000:fffdf000       .debug$S                   10000000     jvm:jvm.dll
 0000:fffdf000       .debug$S                   10000000     jvm:jvm.dll
 0000:fffdf000       .debug$S                   10000000     jvm:jvm.dll
 0000:fffdf000       .debug$S                   10000000     jvm:jvm.dll
 0000:fffdf000       .debug$S                   10000000     jvm:jvm.dll
 0000:fffdf000       .debug$S                   10000000     jvm:jvm.dll
 0000:fffdf000       .debug$S                   10000000     jvm:jvm.dll
 0000:fffdf000       .debug$S                   10000000     jvm:jvm.dll
 0000:fffdf000       .debug$S                   10000000     jvm:jvm.dll
 0000:fffdf000       .debug$S                   10000000     jvm:jvm.dll
 0000:fffdf000       .debug$S                   10000000     jvm:jvm.dll
 0000:fffdf000       .debug$S                   10000000     jvm:jvm.dll
 0000:fffdf000       .debug$S                   10000000     jvm:jvm.dll
 0000:fffdf000       .debug$S                   10000000     jvm:jvm.dll
 0000:fffdf000       .debug$S                   10000000     jvm:jvm.dll
 0000:fffdf000       .debug$S                   10000000     jvm:jvm.dll
 0000:fffdf000       .debug$S                   10000000     jvm:jvm.dll
 0000:fffdf000       .debug$S                   10000000     jvm:jvm.dll
 0000:fffdf000       .debug$S                   10000000     jvm:jvm.dll
 0000:fffdf000       .debug$S                   10000000     jvm:jvm.dll
 0000:fffdf000       .debug$S                   10000000     jvm:jvm.dll
 0000:fffdf000       .debug$S                   10000000     jvm:jvm.dll
 0000:fffdf000       .debug$S                   10000000     jvm:jvm.dll
 0000:fffdf000       .debug$S                   10000000     jvm:jvm.dll
 0000:fffdf000       .debug$S                   10000000     jvm:jvm.dll
 0000:fffdf000       .debug$S                   10000000     jvm:jvm.dll
 0000:fffdf000       .debug$S                   10000000     jvm:jvm.dll
 0000:fffdf000       .debug$S                   10000000     jvm:jvm.dll
 0000:fffdf000       .debug$S                   10000000     jvm:jvm.dll
 0000:fffdf000       .debug$S                   10000000     jvm:jvm.dll
 0000:fffdf000       .debug$S                   10000000     jvm:jvm.dll
 0000:fffdf000       .debug$S                   10000000     jvm:jvm.dll
 0000:fffdf000       .debug$S                   10000000     jvm:jvm.dll
 0000:fffdf000       .debug$S                   10000000     jvm:jvm.dll
 0000:fffdf000       .debug$S                   10000000     jvm:jvm.dll
 0000:fffdf000       .debug$S                   10000000     jvm:jvm.dll
 0000:fffdf000       .debug$S                   10000000     jvm:jvm.dll
 0000:fffdf000       .debug$S                   10000000     jvm:jvm.dll
 0000:fffdf000       .debug$S                   10000000     jvm:jvm.dll
 0000:fffdf000       .debug$S                   10000000     jvm:jvm.dll
 0000:fffdf000       .debug$S                   10000000     jvm:jvm.dll
 0000:fffdf000       .debug$S                   10000000     jvm:jvm.dll
 0000:fffdf000       .debug$S                   10000000     jvm:jvm.dll
 0000:fffdf000       .debug$S                   10000000     jvm:jvm.dll
 0000:fffdf000       .debug$S                   10000000     jvm:jvm.dll
 0000:fffdf000       .debug$S                   10000000     jvm:jvm.dll
 0000:fffdf000       .debug$S                   10000000     jvm:jvm.dll
 0000:fffdf000       .debug$S                   10000000     jvm:jvm.dll
 0000:fffdf000       .debug$S                   10000000     jvm:jvm.dll
 0000:fffdf000       .debug$S                   10000000     jvm:jvm.dll
 0000:fffdf000       .debug$S                   10000000     jvm:jvm.dll
 0000:fffdf000       .debug$S                   10000000     jvm:jvm.dll
 0000:fffdf000       .debug$S                   10000000     jvm:jvm.dll
 0000:fffdf000       .debug$S                   10000000     jvm:jvm.dll
 0000:fffdf000       .debug$S                   10000000     jvm:jvm.dll
 0000:fffdf000       .debug$S                   10000000     jvm:jvm.dll
 0000:fffdf000       .debug$S                   10000000     jvm:jvm.dll
 0000:fffdf000       .debug$S                   10000000     jvm:jvm.dll
 0000:fffdf000       .debug$S                   10000000     jvm:jvm.dll
 0000:fffdf000       .debug$S                   10000000     jvm:jvm.dll
 0000:fffdf000       .debug$S                   10000000     jvm:jvm.dll
 0000:fffdf000       .debug$S                   10000000     jvm:jvm.dll
 0000:fffdf000       .debug$S                   10000000     jvm:jvm.dll
 0000:fffdf000       .debug$S                   10000000     jvm:jvm.dll
 0000:fffdf000       .debug$S                   10000000     jvm:jvm.dll
 0000:fffdf000       .debug$S                   10000000     jvm:jvm.dll
 0000:fffdf000       .debug$S                   10000000     jvm:jvm.dll
 0000:fffdf000       .debug$S                   10000000     jvm:jvm.dll
 0000:fffdf000       .debug$S                   10000000     jvm:jvm.dll
 0000:fffdf000       .debug$S                   10000000     jvm:jvm.dll
 0000:fffdf000       .debug$S                   10000000     jvm:jvm.dll
 0000:fffdf000       .debug$S                   10000000     jvm:jvm.dll
 0000:fffdf000       .debug$S                   10000000     jvm:jvm.dll
 0000:fffdf000       .debug$S                   10000000     jvm:jvm.dll
 0000:fffdf000       .debug$S                   10000000     jvm:jvm.dll
 0000:fffdf000       .debug$S                   10000000     jvm:jvm.dll
 0000:fffdf000       .debug$S                   10000000     jvm:jvm.dll
 0000:fffdf000       .debug$S                   10000000     jvm:jvm.dll
 0000:fffdf000       .debug$S                   10000000     jvm:jvm.dll
 0000:fffdf000       .debug$S                   10000000     jvm:jvm.dll
 0000:fffdf000       .debug$S                   10000000     jvm:jvm.dll
 0000:fffdf000       .debug$S                   10000000     jvm:jvm.dll
 0000:fffdf000       .debug$S                   10000000     jvm:jvm.dll
 0000:fffdf000       .debug$S                   10000000     jvm:jvm.dll
 0000:fffdf000       .debug$S                   10000000     jvm:jvm.dll
 0000:fffdf000       .debug$S                   10000000     jvm:jvm.dll
 0000:fffdf000       .debug$S                   10000000     jvm:jvm.dll
 0000:fffdf000       .debug$S                   10000000     jvm:jvm.dll
 0000:fffdf000       .debug$S                   10000000     jvm:jvm.dll
 0000:fffdf000       .debug$S                   10000000     jvm:jvm.dll
 0000:fffdf000       .debug$S                   10000000     jvm:jvm.dll
 0000:fffdf000       .debug$S                   10000000     jvm:jvm.dll
 0001:000009db       _getUTF                    100019db f   ClassLoader.obj
 0001:000029f6       _findJniFunction           100039f6 f   NativeLibraries.obj
 0001:00002aaf       _initIDs                   10003aaf f   NativeLibraries.obj
 0001:00002c6c       _environmentBlock9x        10003c6c f   ProcessEnvironment_md.obj
 0001:000032fe       _getCmdlineInfo            100042fe f   ProcessHandleImpl_win.obj
 0001:000033f4       _getStartTime              100043f4 f   ProcessHandleImpl_win.obj
 0001:00003441       _getStatInfo               10004441 f   ProcessHandleImpl_win.obj
 0001:00003533       _procToUser                10004533 f   ProcessHandleImpl_win.obj
 0001:00003935       _initHolder                10004935 f   ProcessImpl_md.obj
 0001:00003a00       _processCreate             10004a00 f   ProcessImpl_md.obj
 0001:00003d13       _releaseHolder             10004d13 f   ProcessImpl_md.obj
 0001:00003d69       _win32Error                10004d69 f   ProcessImpl_md.obj
 0001:000041cc       _check                     100051cc f   SecurityManager.obj
 0001:00004d77       _cpchars                   10005d77 f   System.obj
 0001:00004e5c       _customZoneName            10005e5c f   TimeZone_md.obj
 0001:00004fb3       _getValueInRegistry        10005fb3 f   TimeZone_md.obj
 0001:0000507e       _getWinTimeZone            1000607e f   TimeZone_md.obj
 0001:000054a1       _matchJavaTZ               100064a1 f   TimeZone_md.obj
 0001:000065ac       _getFileInformation        100075ac f   WinNTFileSystem_md.obj
 0001:000066ed       _getFinalAttributesUnixSocket 100076ed f   WinNTFileSystem_md.obj
 0001:000067a0       _getFinalPath              100077a0 f   WinNTFileSystem_md.obj
 0001:000068eb       _isReservedDeviceNameW     100078eb f   WinNTFileSystem_md.obj
 0001:000069e4       _removeFileOrDirectory     100079e4 f   WinNTFileSystem_md.obj
 0001:00006f30       _wcp                       10007f30 f   canonicalize_md.obj
 0001:00006f97       _wdots                     10007f97 f   canonicalize_md.obj
 0001:00007012       _wnextsep                  10008012 f   canonicalize_md.obj
 0001:00007067       _isJvmIdentifier           10008067 f   check_classname.obj
 0001:00007096       _next_utf2unicode          10008096 f   check_classname.obj
 0001:0000714b       _skip_over_field_signature 1000814b f   check_classname.obj
 0001:000071dc       _skip_over_fieldname       100081dc f   check_classname.obj
 0001:00007347       _outOfBounds               10008347 f   io_util.obj
 0001:00007a9f       _handleNonSeekAvailable    10008a9f f   io_util_md.obj
 0001:00007b4d       _handleStdinAvailable      10008b4d f   io_util_md.obj
 0001:00007e9a       _writeInternal             10008e9a f   io_util_md.obj
 0001:00008496       _SetupI18nProps            10009496 f   java_props_md.obj
 0001:0000868c       _cpu_isalist               1000968c f   java_props_md.obj
 0001:00008715       _getConsoleEncoding        10009715 f   java_props_md.obj
 0001:00008776       _getEncodingInternal       10009776 f   java_props_md.obj
 0001:00009aa7       _getString646_USChars      1000aaa7 f   jni_util.obj
 0001:00009b54       _getString8859_1Chars      1000ab54 f   jni_util.obj
 0001:00009c0e       _getStringBytes            1000ac0e f   jni_util.obj
 0001:00009cf8       _getStringCp1252Chars      1000acf8 f   jni_util.obj
 0001:00009f0c       _getStringUTF8             1000af0c f   jni_util.obj
 0001:0000a055       _jnuEncodingSupported      1000b055 f   jni_util.obj
 0001:0000a091       _newSizedString8859_1      1000b091 f   jni_util.obj
 0001:0000a12d       _newSizedStringJava        1000b12d f   jni_util.obj
 0001:0000a1d3       _newString646_US           1000b1d3 f   jni_util.obj
 0001:0000a29d       _newStringCp1252           1000b29d f   jni_util.obj
 0001:0000c528       $LN43                      1000d528     fdlibm:e_atan2.obj
 0001:0000c538       $LN44                      1000d538     fdlibm:e_atan2.obj
 0001:0000c548       $LN45                      1000d548     fdlibm:e_atan2.obj
 0001:0000ef5c       $LN97                      1000ff5c     fdlibm:k_rem_pio2.obj
 0001:00010580       $$000000                   10011580     MSVCRT:lldiv.obj
 0001:00010630       $$000000                   10011630     MSVCRT:llmul.obj
 0001:00010670       $$000000                   10011670     MSVCRT:ulldiv.obj
 0001:000106e0       $$000000                   100116e0     MSVCRT:chkstk.obj
 0001:00010710       $$000000                   10011710     MSVCRT:sehprolg4gs.obj
 0001:00010797       ?dllmain_crt_dispatch@@YGHQAUHINSTANCE__@@KQAX@Z 10011797 f   MSVCRT:dll_dllmain.obj
 0001:000107ea       ?dllmain_crt_process_attach@@YAHQAUHINSTANCE__@@QAX@Z 100117ea f   MSVCRT:dll_dllmain.obj
 0001:000108f1       ?dllmain_crt_process_detach@@YAH_N@Z 100118f1 f   MSVCRT:dll_dllmain.obj
 0001:000109a1       ?dllmain_dispatch@@YAHQAUHINSTANCE__@@KQAX@Z 100119a1 f   MSVCRT:dll_dllmain.obj
 0001:00010aac       ?dllmain_raw@@YGHQAUHINSTANCE__@@KQAX@Z 10011aac f   MSVCRT:dll_dllmain.obj
 0001:00010b00       $$000000                   10011b00     MSVCRT:sehprolg4.obj
 0001:00010b58       ___get_entropy             10011b58 f   MSVCRT:gs_support.obj
 0001:00010c47       ?find_pe_section@@YAPAU_IMAGE_SECTION_HEADER@@QAEI@Z 10011c47 f   MSVCRT:utility.obj
 0002:00001ca0       _GS_ExceptionPointers      10014ca0     MSVCRT:gs_report.obj
 0002:000020e8       __sehtable$_getHomeFromShell32 100150e8     java_props_md.obj
 0002:00002108       __sehtable$?dllmain_crt_process_attach@@YAHQAUHINSTANCE__@@QAX@Z 10015108     MSVCRT:dll_dllmain.obj
 0002:00002128       __sehtable$?dllmain_crt_process_detach@@YAH_N@Z 10015128     MSVCRT:dll_dllmain.obj
 0002:00002150       __sehtable$?dllmain_dispatch@@YAHQAUHINSTANCE__@@KQAX@Z 10015150     MSVCRT:dll_dllmain.obj
 0002:00002170       __sehtable$___scrt_is_nonwritable_in_current_image 10015170     MSVCRT:utility.obj
 0002:00002210       .edata                     10015210     java.exp
 0002:00002238       rgpv                       10015238     java.exp
 0002:000026d0       rgszName                   100156d0     java.exp
 0002:00002b68       rgwOrd                     10015b68     java.exp
 0002:00002db4       szName                     10015db4     java.exp
 0002:00002dbd       $N00001                    10015dbd     java.exp
 0002:00002dd4       $N00002                    10015dd4     java.exp
 0002:00002de7       $N00003                    10015de7     java.exp
 0002:00002df8       $N00004                    10015df8     java.exp
 0002:00002e0e       $N00005                    10015e0e     java.exp
 0002:00002e1c       $N00006                    10015e1c     java.exp
 0002:00002e31       $N00007                    10015e31     java.exp
 0002:00002e4b       $N00008                    10015e4b     java.exp
 0002:00002e66       $N00009                    10015e66     java.exp
 0002:00002e79       $N00010                    10015e79     java.exp
 0002:00002e91       $N00011                    10015e91     java.exp
 0002:00002e9f       $N00012                    10015e9f     java.exp
 0002:00002eb6       $N00013                    10015eb6     java.exp
 0002:00002ed3       $N00014                    10015ed3     java.exp
 0002:00002ef2       $N00015                    10015ef2     java.exp
 0002:00002f0d       $N00016                    10015f0d     java.exp
 0002:00002f21       $N00017                    10015f21     java.exp
 0002:00002f3a       $N00018                    10015f3a     java.exp
 0002:00002f5d       $N00019                    10015f5d     java.exp
 0002:00002f70       $N00020                    10015f70     java.exp
 0002:00002f9b       $N00021                    10015f9b     java.exp
 0002:00002faf       $N00022                    10015faf     java.exp
 0002:00002fd0       $N00023                    10015fd0     java.exp
 0002:00002ffb       $N00024                    10015ffb     java.exp
 0002:0000301e       $N00025                    1001601e     java.exp
 0002:00003036       $N00026                    10016036     java.exp
 0002:0000305b       $N00027                    1001605b     java.exp
 0002:00003080       $N00028                    10016080     java.exp
 0002:0000309a       $N00029                    1001609a     java.exp
 0002:000030bb       $N00030                    100160bb     java.exp
 0002:000030d8       $N00031                    100160d8     java.exp
 0002:000030e8       $N00032                    100160e8     java.exp
 0002:00003106       $N00033                    10016106     java.exp
 0002:00003127       $N00034                    10016127     java.exp
 0002:00003145       $N00035                    10016145     java.exp
 0002:00003172       $N00036                    10016172     java.exp
 0002:00003198       $N00037                    10016198     java.exp
 0002:000031c2       $N00038                    100161c2     java.exp
 0002:000031ec       $N00039                    100161ec     java.exp
 0002:00003213       $N00040                    10016213     java.exp
 0002:00003237       $N00041                    10016237     java.exp
 0002:00003262       $N00042                    10016262     java.exp
 0002:0000328a       $N00043                    1001628a     java.exp
 0002:000032b2       $N00044                    100162b2     java.exp
 0002:000032d9       $N00045                    100162d9     java.exp
 0002:00003303       $N00046                    10016303     java.exp
 0002:00003329       $N00047                    10016329     java.exp
 0002:00003354       $N00048                    10016354     java.exp
 0002:0000337b       $N00049                    1001637b     java.exp
 0002:000033a4       $N00050                    100163a4     java.exp
 0002:000033cc       $N00051                    100163cc     java.exp
 0002:000033f4       $N00052                    100163f4     java.exp
 0002:00003421       $N00053                    10016421     java.exp
 0002:00003459       $N00054                    10016459     java.exp
 0002:00003486       $N00055                    10016486     java.exp
 0002:000034b6       $N00056                    100164b6     java.exp
 0002:000034df       $N00057                    100164df     java.exp
 0002:00003507       $N00058                    10016507     java.exp
 0002:0000352f       $N00059                    1001652f     java.exp
 0002:00003556       $N00060                    10016556     java.exp
 0002:00003582       $N00061                    10016582     java.exp
 0002:000035aa       $N00062                    100165aa     java.exp
 0002:000035d6       $N00063                    100165d6     java.exp
 0002:000035ff       $N00064                    100165ff     java.exp
 0002:0000362c       $N00065                    1001662c     java.exp
 0002:0000365b       $N00066                    1001665b     java.exp
 0002:00003694       $N00067                    10016694     java.exp
 0002:000036c1       $N00068                    100166c1     java.exp
 0002:000036f2       $N00069                    100166f2     java.exp
 0002:00003729       $N00070                    10016729     java.exp
 0002:00003752       $N00071                    10016752     java.exp
 0002:00003788       $N00072                    10016788     java.exp
 0002:000037bb       $N00073                    100167bb     java.exp
 0002:000037f0       $N00074                    100167f0     java.exp
 0002:0000381b       $N00075                    1001681b     java.exp
 0002:00003848       $N00076                    10016848     java.exp
 0002:00003873       $N00077                    10016873     java.exp
 0002:0000389b       $N00078                    1001689b     java.exp
 0002:000038c1       $N00079                    100168c1     java.exp
 0002:000038ec       $N00080                    100168ec     java.exp
 0002:00003915       $N00081                    10016915     java.exp
 0002:0000394a       $N00082                    1001694a     java.exp
 0002:00003979       $N00083                    10016979     java.exp
 0002:000039a6       $N00084                    100169a6     java.exp
 0002:000039d2       $N00085                    100169d2     java.exp
 0002:000039fe       $N00086                    100169fe     java.exp
 0002:00003a2a       $N00087                    10016a2a     java.exp
 0002:00003a5c       $N00088                    10016a5c     java.exp
 0002:00003a8c       $N00089                    10016a8c     java.exp
 0002:00003aba       $N00090                    10016aba     java.exp
 0002:00003adc       $N00091                    10016adc     java.exp
 0002:00003b07       $N00092                    10016b07     java.exp
 0002:00003b31       $N00093                    10016b31     java.exp
 0002:00003b55       $N00094                    10016b55     java.exp
 0002:00003b7d       $N00095                    10016b7d     java.exp
 0002:00003bab       $N00096                    10016bab     java.exp
 0002:00003bd6       $N00097                    10016bd6     java.exp
 0002:00003c01       $N00098                    10016c01     java.exp
 0002:00003c29       $N00099                    10016c29     java.exp
 0002:00003c4f       $N00100                    10016c4f     java.exp
 0002:00003c7a       $N00101                    10016c7a     java.exp
 0002:00003cac       $N00102                    10016cac     java.exp
 0002:00003cd0       $N00103                    10016cd0     java.exp
 0002:00003cf8       $N00104                    10016cf8     java.exp
 0002:00003d35       $N00105                    10016d35     java.exp
 0002:00003d57       $N00106                    10016d57     java.exp
 0002:00003d8d       $N00107                    10016d8d     java.exp
 0002:00003dc2       $N00108                    10016dc2     java.exp
 0002:00003df8       $N00109                    10016df8     java.exp
 0002:00003e26       $N00110                    10016e26     java.exp
 0002:00003e59       $N00111                    10016e59     java.exp
 0002:00003e8e       $N00112                    10016e8e     java.exp
 0002:00003ebd       $N00113                    10016ebd     java.exp
 0002:00003eeb       $N00114                    10016eeb     java.exp
 0002:00003f18       $N00115                    10016f18     java.exp
 0002:00003f51       $N00116                    10016f51     java.exp
 0002:00003f7c       $N00117                    10016f7c     java.exp
 0002:00003fa2       $N00118                    10016fa2     java.exp
 0002:00003fd4       $N00119                    10016fd4     java.exp
 0002:00004001       $N00120                    10017001     java.exp
 0002:0000402e       $N00121                    1001702e     java.exp
 0002:0000405c       $N00122                    1001705c     java.exp
 0002:0000408f       $N00123                    1001708f     java.exp
 0002:000040bf       $N00124                    100170bf     java.exp
 0002:000040f3       $N00125                    100170f3     java.exp
 0002:0000412e       $N00126                    1001712e     java.exp
 0002:0000415c       $N00127                    1001715c     java.exp
 0002:00004181       $N00128                    10017181     java.exp
 0002:0000419e       $N00129                    1001719e     java.exp
 0002:000041c2       $N00130                    100171c2     java.exp
 0002:000041e8       $N00131                    100171e8     java.exp
 0002:0000421a       $N00132                    1001721a     java.exp
 0002:00004240       $N00133                    10017240     java.exp
 0002:00004262       $N00134                    10017262     java.exp
 0002:000042af       $N00135                    100172af     java.exp
 0002:000042ff       $N00136                    100172ff     java.exp
 0002:00004338       $N00137                    10017338     java.exp
 0002:00004373       $N00138                    10017373     java.exp
 0002:000043af       $N00139                    100173af     java.exp
 0002:000043db       $N00140                    100173db     java.exp
 0002:000043fe       $N00141                    100173fe     java.exp
 0002:00004421       $N00142                    10017421     java.exp
 0002:00004445       $N00143                    10017445     java.exp
 0002:00004468       $N00144                    10017468     java.exp
 0002:0000448a       $N00145                    1001748a     java.exp
 0002:000044ad       $N00146                    100174ad     java.exp
 0002:000044d1       $N00147                    100174d1     java.exp
 0002:000044f5       $N00148                    100174f5     java.exp
 0002:00004519       $N00149                    10017519     java.exp
 0002:0000453b       $N00150                    1001753b     java.exp
 0002:0000455d       $N00151                    1001755d     java.exp
 0002:00004580       $N00152                    10017580     java.exp
 0002:000045a3       $N00153                    100175a3     java.exp
 0002:000045c5       $N00154                    100175c5     java.exp
 0002:000045e8       $N00155                    100175e8     java.exp
 0002:00004612       $N00156                    10017612     java.exp
 0002:00004632       $N00157                    10017632     java.exp
 0002:0000465d       $N00158                    1001765d     java.exp
 0002:00004686       $N00159                    10017686     java.exp
 0002:000046af       $N00160                    100176af     java.exp
 0002:000046d1       $N00161                    100176d1     java.exp
 0002:000046f2       $N00162                    100176f2     java.exp
 0002:00004714       $N00163                    10017714     java.exp
 0002:00004741       $N00164                    10017741     java.exp
 0002:0000476a       $N00165                    1001776a     java.exp
 0002:00004798       $N00166                    10017798     java.exp
 0002:000047d7       $N00167                    100177d7     java.exp
 0002:00004819       $N00168                    10017819     java.exp
 0002:0000484b       $N00169                    1001784b     java.exp
 0002:00004872       $N00170                    10017872     java.exp
 0002:000048b2       $N00171                    100178b2     java.exp
 0002:000048ea       $N00172                    100178ea     java.exp
 0002:00004915       $N00173                    10017915     java.exp
 0002:00004951       $N00174                    10017951     java.exp
 0002:00004976       $N00175                    10017976     java.exp
 0002:000049a2       $N00176                    100179a2     java.exp
 0002:000049cb       $N00177                    100179cb     java.exp
 0002:000049f4       $N00178                    100179f4     java.exp
 0002:00004a1f       $N00179                    10017a1f     java.exp
 0002:00004a49       $N00180                    10017a49     java.exp
 0002:00004a71       $N00181                    10017a71     java.exp
 0002:00004a9c       $N00182                    10017a9c     java.exp
 0002:00004ac5       $N00183                    10017ac5     java.exp
 0002:00004aef       $N00184                    10017aef     java.exp
 0002:00004b1e       $N00185                    10017b1e     java.exp
 0002:00004b48       $N00186                    10017b48     java.exp
 0002:00004b6d       $N00187                    10017b6d     java.exp
 0002:00004b99       $N00188                    10017b99     java.exp
 0002:00004bc2       $N00189                    10017bc2     java.exp
 0002:00004beb       $N00190                    10017beb     java.exp
 0002:00004c16       $N00191                    10017c16     java.exp
 0002:00004c40       $N00192                    10017c40     java.exp
 0002:00004c68       $N00193                    10017c68     java.exp
 0002:00004c91       $N00194                    10017c91     java.exp
 0002:00004cbb       $N00195                    10017cbb     java.exp
 0002:00004cef       $N00196                    10017cef     java.exp
 0002:00004d2c       $N00197                    10017d2c     java.exp
 0002:00004d64       $N00198                    10017d64     java.exp
 0002:00004dab       $N00199                    10017dab     java.exp
 0002:00004df3       $N00200                    10017df3     java.exp
 0002:00004e2f       $N00201                    10017e2f     java.exp
 0002:00004e73       $N00202                    10017e73     java.exp
 0002:00004ea3       $N00203                    10017ea3     java.exp
 0002:00004ed3       $N00204                    10017ed3     java.exp
 0002:00004f10       $N00205                    10017f10     java.exp
 0002:00004f51       $N00206                    10017f51     java.exp
 0002:00004f8e       $N00207                    10017f8e     java.exp
 0002:00004fd2       $N00208                    10017fd2     java.exp
 0002:0000500e       $N00209                    1001800e     java.exp
 0002:00005046       $N00210                    10018046     java.exp
 0002:00005078       $N00211                    10018078     java.exp
 0002:000050ac       $N00212                    100180ac     java.exp
 0002:000050e1       $N00213                    100180e1     java.exp
 0002:0000510e       $N00214                    1001810e     java.exp
 0002:00005140       $N00215                    10018140     java.exp
 0002:00005176       $N00216                    10018176     java.exp
 0002:000051ab       $N00217                    100181ab     java.exp
 0002:000051db       $N00218                    100181db     java.exp
 0002:0000520d       $N00219                    1001820d     java.exp
 0002:0000523d       $N00220                    1001823d     java.exp
 0002:00005271       $N00221                    10018271     java.exp
 0002:0000529f       $N00222                    1001829f     java.exp
 0002:000052c9       $N00223                    100182c9     java.exp
 0002:000052f2       $N00224                    100182f2     java.exp
 0002:00005323       $N00225                    10018323     java.exp
 0002:00005348       $N00226                    10018348     java.exp
 0002:0000536d       $N00227                    1001836d     java.exp
 0002:00005391       $N00228                    10018391     java.exp
 0002:000053b5       $N00229                    100183b5     java.exp
 0002:000053dd       $N00230                    100183dd     java.exp
 0002:00005413       $N00231                    10018413     java.exp
 0002:0000544a       $N00232                    1001844a     java.exp
 0002:00005489       $N00233                    10018489     java.exp
 0002:000054c8       $N00234                    100184c8     java.exp
 0002:00005500       $N00235                    10018500     java.exp
 0002:00005537       $N00236                    10018537     java.exp
 0002:00005576       $N00237                    10018576     java.exp
 0002:000055ad       $N00238                    100185ad     java.exp
 0002:000055e2       $N00239                    100185e2     java.exp
 0002:00005618       $N00240                    10018618     java.exp
 0002:00005657       $N00241                    10018657     java.exp
 0002:0000568f       $N00242                    1001868f     java.exp
 0002:000056cf       $N00243                    100186cf     java.exp
 0002:00005714       $N00244                    10018714     java.exp
 0002:00005758       $N00245                    10018758     java.exp
 0002:0000578c       $N00246                    1001878c     java.exp
 0002:000057c4       $N00247                    100187c4     java.exp
 0002:000057f9       $N00248                    100187f9     java.exp
 0002:0000582f       $N00249                    1001882f     java.exp
 0002:00005878       $N00250                    10018878     java.exp
 0002:000058b7       $N00251                    100188b7     java.exp
 0002:000058ed       $N00252                    100188ed     java.exp
 0002:00005924       $N00253                    10018924     java.exp
 0002:00005961       $N00254                    10018961     java.exp
 0002:000059a3       $N00255                    100189a3     java.exp
 0002:000059df       $N00256                    100189df     java.exp
 0002:00005a19       $N00257                    10018a19     java.exp
 0002:00005a50       $N00258                    10018a50     java.exp
 0002:00005a7c       $N00259                    10018a7c     java.exp
 0002:00005ac2       $N00260                    10018ac2     java.exp
 0002:00005b11       $N00261                    10018b11     java.exp
 0002:00005b66       $N00262                    10018b66     java.exp
 0002:00005bc0       $N00263                    10018bc0     java.exp
 0002:00005c0e       $N00264                    10018c0e     java.exp
 0002:00005c60       $N00265                    10018c60     java.exp
 0002:00005cb3       $N00266                    10018cb3     java.exp
 0002:00005d07       $N00267                    10018d07     java.exp
 0002:00005d58       $N00268                    10018d58     java.exp
 0002:00005da9       $N00269                    10018da9     java.exp
 0002:00005df1       $N00270                    10018df1     java.exp
 0002:00005e46       $N00271                    10018e46     java.exp
 0002:00005e92       $N00272                    10018e92     java.exp
 0002:00005ef1       $N00273                    10018ef1     java.exp
 0002:00005f3e       $N00274                    10018f3e     java.exp
 0002:00005f9a       $N00275                    10018f9a     java.exp
 0002:00005fe4       $N00276                    10018fe4     java.exp
 0002:0000602b       $N00277                    1001902b     java.exp
 0002:0000607c       $N00278                    1001907c     java.exp
 0002:000060c7       $N00279                    100190c7     java.exp
 0002:00006112       $N00280                    10019112     java.exp
 0002:00006161       $N00281                    10019161     java.exp
 0002:000061b2       $N00282                    100191b2     java.exp
 0002:000061fe       $N00283                    100191fe     java.exp
 0002:0000624b       $N00284                    1001924b     java.exp
 0002:00006295       $N00285                    10019295     java.exp
 0002:000062e3       $N00286                    100192e3     java.exp
 0002:000062f9       $N00287                    100192f9     java.exp
 0002:0000630c       $N00288                    1001930c     java.exp
 0002:00006320       $N00289                    10019320     java.exp
 0002:00006336       $N00290                    10019336     java.exp
 0002:00006342       $N00291                    10019342     java.exp
 0002:00006352       $N00292                    10019352     java.exp
 0002:0000635d       $N00293                    1001935d     java.exp
 0002:00006369       $N00294                    10019369     java.exp
 0002:000079ce       .idata$6                   1001a9ce     jvm:jvm.dll
 0002:00007af8       .idata$6                   1001aaf8     advapi32:ADVAPI32.dll
 0002:00007b48       .idata$6                   1001ab48     version:VERSION.dll
 0002:00008336       .idata$6                   1001b336     kernel32:KERNEL32.dll
 0002:000083ba       .idata$6                   1001b3ba     vcruntime:VCRUNTIME140.dll
 0002:0000862e       .idata$6                   1001b62e     ucrt:api-ms-win-crt-heap-l1-1-0.dll
 0002:0000864e       .idata$6                   1001b64e     ucrt:api-ms-win-crt-stdio-l1-1-0.dll
 0002:0000866e       .idata$6                   1001b66e     ucrt:api-ms-win-crt-string-l1-1-0.dll
 0002:00008690       .idata$6                   1001b690     ucrt:api-ms-win-crt-convert-l1-1-0.dll
 0002:000086b2       .idata$6                   1001b6b2     ucrt:api-ms-win-crt-runtime-l1-1-0.dll
 0002:000086d4       .idata$6                   1001b6d4     ucrt:api-ms-win-crt-filesystem-l1-1-0.dll
 0002:000086fa       .idata$6                   1001b6fa     ucrt:api-ms-win-crt-environment-l1-1-0.dll
 0003:00000000       _methods                   1001c000     Class.obj
 0003:00000150       _methods                   1001c150     ClassLoader.obj
 0003:0000015c       _hStdOut                   1001c15c     Console_md.obj
 0003:00000160       _hStdIn                    1001c160     Console_md.obj
 0003:00000510       _methods                   1001c510     System.obj
 0003:00000538       _methods                   1001c538     Thread.obj
 0003:000005e0       _keyNames                  1001c5e0     TimeZone_md.obj
 0003:000005f0       _methods                   1001c5f0     VM.obj
 0003:000005fc       _MAX_INPUT_EVENTS          1001c5fc     io_util_md.obj
 0003:00000600       ?curDirLenCached@?4??currentDirLength@@9@9 1001c600     io_util_md.obj
 0003:00000608       _cp1252c1chars             1001c608     jni_util.obj
 0003:00000688       _atanhi                    1001c688     fdlibm:s_atan.obj
 0003:000006a8       _atanlo                    1001c6a8     fdlibm:s_atan.obj
 0003:000006c8       _aT                        1001c6c8     fdlibm:s_atan.obj
 0003:00000720       _one                       1001c720     fdlibm:s_atan.obj
 0003:00000728       _HUGE_NUMBER               1001c728     fdlibm:s_atan.obj
 0003:00000730       _one                       1001c730     fdlibm:s_tanh.obj
 0003:00000738       _two                       1001c738     fdlibm:s_tanh.obj
 0003:00000740       _tiny                      1001c740     fdlibm:s_tanh.obj
 0003:00000748       _one                       1001c748     fdlibm:s_expm1.obj
 0003:00000750       _HUGE_NUMBER               1001c750     fdlibm:s_expm1.obj
 0003:00000758       _tiny                      1001c758     fdlibm:s_expm1.obj
 0003:00000760       _o_threshold               1001c760     fdlibm:s_expm1.obj
 0003:00000768       _ln2_hi                    1001c768     fdlibm:s_expm1.obj
 0003:00000770       _ln2_lo                    1001c770     fdlibm:s_expm1.obj
 0003:00000778       _invln2                    1001c778     fdlibm:s_expm1.obj
 0003:00000780       _Q1                        1001c780     fdlibm:s_expm1.obj
 0003:00000788       _Q2                        1001c788     fdlibm:s_expm1.obj
 0003:00000790       _Q3                        1001c790     fdlibm:s_expm1.obj
 0003:00000798       _Q4                        1001c798     fdlibm:s_expm1.obj
 0003:000007a0       _Q5                        1001c7a0     fdlibm:s_expm1.obj
 0003:000007a8       _ln2_hi                    1001c7a8     fdlibm:s_log1p.obj
 0003:000007b0       _ln2_lo                    1001c7b0     fdlibm:s_log1p.obj
 0003:000007b8       _two54                     1001c7b8     fdlibm:s_log1p.obj
 0003:000007c0       _Lp1                       1001c7c0     fdlibm:s_log1p.obj
 0003:000007c8       _Lp2                       1001c7c8     fdlibm:s_log1p.obj
 0003:000007d0       _Lp3                       1001c7d0     fdlibm:s_log1p.obj
 0003:000007d8       _Lp4                       1001c7d8     fdlibm:s_log1p.obj
 0003:000007e0       _Lp5                       1001c7e0     fdlibm:s_log1p.obj
 0003:000007e8       _Lp6                       1001c7e8     fdlibm:s_log1p.obj
 0003:000007f0       _Lp7                       1001c7f0     fdlibm:s_log1p.obj
 0003:000007f8       _one                       1001c7f8     fdlibm:e_acos.obj
 0003:00000800       _pi                        1001c800     fdlibm:e_acos.obj
 0003:00000808       _pio2_hi                   1001c808     fdlibm:e_acos.obj
 0003:00000810       _pio2_lo                   1001c810     fdlibm:e_acos.obj
 0003:00000818       _pS0                       1001c818     fdlibm:e_acos.obj
 0003:00000820       _pS1                       1001c820     fdlibm:e_acos.obj
 0003:00000828       _pS2                       1001c828     fdlibm:e_acos.obj
 0003:00000830       _pS3                       1001c830     fdlibm:e_acos.obj
 0003:00000838       _pS4                       1001c838     fdlibm:e_acos.obj
 0003:00000840       _pS5                       1001c840     fdlibm:e_acos.obj
 0003:00000848       _qS1                       1001c848     fdlibm:e_acos.obj
 0003:00000850       _qS2                       1001c850     fdlibm:e_acos.obj
 0003:00000858       _qS3                       1001c858     fdlibm:e_acos.obj
 0003:00000860       _qS4                       1001c860     fdlibm:e_acos.obj
 0003:00000868       _one                       1001c868     fdlibm:e_asin.obj
 0003:00000870       _HUGE_NUMBER               1001c870     fdlibm:e_asin.obj
 0003:00000878       _pio2_hi                   1001c878     fdlibm:e_asin.obj
 0003:00000880       _pio2_lo                   1001c880     fdlibm:e_asin.obj
 0003:00000888       _pio4_hi                   1001c888     fdlibm:e_asin.obj
 0003:00000890       _pS0                       1001c890     fdlibm:e_asin.obj
 0003:00000898       _pS1                       1001c898     fdlibm:e_asin.obj
 0003:000008a0       _pS2                       1001c8a0     fdlibm:e_asin.obj
 0003:000008a8       _pS3                       1001c8a8     fdlibm:e_asin.obj
 0003:000008b0       _pS4                       1001c8b0     fdlibm:e_asin.obj
 0003:000008b8       _pS5                       1001c8b8     fdlibm:e_asin.obj
 0003:000008c0       _qS1                       1001c8c0     fdlibm:e_asin.obj
 0003:000008c8       _qS2                       1001c8c8     fdlibm:e_asin.obj
 0003:000008d0       _qS3                       1001c8d0     fdlibm:e_asin.obj
 0003:000008d8       _qS4                       1001c8d8     fdlibm:e_asin.obj
 0003:000008e0       _tiny                      1001c8e0     fdlibm:e_atan2.obj
 0003:000008e8       _pi_o_4                    1001c8e8     fdlibm:e_atan2.obj
 0003:000008f0       _pi_o_2                    1001c8f0     fdlibm:e_atan2.obj
 0003:000008f8       _pi                        1001c8f8     fdlibm:e_atan2.obj
 0003:00000900       _pi_lo                     1001c900     fdlibm:e_atan2.obj
 0003:00000908       _two_over_pi               1001c908     fdlibm:e_rem_pio2.obj
 0003:00000a10       _npio2_hw                  1001ca10     fdlibm:e_rem_pio2.obj
 0003:00000a90       _half                      1001ca90     fdlibm:e_rem_pio2.obj
 0003:00000a98       _two24                     1001ca98     fdlibm:e_rem_pio2.obj
 0003:00000aa0       _invpio2                   1001caa0     fdlibm:e_rem_pio2.obj
 0003:00000aa8       _pio2_1                    1001caa8     fdlibm:e_rem_pio2.obj
 0003:00000ab0       _pio2_1t                   1001cab0     fdlibm:e_rem_pio2.obj
 0003:00000ab8       _pio2_2                    1001cab8     fdlibm:e_rem_pio2.obj
 0003:00000ac0       _pio2_2t                   1001cac0     fdlibm:e_rem_pio2.obj
 0003:00000ac8       _pio2_3                    1001cac8     fdlibm:e_rem_pio2.obj
 0003:00000ad0       _pio2_3t                   1001cad0     fdlibm:e_rem_pio2.obj
 0003:00000ad8       _half                      1001cad8     fdlibm:k_sin.obj
 0003:00000ae0       _S1                        1001cae0     fdlibm:k_sin.obj
 0003:00000ae8       _S2                        1001cae8     fdlibm:k_sin.obj
 0003:00000af0       _S3                        1001caf0     fdlibm:k_sin.obj
 0003:00000af8       _S4                        1001caf8     fdlibm:k_sin.obj
 0003:00000b00       _S5                        1001cb00     fdlibm:k_sin.obj
 0003:00000b08       _S6                        1001cb08     fdlibm:k_sin.obj
 0003:00000b10       _one                       1001cb10     fdlibm:k_cos.obj
 0003:00000b18       _C1                        1001cb18     fdlibm:k_cos.obj
 0003:00000b20       _C2                        1001cb20     fdlibm:k_cos.obj
 0003:00000b28       _C3                        1001cb28     fdlibm:k_cos.obj
 0003:00000b30       _C4                        1001cb30     fdlibm:k_cos.obj
 0003:00000b38       _C5                        1001cb38     fdlibm:k_cos.obj
 0003:00000b40       _C6                        1001cb40     fdlibm:k_cos.obj
 0003:00000b48       _one                       1001cb48     fdlibm:k_tan.obj
 0003:00000b50       _pio4                      1001cb50     fdlibm:k_tan.obj
 0003:00000b58       _pio4lo                    1001cb58     fdlibm:k_tan.obj
 0003:00000b60       _T                         1001cb60     fdlibm:k_tan.obj
 0003:00000bc8       _one                       1001cbc8     fdlibm:e_cosh.obj
 0003:00000bd0       _half                      1001cbd0     fdlibm:e_cosh.obj
 0003:00000bd8       _HUGE_NUMBER               1001cbd8     fdlibm:e_cosh.obj
 0003:00000be0       _one                       1001cbe0     fdlibm:e_sinh.obj
 0003:00000be8       _shuge                     1001cbe8     fdlibm:e_sinh.obj
 0003:00000bf0       _ln2_hi                    1001cbf0     fdlibm:e_log.obj
 0003:00000bf8       _ln2_lo                    1001cbf8     fdlibm:e_log.obj
 0003:00000c00       _two54                     1001cc00     fdlibm:e_log.obj
 0003:00000c08       _Lg1                       1001cc08     fdlibm:e_log.obj
 0003:00000c10       _Lg2                       1001cc10     fdlibm:e_log.obj
 0003:00000c18       _Lg3                       1001cc18     fdlibm:e_log.obj
 0003:00000c20       _Lg4                       1001cc20     fdlibm:e_log.obj
 0003:00000c28       _Lg5                       1001cc28     fdlibm:e_log.obj
 0003:00000c30       _Lg6                       1001cc30     fdlibm:e_log.obj
 0003:00000c38       _Lg7                       1001cc38     fdlibm:e_log.obj
 0003:00000c40       _two54                     1001cc40     fdlibm:e_log10.obj
 0003:00000c48       _ivln10                    1001cc48     fdlibm:e_log10.obj
 0003:00000c50       _log10_2hi                 1001cc50     fdlibm:e_log10.obj
 0003:00000c58       _log10_2lo                 1001cc58     fdlibm:e_log10.obj
 0003:00000c60       _one                       1001cc60     fdlibm:e_sqrt.obj
 0003:00000c68       _tiny                      1001cc68     fdlibm:e_sqrt.obj
 0003:00000c70       _init_jk                   1001cc70     fdlibm:k_rem_pio2.obj
 0003:00000c80       _PIo2                      1001cc80     fdlibm:k_rem_pio2.obj
 0003:00000cc0       _one                       1001ccc0     fdlibm:k_rem_pio2.obj
 0003:00000cc8       _two24                     1001ccc8     fdlibm:k_rem_pio2.obj
 0003:00000cd0       _twon24                    1001ccd0     fdlibm:k_rem_pio2.obj
 0003:00000cd8       _one                       1001ccd8     fdlibm:e_exp.obj
 0003:00000ce0       _halF                      1001cce0     fdlibm:e_exp.obj
 0003:00000cf0       _HUGE_NUMBER               1001ccf0     fdlibm:e_exp.obj
 0003:00000cf8       _twom1000                  1001ccf8     fdlibm:e_exp.obj
 0003:00000d00       _o_threshold               1001cd00     fdlibm:e_exp.obj
 0003:00000d08       _u_threshold               1001cd08     fdlibm:e_exp.obj
 0003:00000d10       _ln2HI                     1001cd10     fdlibm:e_exp.obj
 0003:00000d20       _ln2LO                     1001cd20     fdlibm:e_exp.obj
 0003:00000d30       _invln2                    1001cd30     fdlibm:e_exp.obj
 0003:00000d38       _P1                        1001cd38     fdlibm:e_exp.obj
 0003:00000d40       _P2                        1001cd40     fdlibm:e_exp.obj
 0003:00000d48       _P3                        1001cd48     fdlibm:e_exp.obj
 0003:00000d50       _P4                        1001cd50     fdlibm:e_exp.obj
 0003:00000d58       _P5                        1001cd58     fdlibm:e_exp.obj
 0003:00000d60       _one                       1001cd60     fdlibm:e_fmod.obj
 0003:00000d68       _Zero                      1001cd68     fdlibm:e_fmod.obj
 0003:00000d78       _HUGE_NUMBER               1001cd78     fdlibm:s_floor.obj
 0003:00000d80       _two54                     1001cd80     fdlibm:s_scalbn.obj
 0003:00000d88       _twom54                    1001cd88     fdlibm:s_scalbn.obj
 0003:00000d90       _HUGE_NUMBER               1001cd90     fdlibm:s_scalbn.obj
 0003:00000d98       _tiny                      1001cd98     fdlibm:s_scalbn.obj
 0003:00000dcc       _handleID                  1001cdcc     NativeLibraries.obj
 0003:00000dd0       _jniVersionID              1001cdd0     NativeLibraries.obj
 0003:00000dd4       _procHandle                1001cdd4     NativeLibraries.obj
 0003:00000dd8       _noSuchMethodErrCl         1001cdd8     ObjectStreamClass.obj
 0003:00000ddc       _ProcessHandleImpl_Info_commandID 1001cddc     ProcessHandleImpl_win.obj
 0003:00000de0       _ProcessHandleImpl_Info_commandLineID 1001cde0     ProcessHandleImpl_win.obj
 0003:00000de4       _ProcessHandleImpl_Info_argumentsID 1001cde4     ProcessHandleImpl_win.obj
 0003:00000de8       _ProcessHandleImpl_Info_totalTimeID 1001cde8     ProcessHandleImpl_win.obj
 0003:00000dec       _ProcessHandleImpl_Info_startTimeID 1001cdec     ProcessHandleImpl_win.obj
 0003:00000df0       _ProcessHandleImpl_Info_userID 1001cdf0     ProcessHandleImpl_win.obj
 0003:00000df4       ?initField@?1??check@@9@9  1001cdf4     SecurityManager.obj
 0003:00000df8       _ids                       1001cdf8     WinNTFileSystem_md.obj
 0003:00000dfc       _GetFinalPathNameByHandle_func 1001cdfc     WinNTFileSystem_md.obj
 0003:00000e00       ?u_path@?1??getHomeFromShell32@@9@9 1001ce00     java_props_md.obj
 0003:00000e08       ?sprops@?1??GetJavaProperties@@9@9 1001ce08     java_props_md.obj
 0003:00000e74       _fastEncoding              1001ce74     jni_util.obj
 0003:00000e78       _jnuEncoding               1001ce78     jni_util.obj
 0003:00000e7c       _String_init_ID            1001ce7c     jni_util.obj
 0003:00000e80       _String_getBytes_ID        1001ce80     jni_util.obj
 0003:00000e84       _String_coder_ID           1001ce84     jni_util.obj
 0003:00000e88       _String_value_ID           1001ce88     jni_util.obj
 0003:00000e8c       _isJNUEncodingSupported    1001ce8c     jni_util.obj
 0003:00000e90       ?cls@?1??JNU_ClassString@@9@9 1001ce90     jni_util.obj
 0003:00000e98       _zero                      1001ce98     fdlibm:s_log1p.obj
 0003:00000ea0       _zero                      1001cea0     fdlibm:e_atan2.obj
 0003:00000ea8       _zero                      1001cea8     fdlibm:e_rem_pio2.obj
 0003:00000eb0       _zero                      1001ceb0     fdlibm:e_log.obj
 0003:00000eb8       _zero                      1001ceb8     fdlibm:e_log10.obj
 0003:00000ec0       _zero                      1001cec0     fdlibm:e_remainder.obj
 0003:00000ec8       _zero                      1001cec8     fdlibm:k_rem_pio2.obj
 0003:00000ef0       _GS_ExceptionRecord        1001cef0     MSVCRT:gs_report.obj
 0003:00000f40       _GS_ContextRecord          1001cf40     MSVCRT:gs_report.obj
 0003:0000120c       ?__proc_attached@@3HA      1001d20c     MSVCRT:dll_dllmain.obj
 0003:00001220       ?is_initialized_as_dll@@3_NA 1001d220     MSVCRT:utility.obj
 0003:00001221       ?module_local_atexit_table_initialized@@3_NA 1001d221     MSVCRT:utility.obj
 0003:00001224       ?module_local_atexit_table@@3U_onexit_table_t@@A 1001d224     MSVCRT:utility.obj
 0003:00001230       ?module_local_at_quick_exit_table@@3U_onexit_table_t@@A 1001d230     MSVCRT:utility.obj
 0004:00000060       $R000000                   1001e060     java.dll.res
